:100000000C94AA510C9409520C9409520C94095264
:100010000C9409520C9409520C9409520C940952F4
:100020000C9409520C9409520C9409520C940952E4
:100030000C9409520C9480520C94BF520C940952A7
:100040000C9409520C9409520C9409520C940952C4
:100050000C9409520C9409520C9409520C940952B4
:100060000C9409520C9409520C9409520C940952A4
:100070005A5501200101003808000000000000006E
:100080000000000000000000000000000000000070
:10009000810045005DFF5E1027FF2AD22B7D210CD9
:1000A00022FB850084008903888D81096F02444208
:1000B00047004501B083B300B10124B925578A1D1B
:1000C0008B03AD55B055B855BC55C355CB55D05520
:1000D000D555D855E855EB55EE5529562C562F5683
:1000E000FFFFFFFFFFF7FFFFFFFFFFF7FFF7F7F748
:1000F000F7EFFFF7F7F7F7EFFFF7F7F7F7EFFFF790
:10010000F7F7F7EFFFF7F7F7F7EFFFF7F7F7F7EF87
:10011000FFF7F7F7F7EFFFF7F7F7F7EFFFF7F7F767
:10012000F7EFFFF7F7F7F7EFFFF7F7F7F7EFFFF75F
:10013000F7F7F7EFF7EFEFEFEFEFF7EFEFEFEFEFA7
:10014000FFFFFFFFFFF7FFFFFFFFFFF7FFF7F7F7E7
:10015000F7EFFFF7F7F7F7EFFFF7F7F7F7EFFFF72F
:10016000F7F7F7EFFFF7F7F7F7EFFFF7F7F7F7EF27
:10017000FFF7F7F7F7EFFFF7F7F7F7EFFFF7F7F707
:10018000F7EFFFF7F7F7F7EFFFF7F7F7F7EFFFF7FF
:10019000F7F7F7EFF7EFEFEFEFEFF7EFEFEFEFEF47
:1001A000FFFFFFFFFFF7FFFFFFFFFFF7FFF7F7F787
:1001B000F7EFFFF7F7F7F7EFFFF7F7F7F7EFEFF7DF
:1001C000F7F7F7EFFFF7F7F7EF0000EFF7F7F7EFC5
:1001D000FFF7F7EF00000000EFF7F7EFFFF7EF0092
:1001E0000000000000FFF7EFFFEF0000000000003C
:1001F0000000FFEFEF00000000000000000000FF23
:10020000EF00000000000000000000FFFFEF000012
:10021000000000000000FFEFFFF7EF00000000000B
:1002200000FFF7EFFFF7F7FF00000000FFF7F7EF21
:10023000FFF7F7F7FF0000FFF7F7F7EFFFF7F7F724
:10024000F7FFFFF7F7F7F7EFFFF7F7F7F7EFFFF72E
:10025000F7F7F7EFF7EFEFEFEFEFF7EFEFEFEFEF86
:10026000FFFFFFFFFFF7FFFFFFFFFFF7FFF7F7F7C6
:10027000F7EFFFF7F7F7F7EFFFF7F7F7F7EFFFF70E
:10028000F7F7F7EFFFF7F7F7F7EFFFF7F7F7F7EF06
:10029000FFF7F7F7F7A5A5F7F7F7F7EFFFF7F7F78A
:1002A000A55C5CA5F7F7F7EFFFF7F7A55CA5A55CE4
:1002B0000AF7F7EFF7EFA55CA55C5C0A5C0AEFEFC5
:1002C000FFFFA55CA55C5C0A5C0AFFF7FFF7F7A5DA
:1002D0005C0A0A5C0AF7F7EFFFF7F7F70A5C5C0ABB
:1002E000F7F7F7EFFFF7F7F7F70A0AF7F7F7F7EF80
:1002F000FFF7F7F7F7EFFFF7F7F7F7EFFFF7F7F786
:10030000F7EFFFF7F7F7F7EFFFF7F7F7F7EFFFF77D
:10031000F7F7F7EFF7EFEFEFEFEFF7EFEFEFEFEFC5
:10032000FFFFFFFFFFF7FFFFFFFFFFF7FFF7F7F705
:10033000F7EFFFF7F7F7F7EFFFF7F7F7F7EFEFF75D
:10034000F7F7F7EFFFF7F7F7EF0000EFF7F7F7EF43
:10035000FFF7F7EF00383800EFF7F7EFFFF7EF00A0
:100360003820203800FFF7EFFFEF00382038382022
:100370000800FFEFEF00382038202008200800FF99
:10038000EF00382038202008200800FFFFEF003859
:10039000200808200800FFEFFFF7EF0008202008E2
:1003A00000FFF7EFFFF7F7FF00080800FFF7F7EF90
:1003B000FFF7F7F7FF0000FFF7F7F7EFFFF7F7F7A3
:1003C000F7FFFFF7F7F7F7EFFFF7F7F7F7EFFFF7AD
:1003D000F7F7F7EFF7EFEFEFEFEFF7EFEFEFEFEF05
:1003E000000000000000000000000000000000000D
:1003F00000000000000000000000000000000000FD
:1004000000000000000000000000000000000000EC
:1004100000000000000000000000000000000000DC
:1004200000000000000000000000000000000000CC
:1004300000000000000000000000000000000000BC
:1004400000000000000000000000000000000000AC
:10045000000000000000000000000000000000009C
:10046000000000000000000000000000000000008C
:10047000000000000000000000000000000000007C
:10048000000000000000000000000000000000006C
:10049000000000000000000000000000000000005C
:1004A00006060606060306060606060603030303FB
:1004B000030106030303030303030303030106030A
:1004C00003030303030303030301060303030303FB
:1004D00003030303030106030303030303030303EB
:1004E00003010603030303030303030303010603DA
:1004F00003030303010101010101030101010101E2
:100500000606060606060606060606030603030397
:1005100003030303030303010603030303030303AA
:10052000030303010603030303030303030303019C
:100530000603030303030303030303010603030387
:10054000030303030303030106030303030303037A
:100550000303030103010101010101010101010183
:10056000FFFFFFFFFFF7FFFFFFFFFFF7FFF7F7F7C3
:10057000F7EFFFF7F7F7F7EFFFF7F7F7F72525F7AF
:10058000F7F7F7EFFFF7F7F725252513F7F7F7EF5D
:10059000FFF7F7F725252513F7F7F7EFFFF7F7F73D
:1005A000F71313F7F7F7F7EFFFF7F7F76A6A6A1829
:1005B000F7F7F7EFF7EFEF6A6A6A6A1818EFEFEFED
:1005C000FFFF6AFF6A6A6A18FF18FFF7FFF76AF70A
:1005D00018181818F718F7EFFFF76AF7C180C180ED
:1005E000F718F7EFFFF7F7F7C180C180F7F7F7EFDC
:1005F000FFF7F7F7C180C180F7F7F7EFFFF7F7F7DD
:10060000C180C180F7F7F7EFFFF7F7F75C0A5C0AE4
:10061000F7F7F7EFF7EFEFEFEFEFF7EFEFEFEFEFC2
:10062000FFFFFFFFFFF7FFFFFFFFFFF7FFF7F7F702
:10063000F7EFFFF7F7F7F7EFFFF7F7F7F72525F7EE
:10064000F7F7F7EFFFF7F7F725252513F7F7F7EF9C
:10065000FFF7F7EF25252513EFF7F7EFFFF7EF008B
:100660000013130000FFF7EFFFEF00006A6A6A183B
:100670000000FFEFEF00006A6A6A6A18180000FFC6
:10068000EF006A006A6A6A18001800FFFFEF6A004C
:10069000181818180018FFEFFFF76A00C180C18012
:1006A0000018F7EFFFF7F7FFC180C180FFF7F7EF02
:1006B000FFF7F7F7C180C180F7F7F7EFFFF7F7F71C
:1006C000C180C180F7F7F7EFFFF7F7F75C0A5C0A24
:1006D000F7F7F7EFF7EFEFEFEFEFF7EFEFEFEFEF02
:1006E000000000000000000000000000000000000A
:1006F00000000000000000000000000000000000FA
:1007000000000000000000000000000000000000E9
:1007100000000000000000000000000000000000D9
:10072000000000000000F8000000000000000000D1
:100730000000F800000000000000F8F8F8F8F800E9
:1007400000000000000000000000000000000000A9
:100750000000F8F8F8F800000000000000000000B9
:100760000000F800000000000000F8F8F8F80000B1
:100770000000000000000000000000000000000079
:10078000000000000000F800000000000000000071
:100790000000F800000000000000F8F8F8F8F80089
:1007A0000000000000000000000000000000000049
:1007B0000000F800F800F800000000000000F80059
:1007C000F800F800000000000000F8F8F8F8F80061
:1007D0000000000000000000000000000000000019
:1007E0000000F8F8F8F80000000000000000000029
:1007F0000000F800000000000000F8F8F8F8000021
:1008000000000000000000000000000000000000E8
:100810000000F8F8F8F8F800000000000000F80008
:100820000000F800000000000000F8F8F8F8F800F8
:1008300000000000000000000000000000000000B8
:100840000000F8F8F8F8F80000000000000000F8D8
:1008500000000000000000000000F8F8F8F8F800C0
:100860000000000000000000000000000000000088
:100870000000F8F8F8F8F8000000000000000000A0
:10088000F8000000000000000000F8F8F8F8F80098
:100890000000000000000000000000000000000058
:1008A0000000F800F8F8F800000000000000F80070
:1008B000F800F800000000000000F8F8F800F80068
:1008C0000000000000000000000000000000000028
:1008D0000000F8F8F8F8F800000000000000000040
:1008E0000000F800000000000000F8F8F8F8F80038
:1008F00000000000000000000000000000000000F8
:100900000000F8F8F8000000000000000000F80007
:10091000F8000000000000000000F8F8F8F8F80007
:10092000000000000000000000000000000000FFC8
:10093000FFFFFFFFFFFF000000FF0000FFFFFFFFC2
:10094000FF0000FF00FFFF00000000000000FFFFAD
:1009500000FFFF00000000000000FFFF00FFFF009D
:10096000000000000000FFFF00FF0000000000008A
:10097000000000FF00000000000000000000000078
:100980000000000000000000000000000000000067
:10099000000000000000000000FF00000000000058
:1009A000000000FF00FFFF00000000000000FFFF4C
:1009B00000FFFF00000000000000FFFF00FFFF003D
:1009C000000000000000FFFF00FF0000FFFFFFFF2E
:1009D000FF0000FF000000FFFFFFFFFFFFFF000020
:1009E0000000000000000000000000000000000007
:1009F00000000000000000000000000000000000F7
:100A0000000000FF00000000000000000000FFFFE9
:100A100000000000000000000000FFFF00000000D8
:100A2000000000000000FFFF0000000000000000C8
:100A3000000000FF000000000000000000000000B7
:100A400000000000000000000000000000000000A6
:100A50000000000000000000000000000000000096
:100A6000000000FF00000000000000000000FFFF89
:100A700000000000000000000000FFFF0000000078
:100A8000000000000000FFFF000000000000000068
:100A9000000000FF00000000000000000000000057
:100AA000000000000000000000000000000000FF47
:100AB000FFFFFFFFFFFF000000000000FFFFFFFF40
:100AC000FF0000FF00000000000000000000FFFF2A
:100AD00000000000000000000000FFFF0000000018
:100AE000000000000000FFFF000000000000000008
:100AF000000000FF000000FFFFFFFFFFFFFF0000FE
:100B00000000FFFFFFFFFFFFFFFFFF00000000FFEF
:100B1000FFFFFFFFFFFF000000FF000000000000DC
:100B20000000000000FFFF000000000000000000C7
:100B300000FFFF00000000000000000000FFFF00B9
:100B4000000000000000000000FF0000FFFFFFFFAA
:100B5000FF000000000000FFFFFFFFFFFFFF00009D
:100B6000000000000000000000000000000000FF86
:100B7000FFFFFFFFFFFF000000000000FFFFFFFF7F
:100B8000FF0000FF00000000000000000000FFFF69
:100B900000000000000000000000FFFF0000000057
:100BA000000000000000FFFF000000000000000047
:100BB000000000FF000000FFFFFFFFFFFFFF00003D
:100BC0000000FFFFFFFFFFFFFFFFFF00000000FF2F
:100BD000FFFFFFFFFFFF000000000000000000001B
:100BE000000000FF00000000000000000000FFFF08
:100BF00000000000000000000000FFFF00000000F7
:100C0000000000000000FFFF00000000FFFFFFFFEA
:100C1000FF0000FF000000FFFFFFFFFFFFFF0000DD
:100C200000000000000000000000000000000000C4
:100C3000000000000000000000FF000000000000B5
:100C4000000000FF00FFFF00000000000000FFFFA9
:100C500000FFFF00000000000000FFFF00FFFF009A
:100C6000000000000000FFFF00FF00000000000087
:100C7000000000FF000000FFFFFFFFFFFFFF00007C
:100C80000000FFFFFFFFFFFFFFFFFF00000000FF6E
:100C9000FFFFFFFFFFFF000000000000000000005A
:100CA000000000FF00000000000000000000FFFF47
:100CB00000000000000000000000FFFF0000000036
:100CC000000000000000FFFF000000000000000026
:100CD000000000FF00000000000000000000000015
:100CE000000000000000000000000000000000FF05
:100CF000FFFFFFFFFFFF000000FF0000FFFFFFFFFF
:100D0000FF00000000FFFF000000000000000000E6
:100D100000FFFF00000000000000000000FFFF00D7
:100D2000000000000000000000FF000000000000C4
:100D300000000000000000FFFFFFFFFFFFFF0000BA
:100D40000000FFFFFFFFFFFFFFFFFF00000000FFAD
:100D5000FFFFFFFFFFFF0000000000000000000099
:100D6000000000FF00000000000000000000FFFF86
:100D700000000000000000000000FFFF0000000075
:100D8000000000000000FFFF00000000FFFFFFFF69
:100D9000FF0000FF000000FFFFFFFFFFFFFF00005C
:100DA000000000000000000000000000000000FF44
:100DB000FFFFFFFFFFFF000000FF0000FFFFFFFF3E
:100DC000FF00000000FFFF00000000000000000026
:100DD00000FFFF00000000000000000000FFFF0017
:100DE000000000000000000000FF00000000000004
:100DF00000000000000000FFFFFFFFFFFFFF0000FA
:100E00000000FFFFFFFFFFFFFFFFFF00000000FFEC
:100E1000FFFFFFFFFFFF000000FF000000000000D9
:100E2000000000FF00FFFF00000000000000FFFFC7
:100E300000FFFF00000000000000FFFF00FFFF00B8
:100E4000000000000000FFFF00FF0000FFFFFFFFA9
:100E5000FF0000FF000000FFFFFFFFFFFFFF00009B
:100E6000000000000000000000000000000000FF83
:100E7000FFFFFFFFFFFF000000000000FFFFFFFF7C
:100E8000FF0000FF00000000000000000000FFFF66
:100E900000000000000000000000FFFF0000000054
:100EA000000000000000FFFF000000000000000044
:100EB000000000FF00000000000000000000000033
:100EC0000000000000000000000000000000000022
:100ED0000000000000000000000000000000000012
:100EE000000000FF00000000000000000000FFFF05
:100EF00000000000000000000000FFFF00000000F4
:100F0000000000000000FFFF0000000000000000E3
:100F1000000000FF000000000000000000000000D2
:100F2000000000000000000000000000000000FFC2
:100F3000FFFFFFFFFFFF000000FF0000FFFFFFFFBC
:100F4000FF0000FF00FFFF00000000000000FFFFA7
:100F500000FFFF00000000000000FFFF00FFFF0097
:100F6000000000000000FFFF00FF00000000000084
:100F7000000000FF000000FFFFFFFFFFFFFF000079
:100F80000000FFFFFFFFFFFFFFFFFF00000000FF6B
:100F9000FFFFFFFFFFFF000000FF00000000000058
:100FA000000000FF00FFFF00000000000000FFFF46
:100FB00000FFFF00000000000000FFFF00FFFF0037
:100FC000000000000000FFFF00FF0000FFFFFFFF28
:100FD000FF0000FF000000FFFFFFFFFFFFFF00001A
:100FE000000000000000000000000000000000FF02
:100FF000FFFFFFFFFFFF000000FF0000FFFFFFFFFC
:10100000FF0000FF00FFFF00000000000000FFFFE6
:1010100000FFFF00000000000000FFFF00FFFF00D6
:10102000000000000000FFFF00FF000000000000C3
:10103000000000FF000000FFFFFFFFFFFFFF0000B8
:101040000000FFFFFFFFFFFFFFFFFF00000000FFAA
:10105000FFFFFFFFFFFF0000000000000000000096
:10106000000000FF00000000000000000000FFFF83
:1010700000000000000000000000FFFF0000000072
:10108000000000000000FFFF00000000FFFFFFFF66
:10109000FF0000FF000000FFFFFFFFFFFFFF000059
:1010A0000000000000000000000000000000000040
:1010B0000000000000000000000000000000000030
:1010C0000000000000000000000000000000000020
:1010D0000000000000000000000000000000000010
:1010E000000000000000000000FFFFFFFFFFFFFF07
:1010F0000000000000FF0000000000FF00000000F2
:1011000000FF0000000000FF0000000000FF0000E2
:10111000000000FF0000000000FF0000000000FFD2
:101120000000000000FF0000000000FF00000000C1
:1011300000FF0000000000FF0000000000FFFFFFB4
:10114000FFFFFFFF000000000000000000000000A3
:10115000000000000000000000000000000000008F
:10116000000000000000000000000000000000007F
:10117000000000000000000000000000000000006F
:10118000000000000000000000000000000000005F
:101190000000000000000000000000380000000017
:1011A000000000000000383800FFFFFFFFFFFFFFD6
:1011B0000038380038FF0000000000FF3838000019
:1011C00038380000000000383800000000383800CF
:1011D000000038380000000000FF3838003838FFC1
:1011E0000000000000FF0038383800FF0000000059
:1011F00000FF0000380000FF0000000000FFFFFFBC
:10120000FFFFFFFF000000000000000000000000E2
:1012100000000000000000000000000000000000CE
:101220000707070707070707070707070700000063
:1012300000000000000000070700000000000000A0
:101240000000000707000000000000000000000789
:101250000700000000000000000000070700000079
:10126000000000000000000707FFFFFFFFFFFFFF77
:101270000000000707FF0000000000FF000000075B
:1012800007FF0000000000FF0000000707FF00004C
:10129000000000FF0000000707FF0000000000FF43
:1012A0000000000707FF0000000000FF000000072B
:1012B00007FF0000000000FF0000000707FFFFFF1E
:1012C000FFFFFFFF00000007070000000000000014
:1012D00000000007070707070707070707070707B3
:1012E00007070707070707070707070707000000A3
:1012F00000000000000000070700000000000000E0
:1013000000000007070000000000000000000007C8
:1013100007000000000000000000000707000000B8
:10132000000000000000380707FFFFFFFFFFFFFF7E
:101330000038380707FF0000000000FF38380007BA
:101340000738000000000038380000070738380070
:10135000000038380000000707FF3838003838FF31
:101360000000000707FF0038383800FF00000007C2
:1013700007FF0000380000FF0000000707FFFFFF25
:10138000FFFFFFFF00000007070000000000000053
:1013900000000007070707070707070707070707F2
:1013A000C7C7C7C7C7C7C7C7C7C7C7C7C7C7C7C7CD
:1013B000C7C7C7C7C7C7C7C7C7C7C7C7C7C7C7C7BD
:1013C000C7C7C7C7C7C7C7C7C7C7C7C7C7C7C7C7AD
:1013D000C7C7C7C7C7C7C7C7C7C7C7C7C7C7C7C79D
:1013E000C7C7C7C7C7C7C7C7C7C7C7C7C7C7C7C78D
:1013F000C7C7C7C7C7C7C7C7C7C7C7C7C7C7C7C77D
:10140000C7C7C7C7C7C7C7C7C7C7C7C7C7C7C7C76C
:10141000C7C7C7C7C7C7C7C7C7C7C7C7C7C7C7C75C
:10142000C7C7C7C7C7C7C7C7C7C7C7C7C7C7C7C74C
:10143000C7C7C7C7C7C7C7C7C7C7C7C7C7C7C7C73C
:10144000C7C7C7C7C7C7C7C7C7C7C7C7C7C7C7C72C
:10145000C7C7C7C7C7C7C7C7C7C7C7C7C7C7C7C71C
:10146000000000000000000000000000000000007C
:101470000000000000000000FFFF0000000000006E
:10148000FFFF0000FFFFFFFF0000FFFFFFFF000066
:10149000FFFFFFFF0000FFFFFFFF0000FFFF000056
:1014A000FFFF0000FFFF0000FFFF0000FFFF000044
:1014B000FFFF0000FFFF000000000000FFFF000032
:1014C000FFFF000000000000FFFF0000FFFF000022
:1014D00000000000FFFF0000FFFF00000000000010
:1014E000FFFF0000FFFF000000000000FFFF000002
:1014F000FFFF000000000000FFFF000000000000F0
:1015000000000000000000000000000000000000DB
:1015100000000000000000000000000000000000CB
:1015200000000000000000000000000000000000BB
:1015300000000000000000000000000000000000AB
:10154000000000000000000000000000000000009B
:10155000000000000000000000000000000000008B
:10156000FFFFFFFF000000000000FFFF0000000081
:10157000FFFF00000000FFFF00000000FFFF000071
:101580000000FFFF00000000FFFF00000000FFFF61
:10159000FFFFFFFFFFFF00000000FFFF0000000053
:1015A000000000000000FFFF00000000FFFF00003F
:1015B00000000000FFFFFFFF00000000000000002F
:1015C000000000000000000000000000000000001B
:1015D000000000000000000000000000000000000B
:1015E00000000000000000000000000000000000FB
:1015F00000000000000000000000000000000000EB
:1016000000000000000000000000000000000000DA
:1016100000000000000000000000000000000000CA
:10162000FFFFFFFFFFFF00000000FFFF00000000C2
:10163000FFFF00000000FFFF00000000FFFF0000B0
:101640000000FFFF00000000FFFF00000000FFFFA0
:1016500000000000FFFF00000000FFFF000000008E
:10166000FFFF00000000FFFF00000000FFFF000080
:1016700000000000FFFFFFFFFFFF00000000000070
:1016800000000000FFFF000000000000000000005C
:10169000FFFF00000000FFFFFFFFFFFF0000000052
:1016A000000000000000000000000000000000003A
:1016B000000000000000000000000000000000002A
:1016C000000000000000000000000000000000001A
:1016D000000000000000000000000000000000000A
:1016E000FFFFFFFF000000000000000000000000FE
:1016F000FFFF00000000000000000000FFFF0000EE
:1017000000000000FFFFFFFFFFFF00000000FFFFE1
:1017100000000000FFFF00000000FFFF00000000CD
:10172000FFFF00000000FFFF00000000FFFF0000BF
:1017300000000000FFFFFFFFFFFF000000000000AF
:101740000000000000000000000000000000000099
:101750000000000000000000000000000000000089
:101760000000000000000000000000000000000079
:10177000000000000000000000000000FFFFFFFF6D
:10178000000000000000FFFF00000000FFFF00005D
:101790000000FFFF00000000000000000000FFFF4D
:1017A00000000000000000000000FFFF000000003B
:1017B0000000000000000000FFFFFFFF000000002D
:1017C0000000000000000000FFFF0000000000001B
:1017D00000000000FFFF000000000000000000000B
:1017E000FFFF00000000FFFF00000000FFFF0000FF
:1017F00000000000FFFFFFFF0000000000000000ED
:1018000000000000000000000000000000000000D8
:1018100000000000000000000000000000000000C8
:1018200000000000000000000000000000000000B8
:1018300000000000000000000000000000000000A8
:101840000000000000000000000000000000000098
:101850000000000000000000000000000000000088
:10186000FFFFFFFF000000000000FFFF000000007E
:10187000FFFF00000000FFFF00000000FFFF00006E
:101880000000FFFF00000000FFFF00000000FFFF5E
:1018900000000000FFFF00000000FFFF000000004C
:1018A000FFFF00000000FFFF00000000FFFF00003E
:1018B00000000000FFFFFFFF00000000000000002C
:1018C0000000000000000000000000000000000018
:1018D0000000000000000000000000000000000008
:1018E00000000000000000000000000000000000F8
:1018F00000000000000000000000FFFF00000000EA
:10190000000000000000FFFF0000000000000000D9
:101910000000FFFF00000000000000000000FFFFCB
:1019200000000000FFFF00000000FFFF0000FFFFBD
:10193000000000000000FFFFFFFF000000000000AB
:101940000000FFFF00000000000000000000FFFF9B
:10195000FFFF0000000000000000FFFF0000FFFF8D
:10196000000000000000FFFF00000000FFFF00007B
:101970000000FFFF00000000FFFF0000000000006B
:101980000000000000000000000000000000000057
:101990000000000000000000000000000000000047
:1019A0000000000000000000000000000000000037
:1019B00000000000000000000000FFFF0000000029
:1019C000000000000000FFFF000000000000000019
:1019D0000000FFFF00000000000000000000FFFF0B
:1019E000FFFFFFFF000000000000FFFF00000000FD
:1019F000FFFF00000000FFFF00000000FFFF0000ED
:101A00000000FFFF00000000FFFF00000000FFFFDC
:101A100000000000FFFF00000000FFFF00000000CA
:101A2000FFFF00000000FFFF00000000FFFF0000BC
:101A30000000FFFFFFFFFFFF0000000000000000AC
:101A40000000000000000000000000000000000096
:101A50000000000000000000000000000000000086
:101A60000000000000000000000000000000000076
:101A70000000000000000000000000000000000066
:101A80000000000000000000000000000000000056
:101A90000000000000000000000000000000FFFF48
:101AA000FFFFFFFF000000000000FFFF000000003C
:101AB000FFFF00000000FFFF00000000FFFF00002C
:101AC0000000FFFF00000000FFFF00000000FFFF1C
:101AD00000000000FFFF00000000FFFF000000000A
:101AE000FFFF00000000FFFF00000000FFFF0000FC
:101AF0000000FFFF00000000FFFF000000000000EA
:101B000000000000000000000000000000000000D5
:101B100000000000000000000000000000000000C5
:101B200000000000000000000000000000000000B5
:101B300000000000000000000000000000000000A5
:101B40000000000000000000000000000000000095
:101B50000000000000000000000000000000000085
:101B60000000000000000000000000000000000075
:101B70000000000000000000000000000000000065
:101B80000000000000000000000000000000000055
:101B90000000000000000000000000000000000045
:101BA0000000000000000000000000000000000035
:101BB0000000000000000000000000000000000025
:101BC0000000000000000000000000000000000015
:101BD0000000000000000000000000000000000005
:101BE00000000000000000000000000000000000F5
:101BF000000000000000000000000000FFFFFFFFE9
:101C0000000000000000FFFF00000000FFFF0000D8
:101C10000000FFFF00000000FFFF000000000000C8
:101C200000000000FFFF00000000000000000000B6
:101C3000FFFF00000000000000000000FFFF0000A8
:101C4000000000000000FFFF000000000000000096
:101C5000FFFF0000000000000000FFFF0000000088
:101C6000000000000000FFFF000000000000000076
:101C70000000FFFFFFFFFFFFFFFF0000000000006C
:101C80000000000000000000000000000000000054
:101C90000000000000000000000000000000000044
:101CA0000000000000000000000000000000000034
:101CB000000000000000000000000000FFFFFFFF28
:101CC000000000000000FFFF00000000FFFF000018
:101CD0000000FFFF00000000FFFF00000000FFFF0A
:101CE0000000FFFFFFFF00000000FFFF0000FFFFFC
:101CF000FFFF00000000FFFFFFFF0000FFFF0000EC
:101D00000000FFFFFFFF0000FFFF00000000FFFFDB
:101D100000000000FFFF00000000FFFF00000000C7
:101D2000FFFF00000000FFFF00000000FFFF0000B9
:101D300000000000FFFFFFFF0000000000000000A7
:101D40000000000000000000000000000000000093
:101D50000000000000000000000000000000000083
:101D60000000000000000000000000000000000073
:101D70000000000000000000000000000000FFFF65
:101D80000000000000000000FFFFFFFF0000000057
:101D90000000FFFF0000FFFF000000000000000047
:101DA0000000FFFF00000000000000000000FFFF37
:101DB00000000000000000000000FFFF0000000025
:101DC000000000000000FFFF000000000000000015
:101DD0000000FFFF00000000000000000000FFFF07
:101DE00000000000000000000000FFFF00000000F5
:101DF0000000FFFFFFFFFFFFFFFF000000000000EB
:101E000000000000000000000000000000000000D2
:101E100000000000000000000000000000000000C2
:101E200000000000000000000000000000000000B2
:101E30000000000000000000000000000000FFFFA4
:101E40000000000000000000000000000000000092
:101E50000000000000000000000000000000000082
:101E6000FFFFFFFF00000000000000000000FFFF78
:101E700000000000000000000000FFFF0000000064
:101E8000000000000000FFFF000000000000000054
:101E90000000FFFF00000000000000000000FFFF46
:101EA00000000000000000000000FFFF0000000034
:101EB00000000000FFFFFFFFFFFF00000000000028
:101EC0000000000000000000000000000000000012
:101ED0000000000000000000000000000000000002
:101EE00000000000000000000000000000000000F2
:101EF00000000000000000000000000000000000E2
:101F0000FFFF00000000000000000000FFFF0000D5
:101F10000000000000000000FFFF000000000000C3
:101F2000FFFFFFFFFFFF00000000FFFF00000000B9
:101F3000FFFF00000000FFFF00000000FFFF0000A7
:101F40000000FFFF00000000FFFF00000000FFFF97
:101F500000000000FFFF00000000FFFF0000000085
:101F6000FFFF00000000FFFF00000000FFFF000077
:101F700000000000FFFFFFFFFFFF00000000000067
:101F80000000000000000000000000000000000051
:101F90000000000000000000000000000000000041
:101FA0000000000000000000000000000000000031
:101FB00000000000000000000000FFFF0000000023
:101FC000FFFF00000000FFFF00000000FFFF000017
:101FD0000000FFFF00000000FFFF00000000FFFF07
:101FE00000000000FFFF00000000FFFF00000000F5
:101FF000FFFF00000000FFFFFFFFFFFFFFFF0000EB
:102000000000FFFF00000000FFFF00000000FFFFD6
:1020100000000000FFFF00000000FFFF00000000C4
:10202000FFFF00000000FFFF00000000FFFF0000B6
:102030000000FFFF00000000FFFF000000000000A4
:102040000000000000000000000000000000000090
:102050000000000000000000000000000000000080
:102060000000000000000000000000000000000070
:102070000000000000000000000000000000000060
:102080000000000000000000000000000000000050
:102090000000000000000000000000000000FFFF42
:1020A0000000FFFFFFFF00000000FFFFFFFF000038
:1020B000000000000000FFFF000000000000000022
:1020C0000000FFFF00000000000000000000FFFF14
:1020D00000000000000000000000FFFF0000000002
:1020E000000000000000FFFF0000000000000000F2
:1020F0000000FFFF000000000000000000000000E2
:1021000000000000000000000000000000000000CF
:1021100000000000000000000000000000000000BF
:1021200000000000000000000000000000000000AF
:10213000000000000000000000000000000000009F
:10214000000000000000000000000000000000008F
:102150000000000000000000000000000000FFFF81
:1021600000000000FFFF00000000FFFF0000000073
:10217000FFFF00000000FFFF00000000FFFF000065
:102180000000FFFF00000000FFFF00000000FFFF55
:1021900000000000FFFF00000000FFFF0000000043
:1021A000FFFF00000000FFFF00000000FFFF000035
:1021B00000000000FFFFFFFFFFFF00000000000025
:1021C000000000000000000000000000000000000F
:1021D00000000000000000000000000000000000FF
:1021E00000000000000000000000000000000000EF
:1021F000000000000000000000000000FFFFFFFFE3
:10220000FFFF0000000000000000FFFF00000000D2
:10221000000000000000FFFF0000000000000000C0
:102220000000FFFF00000000000000000000FFFFB2
:1022300000000000000000000000FFFF00000000A0
:10224000000000000000FFFF000000000000000090
:102250000000FFFF00000000000000000000FFFF82
:1022600000000000000000000000FFFF0000000070
:1022700000000000FFFFFFFFFFFF00000000000064
:10228000000000000000000000000000000000004E
:10229000000000000000000000000000000000003E
:1022A000000000000000000000000000000000002E
:1022B000000000000000000000000000000000001E
:1022C000000000000000000000000000000000000E
:1022D000000000000000000000000000FFFFFFFF02
:1022E000FFFFFFFF00000000FFFF0000FFFF0000F6
:1022F000FFFF0000FFFF0000FFFF0000FFFF0000E6
:10230000FFFF0000FFFF0000FFFF0000FFFF0000D5
:10231000FFFF0000FFFF0000FFFF0000FFFF0000C5
:10232000FFFF0000FFFF0000FFFF0000FFFF0000B5
:10233000FFFF0000FFFF0000FFFF000000000000A3
:10234000000000000000000000000000000000008D
:10235000000000000000000000000000000000007D
:10236000000000000000000000000000000000006D
:10237000000000000000000000000000000000005D
:10238000000000000000000000000000000000004D
:102390000000000000000000000000000000FFFF3F
:1023A00000000000FFFF00000000FFFF0000000031
:1023B000FFFF00000000FFFF00000000FFFF000023
:1023C0000000FFFF00000000FFFF00000000FFFF13
:1023D00000000000FFFF00000000FFFF0000000001
:1023E000FFFF00000000FFFF00000000FFFF0000F3
:1023F00000000000FFFFFFFFFFFF000000000000E3
:1024000000000000FFFF00000000000000000000CE
:10241000FFFF000000000000FFFFFFFF00000000C2
:1024200000000000000000000000000000000000AC
:10243000000000000000000000000000000000009C
:10244000000000000000000000000000000000008C
:10245000000000000000000000000000000000007C
:10246000FFFFFFFF000000000000FFFF0000000072
:10247000FFFF00000000FFFF000000000000000060
:1024800000000000FFFFFFFF000000000000000050
:1024900000000000FFFF000000000000000000003E
:1024A000FFFF00000000FFFF00000000FFFF000032
:1024B00000000000FFFFFFFF000000000000000020
:1024C000000000000000000000000000000000000C
:1024D00000000000000000000000000000000000FC
:1024E00000000000000000000000000000000000EC
:1024F00000000000000000000000FFFF00000000DE
:10250000000000000000FFFF0000000000000000CD
:102510000000FFFF00000000000000000000FFFFBF
:10252000FFFFFFFF000000000000FFFF00000000B1
:10253000FFFF00000000FFFF00000000FFFF0000A1
:102540000000FFFF00000000FFFF00000000FFFF91
:1025500000000000FFFF00000000FFFF000000007F
:10256000FFFF00000000FFFF00000000FFFF000071
:102570000000FFFF00000000FFFF0000000000005F
:10258000000000000000000000000000000000004B
:10259000000000000000000000000000000000003B
:1025A000000000000000000000000000000000002B
:1025B000000000000000000000000000FFFFFFFF1F
:1025C00000000000000000000000FFFF000000000D
:1025D000000000000000FFFF0000000000000000FD
:1025E0000000FFFF00000000000000000000FFFFEF
:1025F00000000000000000000000FFFF00000000DD
:10260000000000000000FFFF0000000000000000CC
:102610000000FFFF00000000000000000000FFFFBE
:1026200000000000000000000000FFFF00000000AC
:1026300000000000FFFFFFFFFFFF000000000000A0
:10264000000000000000000000000000000000008A
:10265000000000000000000000000000000000007A
:10266000000000000000000000000000000000006A
:10267000000000000000000000000000000000005A
:10268000000000000000000000000000000000004A
:10269000000000000000000000000000FFFF00003C
:1026A00000000000FFFF0000FFFF0000000000002E
:1026B000FFFF0000FFFF000000000000FFFF000020
:1026C0000000FFFF0000FFFF000000000000FFFF10
:1026D0000000FFFF000000000000FFFF0000FFFF00
:1026E0000000000000000000FFFF000000000000EC
:1026F00000000000FFFF00000000000000000000DC
:1027000000000000000000000000000000000000C9
:1027100000000000000000000000000000000000B9
:1027200000000000000000000000000000000000A9
:1027300000000000000000000000FFFFFFFF00009D
:10274000000000000000FFFF0000FFFF000000008D
:102750000000FFFF00000000FFFF00000000FFFF7F
:1027600000000000FFFF00000000FFFF000000006D
:10277000FFFF00000000FFFF00000000FFFF00005F
:102780000000FFFF00000000FFFF00000000FFFF4F
:1027900000000000FFFF00000000FFFF000000003D
:1027A000FFFF00000000FFFF0000FFFF000000002F
:1027B0000000FFFFFFFF000000000000000000001D
:1027C0000000000000000000000000000000000009
:1027D00000000000000000000000000000000000F9
:1027E00000000000000000000000000000000000E9
:1027F0000000000000000000FFFF000000000000DB
:10280000FFFF0000FFFF000000000000FFFF0000CE
:10281000FFFF000000000000FFFF0000FFFF0000BE
:1028200000000000FFFF0000FFFF000000000000AC
:10283000FFFF0000FFFF000000000000FFFF00009E
:10284000FFFF000000000000FFFF0000FFFF00008E
:10285000FFFF0000FFFF0000FFFFFFFF0000FFFF82
:10286000FFFF0000FFFF000000000000FFFF00006E
:10287000FFFF000000000000FFFF0000000000005C
:102880000000000000000000000000000000000048
:102890000000000000000000000000000000000038
:1028A0000000000000000000000000000000000028
:1028B0000000000000000000000000000000000018
:1028C0000000000000000000000000000000000008
:1028D00000000000000000000000000000000000F8
:1028E00000000000000000000000000000000000E8
:1028F00000000000000000000000000000000000D8
:1029000000000000000000000000000000000000C7
:1029100000000000000000000000000000000000B7
:1029200000000000000000000000000000000000A7
:1029300000000000FFFF0000000000000000000099
:102940000000000000000000000000000000000087
:102950000000000000000000000000000000000077
:102960000000000000000000000000000000000067
:102970000000000000000000000000000000FFFF59
:10298000FFFF00000000000000000000FFFF00004B
:102990000000000000000000FFFF00000000000039
:1029A00000000000FFFF0000000000000000000029
:1029B000FFFF00000000000000000000FFFF00001B
:1029C0000000000000000000FFFF00000000000009
:1029D00000000000FFFF00000000FFFF00000000FB
:1029E000FFFF00000000FFFF00000000FFFF0000ED
:1029F00000000000FFFFFFFF0000000000000000DB
:102A000000000000000000000000000000000000C6
:102A100000000000000000000000000000000000B6
:102A200000000000000000000000000000000000A6
:102A300000000000000000000000FFFFFFFFFFFF9C
:102A4000FFFFFFFF000000000000FFFF000000008C
:102A5000000000000000FFFF000000000000000078
:102A60000000FFFF00000000000000000000FFFF6A
:102A700000000000000000000000FFFF0000000058
:102A8000000000000000FFFF000000000000000048
:102A90000000FFFF00000000000000000000FFFF3A
:102AA00000000000000000000000FFFF0000000028
:102AB000000000000000FFFF000000000000000018
:102AC0000000000000000000000000000000000006
:102AD00000000000000000000000000000000000F6
:102AE00000000000000000000000000000000000E6
:102AF00000000000000000000000FFFFFFFFFFFFDC
:102B0000000000000000FFFF00000000FFFF0000C9
:102B10000000FFFF00000000FFFF00000000FFFFBB
:102B200000000000FFFF00000000FFFF00000000A9
:102B3000FFFF00000000FFFFFFFFFFFF000000009D
:102B40000000FFFF00000000000000000000FFFF89
:102B500000000000000000000000FFFF0000000077
:102B6000000000000000FFFF000000000000000067
:102B70000000FFFF00000000000000000000000057
:102B80000000000000000000000000000000000045
:102B90000000000000000000000000000000000035
:102BA0000000000000000000000000000000000025
:102BB0000000000000000000000000000000000015
:102BC0000000000000000000000000000000000005
:102BD0000000000000000000000000000000FFFFF7
:102BE000FFFFFFFF000000000000FFFF00000000EB
:102BF000FFFF00000000FFFF00000000FFFF0000DB
:102C00000000FFFF00000000FFFF00000000FFFFCA
:102C100000000000FFFF00000000FFFF00000000B8
:102C2000FFFF00000000FFFF00000000FFFF0000AA
:102C30000000FFFFFFFFFFFF000000000000FFFF9C
:102C400000000000000000000000FFFF0000000086
:102C5000000000000000FFFF000000000000000076
:102C60000000000000000000000000000000000064
:102C7000000000000000000000000000FFFF000056
:102C80000000000000000000FFFF00000000000046
:102C900000000000FFFF0000000000000000FFFF38
:102CA000FFFFFFFFFFFF000000000000FFFF00002C
:102CB0000000000000000000FFFF00000000000016
:102CC00000000000FFFF0000000000000000000006
:102CD000FFFF00000000000000000000FFFF0000F8
:102CE0000000000000000000FFFF000000000000E6
:102CF000000000000000FFFFFFFF000000000000D8
:102D000000000000000000000000000000000000C3
:102D100000000000000000000000000000000000B3
:102D2000000000FFFF0000FFFF00000000000000A7
:102D300000FFFF0000000000000000000000000095
:102D40000000000000000000FFFFFFFF0000000087
:102D50000000FFFF00000000FFFF00000000FFFF79
:102D600000000000000000000000FFFF0000000065
:102D70000000000000000000FFFFFFFF0000000057
:102D80000000000000000000FFFF00000000000045
:102D900000000000FFFF0000000000000000000035
:102DA000FFFF00000000FFFF00000000FFFF000029
:102DB00000000000FFFFFFFF000000000000000017
:102DC0000000000000000000000000000000000003
:102DD00000000000000000000000000000000000F3
:102DE00000000000000000000000000000000000E3
:102DF000000000000000000000000000FFFFFFFFD7
:102E0000000000000000FFFF00000000FFFF0000C6
:102E10000000FFFF00000000000000000000FFFFB6
:102E200000000000000000000000FFFF00000000A4
:102E3000000000000000FFFF000000000000000094
:102E40000000FFFF00000000000000000000FFFF86
:102E500000000000000000000000FFFF0000000074
:102E6000000000000000FFFF00000000FFFF000066
:102E700000000000FFFFFFFF000000000000000056
:102E80000000000000000000000000000000000042
:102E90000000000000000000000000000000000032
:102EA0000000000000000000000000000000000022
:102EB0000000000000000000000000000000000012
:102EC0000000000000000000000000000000000002
:102ED00000000000000000000000000000000000F2
:102EE000FFFF0000000000000000000000000000E4
:102EF00000000000000000000000000000000000D2
:102F000000000000000000000000000000000000C1
:102F100000000000000000000000000000000000B1
:102F20000000000000000000FFFF000000000000A3
:102F30000000000000000000000000000000000091
:102F40000000000000000000000000000000000081
:102F50000000000000000000000000000000000071
:102F60000000000000000000000000000000000061
:102F70000000000000000000000000000000000051
:102F80000000000000000000000000000000000041
:102F90000000000000000000000000000000000031
:102FA0000000000000000000000000000000000021
:102FB000000000000000FFFFFFFFFFFFFFFF000019
:102FC0000000000000000000000000000000000001
:102FD00000000000000000000000000000000000F1
:102FE00000000000000000000000000000000000E1
:102FF00000000000000000000000000000000000D1
:1030000000000000000000000000000000000000C0
:1030100000000000000000000000000000000000B0
:1030200000000000000000000000000000000000A0
:103030000000000000000000000000000000000090
:103040000000000000000000000000000000000080
:103050000000000000000000000000000000FFFF72
:10306000FFFFFFFFFFFF0000000000000000000066
:103070000000000000000000000000000000000050
:103080000000000000000000000000000000FFFF42
:10309000FFFFFFFFFFFF0000000000000000000036
:1030A0000000000000000000000000000000000020
:1030B0000000000000000000000000000000000010
:1030C0000000000000000000000000000000000000
:1030D00000000000000000000000000000000000F0
:1030E00000000000000000000000000000000000E0
:1030F000000000000000000000000000FFFFFFFFD4
:10310000000000000000FFFF00000000FFFF0000C3
:103110000000FFFF00000000FFFF00000000FFFFB5
:1031200000000000FFFF00000000FFFF00000000A3
:10313000FFFF00000000FFFFFFFFFFFFFFFF000099
:103140000000FFFF00000000FFFF00000000FFFF85
:1031500000000000FFFF00000000FFFF0000000073
:10316000FFFF00000000FFFF00000000FFFF000065
:103170000000FFFF00000000FFFF00000000000053
:10318000000000000000000000000000000000003F
:10319000000000000000000000000000000000002F
:1031A000000000000000000000000000000000001F
:1031B00000000000000000000000FFFFFFFFFFFF15
:1031C000000000000000FFFF00000000FFFF000003
:1031D0000000FFFF00000000FFFF00000000FFFFF5
:1031E00000000000FFFF00000000FFFFFFFFFFFFE7
:1031F000000000000000FFFF00000000FFFF0000D3
:103200000000FFFF00000000FFFF00000000FFFFC4
:1032100000000000FFFF00000000FFFF00000000B2
:10322000FFFF00000000FFFF00000000FFFF0000A4
:103230000000FFFFFFFFFFFF000000000000000094
:10324000000000000000000000000000000000007E
:10325000000000000000000000000000000000006E
:10326000000000000000000000000000000000005E
:103270000000000000000000FFFF00000000000050
:10328000FFFF0000FFFF000000000000FFFF000044
:103290000000FFFF0000FFFF000000000000FFFF34
:1032A0000000FFFF0000000000000000FFFF000022
:1032B0000000000000000000FFFF00000000000010
:1032C00000000000FFFF0000000000000000FFFF02
:1032D0000000FFFF000000000000FFFF0000FFFFF4
:1032E00000000000FFFF000000000000FFFF0000E2
:1032F000FFFF000000000000FFFF000000000000D2
:1033000000000000000000000000000000000000BD
:1033100000000000000000000000000000000000AD
:10332000000000000000000000000000000000009D
:10333000000000000000000000000000000000008D
:10334000000000000000000000000000000000007D
:10335000000000000000000000000000FFFF00006F
:1033600000000000FFFF0000FFFF00000000000061
:10337000FFFF00000000FFFF0000FFFF0000000053
:1033800000000000FFFF000000000000000000003F
:10339000FFFF0000000000000000FFFF0000FFFF33
:1033A00000000000FFFF000000000000FFFF000021
:1033B000FFFF000000000000FFFF00000000000011
:1033C00000000000000000000000000000000000FD
:1033D00000000000000000000000000000000000ED
:1033E00000000000000000000000000000000000DD
:1033F0000000000000000000FFFF000000000000CF
:10340000FFFF0000FFFF000000000000FFFF0000C2
:103410000000FFFF0000FFFF000000000000FFFFB2
:103420000000FFFF0000000000000000FFFF0000A0
:103430000000000000000000FFFF0000000000008E
:1034400000000000FFFF000000000000000000007E
:10345000FFFF00000000000000000000FFFF000070
:103460000000000000000000FFFF0000000000005E
:1034700000000000FFFF000000000000000000004E
:10348000000000000000000000000000000000003C
:10349000000000000000000000000000000000002C
:1034A000000000000000000000000000000000001C
:1034B000000000000000000000000000000000000C
:1034C00000000000000000000000000000000000FC
:1034D00000000000000000000000000000000000EC
:1034E000FFFFFFFF000000000000FFFF00000000E2
:1034F000FFFF00000000FFFF0000000000000000D0
:103500000000FFFF00000000000000000000FFFFBF
:1035100000000000000000000000FFFF00000000AD
:10352000000000000000FFFF00000000FFFF00009F
:1035300000000000FFFFFFFF00000000000000008F
:10354000000000000000000000000000000000007B
:10355000000000000000000000000000000000006B
:10356000000000000000000000000000000000005B
:10357000000000000000000000000000000000004B
:10358000000000000000000000000000000000003B
:10359000000000000000000000000000000000002B
:1035A000000000000000000000000000000000001B
:1035B000000000000000000000000000000000000B
:1035C00000000000000000000000000000000000FB
:1035D00000000000000000000000000000000000EB
:1035E0000000000000000000FFFF000000000000DD
:1035F00000000000FFFF0000000000000000FFFFCF
:1036000000000000000000000000000000000000BA
:1036100000000000000000000000000000000000AA
:10362000000000000000000000000000000000009A
:1036300000000000000000000000FFFF000000008C
:10364000000000000000FFFF00000000000000007C
:103650000000FFFF00000000000000000000FFFF6E
:1036600000000000000000000000FFFF000000005C
:10367000000000000000FFFF00000000000000004C
:103680000000FFFF00000000000000000000FFFF3E
:1036900000000000000000000000FFFF000000002C
:1036A000000000000000FFFF00000000000000001C
:1036B0000000FFFFFFFFFFFFFFFF00000000000012
:1036C00000000000000000000000000000000000FA
:1036D00000000000000000000000000000000000EA
:1036E00000000000000000000000000000000000DA
:1036F00000000000000000000000FFFFFFFFFFFFD0
:10370000000000000000FFFF00000000FFFF0000BD
:103710000000FFFF00000000FFFF00000000FFFFAF
:1037200000000000FFFF00000000FFFF000000009D
:10373000FFFF00000000FFFFFFFFFFFF0000000091
:103740000000FFFFFFFF0000000000000000FFFF7F
:103750000000FFFF000000000000FFFF0000FFFF6F
:10376000000000000000FFFF00000000FFFF00005D
:103770000000FFFF00000000FFFF0000000000004D
:103780000000000000000000000000000000000039
:103790000000000000000000000000000000000029
:1037A000C7C7C7C7C7C7C7C7C7C7C7C7C7C7C7C7A9
:1037B000C7C7C7C7C7C7C7C7C7C7C7C7C7C7C7C799
:1037C000C7C7C7C7C7C7C7C7C7C7C7C7C7C7C7C789
:1037D000C7C7C7C7C7C7C7C7C7C7C7C7C7C7C7C779
:1037E000C7C7C7C7C7C7C7C7C7C7C7C7C7C7C7C769
:1037F000C7C7C7C7C7C7C7C7C7C7C7C7C7C7C7C759
:10380000C7C7C7C7C7C7C7C7C7C7C7C7C7C7C7C748
:10381000C7C7C7C7C7C7C7C7C7C7C7C7C7C7C7C738
:10382000C7C7C7C7C7C7C7C7C7C7C7C7C7C7C7C728
:10383000C7C7C7C7C7C7C7C7C7C7C7C7C7C7C7C718
:10384000C7C7C7C7C7C7C7C7C7C7C7C7C7C7C7C708
:10385000C7C7C7C7C7C7C7C7C7C7C7C7C7C7C7C7F8
:10386000100C0001020304050605070308090A0BF2
:103870000C0A0909090909090909090909090909B4
:1038800009090909090909090909090909090D0E9F
:1038900001030F0D100511060D0909090909090990
:1038A00009091213030703140315160D0909090961
:1038B0000909090909091701180117090E01150D50
:1038C00002081903180D0E091A1B0904060D080831
:1038D00001101C0515161103091D03141705100905
:1038E0000909120308091E03100701101014090921
:1038F00009090909090909090909091F100502101F
:103900000313000310200D080921111520010609D9
:103910000909090909090909090909090909090917
:103920000909100C2205082010051715230909099B
:1039300009090909090909090909090909090909F7
:103940000909090919241F030E092509130518017E
:103950000909090926092509100115200310200964
:10396000090909092709250911080E05091F11155B
:10397000160909092809250908012920091701182C
:10398000011709092A0925091F1001181B09170128
:1039900018011709040117012B2009250913010833
:1039A000110909090909090909090909090909097F
:1039B000090909091208091301081123090909094C
:1039C0000909090919241F030E2C092D2E0925099F
:1039D0001305180104200310200925091F170314DB
:1039E0000909090956DDE5015E58DD368D820D8D28
:1039F000DD5F56DDD588D0560D0230D0130D88DD41
:103A0000D5FF85CDDED58DD588020D058520D0105A
:103A10001560DDDDDF75DDDD5888D01B26D888DD3B
:103A2000D85CCDDF764DDD54588054501210D5024D
:103A3000620D81210D888DDDD5FFB5DDD0DDD88DFE
:103A4000580D0A88056D02059180D80DDDDDD5FF82
:103A500067DDDD880D01210D02120D01210D02121D
:103A60000D868DDDDF56DD5E518D56A0D58054D894
:103A70005CD15C4D5FA7CCCDD5CCC5185CCC51508A
:103A8000DDDD150D060202020D0505050DD88805C0
:103A9000EDDDD5FF87CDDDEC5885EC50D6DD5050FF
:103AA00020D095020D8880D8DDDDDF87DD5E580DE2
:103AB000E50285ED020DD4D56185C581505C588045
:103AC0005CDDD5FF68DDE510DE51605E51025ED23F
:103AD0000D545028545885458D54DDFF65DDDD8833
:103AE0000D05050D10236D80DDDDFF86CC4D5EDDFF
:103AF000D6D588130D80580DDD2505CC5805CCDDB5
:103B00005F974DDE458DDE45880DED0D805E5101E0
:103B10005062D58050A0D81588DDDDD5FF56DD5E1A
:103B200050605E5915E5A2D588D88DDD5F68DDDD72
:103B3000880D1018D0D0D58205ED5205EC5605EC55
:103B4000585ECDDF77DDDD58090D86A0DDD0DC4580
:103B500085EC4585EC4585EC4DDF87DDD5E5880DA9
:103B6000D86A9DD50D05C58805C58DDC585ECDDFAD
:103B700065DDE58DD501010D0A56D58854DDDF6878
:103B8000DD5E580DD1018D8050D50585456A05450E
:103B9000885458D54DDF66DDDD838D880D5050D4B7
:103BA00052615E45805E4DD5FF6650DD5C580DDA92
:103BB0006D80DD880D01010DDDDF664DDE458D5424
:103BC00050A0D5910D8620D80DDDDF574DD5450687
:103BD000054580DD20D091D0A0DD85CDDF66DDDE1E
:103BE00058015E50D0D58A6D0580D18DDDDF66DD50
:103BF0005E5805E50605E50ADD510105458854DDF9
:103C0000DFA8CC4DD5ECC4580DCC458854DDD80D7B
:103C10005880510D0202068D50DDD15E588885ED29
:103C2000DDDDFF56DDE58DD0A0D910D0620D80DD41
:103C3000D5FF66CDDE4D85ED621D50A8D01010DD9C
:103C4000805CDD5F664DDED8DD880D1B26D80DD586
:103C500085E4DDFF66DDDD1058D828D10256D8286E
:103C6000D1058DDDDF85CDDED58DD58880D62B3194
:103C70000D8880DDDDDF69CDDE4D85E451025E45D6
:103C80001205E451205E451205E45102D458065451
:103C9000D805CDD5FFE4DDE58DDDDDD502020202DC
:103CA00002060D09918880DDDDDDDDFF87CCCDDDED
:103CB000D051D80D51D802051D02828DDD6505CC8D
:103CC0005805CCDD5F96DDDDD58888D0D1D50D05D2
:103CD0000A010D01062D0DDD885CCDDDFF98DD5E4E
:103CE000580DDE50505015E58820DDD05218D8050B
:103CF000680D050DDD5805EDD5FF654DD5E458057A
:103D0000ED80D50A20D01710DDDDFF75DDD5E58803
:103D100005E56A20D58591D588D4DDDF67C4DDC48B
:103D2000585C4560DD521D8021D05021D88DDDDFEB
:103D300088CC4DDCC45065CC458DDD501D80281DE0
:103D40008A501D88DDD585ECDDFF42DDD621DDDF23
:103D500056DDD5910D820D052D5820D860DDD5FF9B
:103D6000674DDDD88D8D0D05020D8301D5056D459F
:103D7000805E4DD5FFA6CDDD5ED58805E5020280CB
:103D80005E50D50DDD06010180D80D580DDD0DD535
:103D9000FF77DDDE58605E5850DE50158D501A20DA
:103DA000D01580DD5805C4DD5F79DDDE50685E50DA
:103DB0002505E50285E5020DED50DD45858545913A
:103DC000854588054DDD5F96CDDED58DDD82869DEE
:103DD000028850DD0DD05C58885CDDDDFF76DDE5C6
:103DE0008D5E588DD82360DD01505C5885CDDDFF98
:103DF00057CDDD506D820D831D831D820DD85CDD96
:103E0000FF664DD5ED101D503030D858D02020D54C
:103E1000060D4DD5FFB7CCCDDDCCC5885CDD501887
:103E2000DD8D518D0282810D506A050105ED88DD21
:103E30005E4DDDFF97DDDDE5060585E58885EDD581
:103E4000205ECC58D54D0520954D058D5CCDDF65A8
:103E5000DD5E580DD828D5301054580654DDDF7873
:103E6000CDDEC585EC5605EC585ED50DD58830D82D
:103E7000280DDD105CCDDF66DDE58DD51328D01271
:103E800050D506854580D4DD5FC8DDDDDDE5888859
:103E900085E50DDD506D50588880D05828058D0A75
:103EA0000DD58DD85050915CDD05885CCC4DDDFF83
:103EB000994DDDD5458880D56DD50D858050D85874
:103EC000021D8D2D1D52D851D802851D8058DDDD73
:103ED000D5FF89DDDDE58885E50DD05E5059165E9C
:103EE00050D52DD05880D8A020DD580DC451D5EC28
:103EF0004D5FC5C4DDDDDDD88D8D8A29926D888D3D
:103F000058D80DD0DDDD5F984DDDED885E58020597
:103F1000E58A05ED501DD5CD150605C4518205C4B1
:103F2000510DDC4DDF88CDDDEC5885EC58205E4D21
:103F3000D205ED020205E59950D588060D585805C1
:103F40004DDDDF67DD5E580DE50585E56231DD811C
:103F50000545025054D805CDD5FF964DDE458DDD83
:103F6000D8828D0150280D0152DDD01605EDDDFF00
:103F7000A7DD8DDE58DD85E5858585E585882D58AD
:103F8000101528D60D05020D8010580DDDDDDF79E6
:103F9000DD5E5060DD5888D020A0D52D8D80DD50AD
:103FA000985ED985E4D585EC4DDFC8DDDDD5E588A3
:103FB0000580DD0262050181D0D0D50D0D05888018
:103FC00050D058058050D0DDDD50D888880DDDDD1B
:103FD000DDFF9ACDDE4D8DD5458286054582580D93
:103FE000D50DDD85805E588205E509585E581DDED9
:103FF00058DEDDFF79DDE58DDD0A020D888D50D0BC
:10400000D591565E50D50D5888D8580DDDD5FFA7EF
:104010004DDE458DDD5452065801D505A801D8283E
:10402000D9D8050DDDD805ECDD5F964DDD5ED09964
:10403000DE580DDD58020206DD820205CD5885CC22
:10404000DDDF9A4DD5ED805E588DDD851580D60576
:1040500015020D85158D588585ED8DA5E4D8805EFA
:10406000C58DDECDDFA6DDDDDE50609905E580DDA6
:104070002DD05820205450288854580DDD4DD5FFA0
:10408000A74DDD5ED880DE5820285E502020205EBF
:10409000D0D50DD456899154D880D5CDDD5F954DBE
:1040A000DDD5458858D5025258D812168D81588DC5
:1040B000DDDD5F9ADDE58DDDD810D01D025881D59C
:1040C0000D0501545885854DD0585C50620D5C50EB
:1040D000A05EC5885ECDDDFF584DD545805450109B
:1040E000D5030D83D586DD0205458054DD5F77DD80
:1040F0005E580D5E50180DD3528D015020D06D0DBD
:1041000058805EDDD5FF79DDDE588DE502020DD0E9
:10411000A854505805450D0D458101545061015476
:1041200058DD4DDFB9DDDDE589105E58D50DE5853B
:104130000285ED056285E45050285E450D50DD5442
:1041400058888054580D58054DD50DD5FFAACCC4BC
:10415000DD4DDD58545028885458020285450DDD48
:10416000DD050185E5850585E586010DED0505057E
:10417000E4580105E4DDD5FF87CCDDECD58D4D029B
:1041800080D502850D065A8D098DD09D5EDD5F8933
:10419000CC4DDDDD8D8880D89101D52DDD50285E98
:1041A0005802D5ED8285E4D0685ECDDDFF98DDDD77
:1041B000D580D80D0282650DD5050205C45158D4AD
:1041C00050515025E45051805E45051805EC4DDDF9
:1041D000FF964DDDDE4586805E45028205ED50D0BE
:1041E000DD82928D80980DDDDD5FA4DDDDDD881D33
:1041F0008D0A69A0D80D180DDDDDDFE9CDDEC5859E
:1042000088DD5C585885805C58DDD150DD582881A8
:104210008D80A50D5150D8058050580DDDDD05600D
:10422000DCCCCC585ECCCCCDDFAA4DDDD5ED8058B2
:104230000D588588D8205028D8031380DD5161DDC2
:1042400058031380D8205028D88588D580580D4D24
:10425000DDD5FF87DDDDD060580D020280D52D5001
:10426000D58918D80580DDD585CC4DDF77DDDD56C5
:10427000880D01A10D02920D02920D01A10D888DF4
:10428000DDD5FFAACDDDEC5885EC5885EDD585E56B
:104290008051DDD8026280DDD15805C4D0D0DC4524
:1042A00080215EC4580D5EC4DD5FD9C4DDEC458D50
:1042B000DDDDD0202991D80280DDD56D50D5E58295
:1042C00085E5020505ED0585E45885E4DDDFF9DDCA
:1042D0005E580D0DDE5820D5015E502802815ED05B
:1042E0002DD5150DD502850501D58D885050158623
:1042F0000DD850588805CDD0D880DCCCCDDD5F7787
:10430000DDD5E506585E512805E510502D51258074
:10431000D105020D8580DDDD5FA7DDDDDD99588DDE
:104320008580A0D868D8D880D20DDD58205CC458CC
:1043300085CC4DDDFF77CDD5EC5010DD5028D01069
:10434000256D052010D820DD50105E4DD5FF88CC9E
:10435000DDDDD80D8828D825256DD05805C5091074
:104360005CD58DCC585ECCDDFFAA4DD0DDED8D58EF
:10437000D58050580D8310138DD2802D545806804F
:104380005ED52802DD8310138D8050580D58D58DD1
:104390004DD0DDFF984DDDDE458885E45680205EFA
:1043A000D0D5205E50991DD0202028DDD50505CC24
:1043B00045805CC4DD5F77DDDD5888D02B30D03898
:1043C00030D03830D0B310D8806DDDD5FFE7DD8830
:1043D0000DD5E58D580580D58858052020D950DDAC
:1043E0005058D8688502020D9588880DD80DDDD506
:1043F000E4DD5F88CDDEC585EC502DDD51018D02F9
:1044000005020D8101DDD5205EC45065EC4DDFA8AD
:10441000DDDE588D5E5850205E5820605ED0D0DDC5
:10442000D85999D020202020D580DDD4DD5FB7CCAD
:10443000DD5EDD580DD5880588D859918D58D0504E
:10444000D545A6A205E45880D5E4DDD5FF96CC4D30
:10445000D5C4D580DD5991D06AA20D88050DDD58EF
:1044600005ECCDD5FFA94DD0DDE458D58D45888626
:104470000D59D580D88858D9152850D0D0A020D82B
:10448000288DDD58D5EC4DDF994DD5ED80DE5828CF
:10449000DE502028DED525010DC50501854D0D18FE
:1044A00054506810D4580585E4DDDDFF89CDDDEC7E
:1044B000588D4D0D85450A050545062050545885F3
:1044C0000DD5058D8910D5880DEDDD5FAACCCDDE2B
:1044D000DDD585E502888D502DD58D865858D50DB2
:1044E000980D8509DD5028D5E502D5E585EDDFAAD3
:1044F0004DDDE450185ED21505E58385E509D5ED5F
:104500002050DDD50D0580D8DD050D80602020D53B
:104510008588054DDDDDFFEADDDDE58885E5020AFC
:104520000DDDDDD506D10185CC528501805CC580CD
:1045300051010DCC5250D0505ECC588885ECC58DC1
:1045400058DECC5850DDECCDDFD8DDDDDDD58885FB
:10455000880D026A050109D50D0D50D054505888B8
:104560000505450580580505450DDDD505458888B7
:104570008054DDDDDD5FC7CCCDD5ECCC580DECCC67
:1045800050285EDDDD056D5018502028D8888250F7
:10459000D91DD580DDD80DD5FFB64DDDDDD599917E
:1045A0008D0AAA260D80505050D505058805E58056
:1045B000DDD5EDD5FF98D0DDEDD8DD45020218D56B
:1045C000058120D80D1DD828105E50605805E58D56
:1045D000DDEDDFA7CDDDDDD80580D030201010D88F
:1045E000020D0DDD35805E45868D5E4580D5E4DDAE
:1045F0005FA7CDDDDDD060580D03020390D8020522
:1046000080DD5358D545880DE4580D5E4DD5FFB675
:10461000DD58DDD80DD90D0A2888D8025890DD065E
:1046200058D05C58D885CDDDDDFF6ADD5E5805E5E4
:104630000105E5161DD5158D828D0280D5A854582B
:10464000D54585E4DDFF97DDE506D5E5138DDD95E0
:10465000A020D58880545050D854580DD54DD5FF42
:10466000974DDD5E458101D5450101010DD0DD0D80
:10467000862820D8A820DD580D5C4DD5FFB9CCCCBC
:10468000DDDDDD58D80D0280D8280D8DD0510150C8
:10469000DC50510152DC50580585C50602885C5833
:1046A000DDD5CDDFA6DDD5E5880DDD0A56D9D0589C
:1046B000880D8205058DD502895C4DDDDF874DDDD6
:1046C0005E458805ED0D52D5128060D090520D1DCB
:1046D000820D88DDDDDFC9CCC4DDECCCD8DDD5852D
:1046E000828D8DD02020D80950528D858068DD5074
:1046F0005950D5E450D0505E458885E4DDDDFFBAE1
:10470000CDDED585E588D5E50501015E506091DDFA
:10471000E505050580D58050A80DDD820205CCD2C7
:10472000050DCC45885ECC4DDDFFD8DDDD0DDD858A
:1047300080D580D888D028D15060D028D515805019
:1047400028DE5158828DE510D0DD5ED885E4DDDFAE
:1047500098CDDDDC5850105C5801315C585030DD8C
:1047600052D1D588820D020D020D806580DDDDD528
:10477000FF88CDDEC585EC58DDD52128D81618D8A0
:10478000212DDD585EC4585EC4DDFFAAC4DD5EC4C1
:1047900050605ECD80DED51A21DD829128D821516E
:1047A00028D829128DD1A21D5CD80DEC45805EC49D
:1047B000DD5F884DDD5ED818D501A210D021012023
:1047C000D1206021D0210120D01A210D5818D4DD2C
:1047D000D5FFB9CCC4DDDDDD580D18018651D8D523
:1047E000880D50285885450280DD54502585E4D039
:1047F000585EC580DECDD5FFE6DDDDD5E58185805F
:104800005E505186805E585950DDDD58D0A0202082
:1048100054D8888805CDDDDDD5FFE7CC4DDE4DD5FC
:1048200085E458802DDDD50D095891D020A5286844
:104830000D8888D58DDDD850DDCCCDDFB9C4DDEC59
:104840004585E4D585ED8205E580505E505A0DDD45
:10485000505805801D8286801DD8DD95CDD8DDFF9E
:10486000E8DDD0DDE58805885E51D852D85E580570
:10487000880585E52850D5858D058885850D050D2C
:10488000D85050D10688203010DDDDDDDDFFC9DDD8
:10489000DDDDD150658580D15A805020D15850251A
:1048A00080D150258502D5158502585E5150258549
:1048B000025E598502805E59858585EDDDDDDF5715
:1048C000DDE585E585E58DD1A6D810D8DDD5FF5786
:1048D0004DD54580D5150D860D820D053D5805ED4C
:1048E000D5FF67C4DDDD8D858D01010D06A0D0509B
:1048F000DD805EDD5F974DD5ED060DDE585810D595
:1049000005888D0A0518D588DD4D805ECDD5FF76EA
:10491000DDDE5885E50A0DDD0685C58105CD01DCA6
:104920004DDF87C4DDEDD85E561385E5858DDD58F6
:10493000205C458505C4D805CCDD5F66CDDDD80D8E
:104940008250D8120D50D154580654DDDF76DDDD8B
:1049500058068D8038DD12D5C50305EC5805ECDD11
:104960005F56DDD588D0526D0131D0520D88DDD52E
:10497000FF65DD5E5805E580DDA260D918DDDDFF4D
:1049800055DDD5158D6A0D920D58054DD5FF784D25
:10499000DD5458585458520D58137D80520D80588C
:1049A000D58DD4585E4DDF67DD5E580DD880D88038
:1049B000DD1DD02320D878DDDDFF664DDED8DD019A
:1049C00028D6128D0120DD8DE4DDFF66DDE58DD575
:1049D000858D12B6D58854580D4DD5FF77CCDDCDD9
:1049E000585C50A054D058D501526D888D09DDDD3A
:1049F0005F574DD54580545256D5020D80D51310C2
:104A0000D88DDD5F674DD5E4580D4525605450289D
:104A1000D58DD0218D1018DDDDFF67DDDD880D0A15
:104A200021D50561545050154585054D805CDD5FED
:104A3000674DDE458D5452805450150D5318D020CB
:104A4000DD0605EDD5FF8ACCDDE4DD85E451018D81
:104A5000458506054D058054D0D8545028D545824B
:104A600005E45050DE45805E4DD5FFA84DDDD5E410
:104A7000588585E450202805E4D0D585ED50505662
:104A8000DD80D580D05010180D80DDDDDDFFB74D05
:104A9000D50DD54580D580545628D90DD25888D803
:104AA0000D0D8D8880DD5805805EDDDD5F674DD59D
:104AB000ED80D501210D02520D01210D88DD06DEAC
:104AC0004DDF77DDDD5888D0D520D05820D0513249
:104AD0006D05158D8158DDDD5F69DDDD878D032373
:104AE0000D10501D858D858D858D02520D858DDDB6
:104AF000DF87CDDD5C5880DD0D50D09380D8A60DCA
:104B0000DD8DEC4585EC4DDF77DDDE5885E50D2D3F
:104B1000D05028D061310D58805458DD4DDFD8CCAD
:104B2000CC4DD5CCCC4580DDDDD5050D1880582881
:104B3000D1868588D5150DDD58D88880A0D58DD52E
:104B40008854DD80DDDF98CDDDDC585805C58280D6
:104B50005C58D2DDD0D8D0691520D8888DDD58DCDE
:104B6000C4DDFF79DDDD5888D8850DD9215C505230
:104B7000DC58605CD0205C450505C45805C4DD5F89
:104B8000A6D50DDDD50DD80D0D0915054D5280505A
:104B9000D58AD50D506888DDDDDDFF8ADD5E580DD4
:104BA000DE581585ED098D450D06054505885450DF
:104BB00020DD4502DE450205E45805E4DD5FBA4D1F
:104BC000DDDDE458D88D45880D85450502585054E3
:104BD00050586025054505852805450D58DDD01838
:104BE0000DE581DDE5815EDD5FA7CCDDDECC588D96
:104BF0004DD0D8D588850D062B1050D8050D8DDDEC
:104C000088DCCDDDFF794DD5E45805ED050DE502D5
:104C100080D582510D502010545851054DD065CC8F
:104C2000585CCDDF78CDDDC588DD0D0D0918D820A5
:104C3000DD052DE58205E58605EDDDFF784DDDED31
:104C4000885E58D05E5650205E58395ED052D545A9
:104C500088054D5805C4DD5F584DD54580D5010DFB
:104C6000830D050D5820D503054506054DD5FF7666
:104C7000DD5E580DD505018D05218D062350DD58CB
:104C800005C4DD5F974DDD5E45880DD50D528D89DC
:104C9000028D81D20DD50506DEC580DECDD5FFA7FC
:104CA000CC4DDECC4506DEDDD020D58105028D88D9
:104CB0008250D50958854D8DDDCDDFA9CCDDE4DDF1
:104CC0008D5E45880205E458A0505E450506585E95
:104CD000D0DD8D589188D0D50580D880DDDDDDFF11
:104CE000C6C4D58DDDD50DD80D8D5888D098AA8D28
:104CF00009850658DDDDDDDCCC585FB9DDDDE585F5
:104D0000805E58885E58D0D5ED0D80DD450D0A26B1
:104D10000D50D0588D0101010DD580DD5EDD5F8A1B
:104D2000DDDE588D5E5020685E58D505E50A020527
:104D3000E5880DDD0D8D0998D8880D8DDDDDFF9698
:104D4000CC4DD54DD580D587850D0A1A8D85150D8D
:104D5000D58185E4DDD5FF684DD5ED805E5885E5CC
:104D60000121DD2520545121054588545060D4DDB2
:104D70005F864DDDD458580D58528D0136310D8265
:104D800058D580585EDDDDFF76DDDD58218D821837
:104D9000DD8DD8218D60218DDDD5FF78C4DDEC451A
:104DA00085EC45205EC4585EDD6DD8280D8930D86D
:104DB000058DDDD5FF764DDDE45885E45109DD52E2
:104DC000060D02820D80DDDD5F77C4DD5CD80DD07D
:104DD000150D82326D80150DD0585C580DCDD5FF64
:104DE00077C4DD54D580D5880D0B20D583015ED5E1
:104DF0000565EC5805ECDD5F88CCDDE4DD8D45888C
:104E00002054505850D505A26D098DD090DED5851F
:104E1000ECDDFF974DDDE4588D5E45028205E4D25E
:104E200050505ED505650D50101018D80D80DDDD91
:104E3000D5FF95DD5E5805E580DDD5AA0206D9913E
:104E400080DDDDD5FF87C4DDEC458D5C450185C483
:104E500052160DD50120D8A1DD8805EDDD5FB8DD46
:104E60005E580DD5E5802020D5ED028820D4DDD018
:104E7000905CC45101065CC458805CC4D58DCCC420
:104E8000DDFF96DDDD5E58D80D5020A360D85010B0
:104E900050D505101854580DD54DD5FF89DDDE5875
:104EA00085E50D0DE505030DE505638D5050380DC5
:104EB0000503020D0D051D588D5EDDDF99C4DDEC87
:104EC000D8DE4D038DED020120D58106030D038050
:104ED00018D5021020D4D830DECD8DEC4DDFAACC11
:104EE00045ECC515EC450205EC58805E458B385EF7
:104EF00051203630215458B385EC58805EC4502080
:104F00005ECC515ECC45FF66DDDD01010D1A21D07E
:104F10002620D1A21D01010DDDDF77DDDD58580D02
:104F20008590D0AA2D8591D8580D8680DDDD5F77DC
:104F3000DDDD58058D021210D51820D0281D501225
:104F4000120D8586DDDD5F88DDDDD8880D03232326
:104F50000D029120D0310130D029120D0323230DF1
:104F60008886DDDDDF88DDDDD8880D0121210D0299
:104F700012120D0126210D0212120D0121210D88A0
:104F800080DDDDDF88DDDDD8880D0212120D012104
:104F9000210D521612D50121210D0212120D888009
:104FA000DDDDDF88DDDDD80580D0121210D02121B3
:104FB00020D512621D50212120D0121210D8058058
:104FC000DDDDDF884DDDE45810DD502180D823A0E1
:104FD000D93639D0A328D80120DD50185ECDDDFFA9
:104FE000AACDD5EC580D5E4D0580D545812580D5DF
:104FF00005212150D8216128D05121250D580521A6
:1050000085ED58050DECD5805ECCDD5F884DDD5E0D
:10501000D880D582128D0251520D59690D0251521C
:105020000D82128D8058DDDDDF88CCDDE4DD85E486
:1050300058805ED15050D5620258D01288D512D80F
:1050400054510DD54DDFA84DD0DDD58D580D8105BE
:10505000820D01012020DD53D0505EC5850605EC90
:1050600058DD5EC585ECDDFFBA4DDD5E45858D5EA4
:105070004585810D5458020506054D05020285C57A
:105080000D9DDC58585ED50D50D5E58802805E58E0
:105090000D5185EDD50DD5FFA74DDDDD4588885433
:1050A00051DD80D512060A0D01312058D0D50D0DE5
:1050B000588885EDDDDDFFB9DDD0DDE5018D585E79
:1050C000588868D59950258DDD502805CC4D202075
:1050D0005CCC580DCCC502DECCC585ECCCDDFF76B2
:1050E0004DDDE4510105E45831DD52060D02820D1B
:1050F00080DDDD5F78DDDD5888D05158D8380D521D
:10510000320D5836DE5051DE5805EDD5FF694DD5CC
:10511000E45805E4580D452320D51010D0161D5035
:105120002325ED805E45805E4DD5FFE74DDD88DDB2
:1051300045068DDD854585802880D5099502058D3C
:1051400080D0D028D5888D50205EDDDD0D85ECCC5B
:10515000CCDDFFC7DDDDDDD8880580D88D0580D5A5
:105160000D502020D569150A205E5888885ED9DD4B
:10517000DDE4DDFFAACC4DDECC4585E4DD585E459F
:10518000820205E450158D5E45015A8DD015880DBB
:1051900083D568D8888DD01DDDE4DDFF89DD5E58BC
:1051A0000D5E505020DD050280D0512D6D0512801E
:1051B000D81DDD50185E45885E4DDDFFBACDD5ECBB
:1051C0005805EC5805EC58D5ED51050DDD810D580D
:1051D0000D81050280D051D02020D81068ADD8D5DF
:1051E000805E4DD0DD5F97CDD5ED50105E58102D0F
:1051F000E58A10DDD01A605CD20185C45010D5C498
:10520000DD5F774DDE458D5ED88D583010D032325F
:105210000D50121054568D54DD5F69CDDED585E5F5
:10522000810D50538D02156D52150D828D80DD8DCF
:10523000EDDF8ACDDE4D8DD458A8545058505450CF
:10524000202505450585054565850D505258D099A1
:105250001D580DDEDD5FAAC4DDEC4585ECD02D5E6A
:10526000C5818DDD012180D021262120D801210D8D
:10527000DD8185ECD520DECC585ECCDDFF994DD5A7
:10528000E45010DD54520A020545090101D52801F8
:1052900020D021802D51010905E5620A025EDD5012
:1052A000105ECCDD5F86DDDDD80580D029120D02D1
:1052B00036320D029120D80580DDDDDFA6DDDDDD93
:1052C00088880D8301038D53236323D58301038DC8
:1052D00088588DDDDDDFFADDDDE585805E58885E8E
:1052E00058D0DDDDDD0D8588805450D858880545BF
:1052F0000D820202020D50D50DDD56D8810101014B
:1053000080D80DDDDDDDD5FFAACCC4DD4DDD58D55F
:1053100080D80D885820D050D28D5058020DE565A8
:1053200001520DE5898DED510D5EC585ECDDFF76F1
:10533000C4DDE4D58D45880D53850D032310D86851
:10534000DDDD5FBACDD5ED580DDE58028205E502F0
:10535000D8205ED880505E4DD5050D5CC4509105B7
:10536000CC4D1805CCCD06DCCC4585ECCC4DDF8A88
:10537000DDDDD80580D0203020D95059D0205020F4
:10538000D0126210D0205020D95059D0203020D8CF
:105390000580DDDDDF96DD5E568DDD5820580D136E
:1053A000131020D820DDD5805E4DD5FFA8C4DDD5F3
:1053B000ECD880DD58D58D8058050D62B31050D5DE
:1053C0008885054DD0D85CC588DCCDDDFFAACCC46E
:1053D000DDDDDD8D880280D8D1D8D52D810D4581C8
:1053E0000250D450D51585450D50685458020DD43F
:1053F00058DDE4DDFF77DDE585E585E58DDD1A0225
:105400006D81010D8DDDD5FF65CDDED585E50216FB
:10541000D5838D838DDDDF67DDDD880D0128D51215
:10542000DD868D01250D880DDDDF58DDD5860D0566
:1054300020D0131DD20D830D88DD85CDDF95DDDEF7
:10544000588DDD802028DD291605C58DD5CDDF7668
:10545000DDDD5858D503521D5030210D0688D80D7A
:10546000DDDDDF884DDE458DD5452802054501513E
:105470008D50D50D50215105E5068025EDD585ECE3
:10548000CDDFF7DDDDDDDD5858585858D8185858AD
:1054900058D0258385858D85850638520D8585856F
:1054A000818D858585858DDDDDDDD5FFE7CDDE4D03
:1054B0008DDDD5E458888805E458DD50D0DD50D026
:1054C0005012120D026285888D01018DDDDDDDDF58
:1054D00086DDDDE58885E502159DD21A60D021586C
:1054E0000D80DDDDDFC7DDD50DDD809D580D8D150F
:1054F000880D06D25028D588820D5E5858585EDD3A
:10550000D585ECCCDDFF77DDE58DDE59185E51D811
:10551000D582020DD20205C56805CDDDFF674DDEDF
:10552000458D5450385450356D5038D812D5885E5A
:10553000DDDF77DDDD58860D02820D50D0D50250BB
:1055400025E58905ED0905E4DDDF77DDE506DDE527
:10555000880D501518D5AA0D0101DD885EDDDF79B3
:10556000C4DDE4D5605E4588DD2590D82050D0505C
:1055700028D0952DD885E458D5E4DDFF87DDDE58A9
:105580000D5E580DDED02030DD25910D028060D8F3
:105590000D8DDDDDFF86DDDDE580185E502058D500
:1055A0000B0B0D5850205458106054DDDDFF87DD83
:1055B000DE588DE51A10DE501A10DD01A1054D01EF
:1055C000A15CD0685C4DDDFFA8CCDDE4DD8DE45846
:1055D0005030DED125830D580603030D805838DD89
:1055E000D5885CCD58DCCCDDFF89CCDD5C4D805CA2
:1055F00045860DD5050D5101810D8D58D502020D41
:1056000045820DE4D585EC4DDFCACDD5EC5805ECCF
:105610005150DDD5C50288805C5150D505054D85BA
:1056200080A054D150580DD5888D5E5860DDE5803E
:10563000DEDD5FC9CC4DDEDDD015E588815E5852D8
:10564000561DDD5058010585458D58A05450580D04
:105650002854588880D458DDDDE4DDFF96DD8DD5F3
:105660008DD8D0A8A0D0129210D501810D4D068DF5
:10567000ECDDDFB7CCC4DD54DDD580D58095020DDF
:10568000020295020D020592020D0205980D50606E
:10569000DDD5EDD5FFA7DDDDDD8313138D80272854
:1056A0000DD0D50D5C582805EC585805EC58DD5E3A
:1056B000CDDFBACCC4DDECDDD015ED588805E58A28
:1056C00005095E5028581DE58A5051DDD858805C88
:1056D00058850505CDD50685CCC580DCCCDD5FFAC7
:1056E000DDDDDDE580158585E58015882D5E50655D
:1056F00015025820DE58018050280D58DD50D88DF5
:10570000D580D88505CCCC5058505CCCC58D85CC87
:10571000CCD88DCCCC4DDDFF86CDD5ED5060DD0AEB
:10572000A20D09910D80580DDDDDCC5F77DDE580A0
:10573000D5E5012105E502385E458320545012105D
:1057400054D5865CCDDFAADDDDDD805880D8120D12
:105750008D0512D90D0D80AD5858058D5A80D0D0C9
:105760009D2150D8D0218D8060580DDDDDDF97DD83
:10577000E585E585E58DDDD1A02026D8101010D86F
:10578000DDDDD5FF79DDE5065E58D5E51A05E58155
:1057900005E58DDD1A020D81010D8DDDD5FF9ADD48
:1057A000DD5E580D85E5652885E58AD0DD8850DD0C
:1057B00052D185C5851015CD81D5C45885EC4D8055
:1057C0005EC4DDDFA9DD5E580DDDD809180D50205F
:1057D0002028DDD56DD58202020D5809185EDDD571
:1057E00085ECCC585ECCCDDFAAC4DDEC4585EC451C
:1057F0008DECD210DDD5021A8D89698D8A120DDDEE
:105800005012DEC4D85ECC585ECCDDFF78CDDED53C
:105810008DD888D020202D313131D020202D31312C
:1058200031D0688DDDD5FF86DDDDE506058D583587
:1058300021DD030210D588854D580DCDDD5F77CD74
:10584000DDCD8DD580D581320D83126D580DD58D6E
:10585000EDDDFF77CDDD4D58DD580D581320D831E3
:1058600026D580D54D8505CDDDFF88CCDD54DD8086
:105870005458028D5852DD030185E5830565ED50CE
:10588000185EC58D5ECDDF89CCDD54DD80545802B5
:105890008D5852DD030185E5830565ED8385E45070
:1058A00010D5E4D85ECDDF89CCDD54DD80545802BC
:1058B0008D5852DD030185E5830565ED8385E45050
:1058C000301DE4D805ECDD5FAADD50DDD80D580DA4
:1058D00005105850D82120210D5821210D4D21614E
:1058E0002DED012128D501202128D05850150D80FB
:1058F000D580DDD0DD5FAAC4DD5EC45805ECD012D2
:10590000DEDD210DD502021A8D0916910D8A1202D3
:105910000DD5012DDCD210DEC45805EC4DD5FF7934
:10592000CDD5E4D80DD5058DD2150D82156D052187
:1059300050D0588D850DD580DE4DD5FF76DDDD58F4
:1059400088D052160D821DD05215E580DEDD5F86AF
:105950004DD5E4580DD45821854D02185CD21D5CFC
:1059600045605EC4DDFF67CDDEC585EC585ED521A0
:105970005E5821D505210D8060DDDDFF97DD50DD0E
:10598000580D58D88D60D58852154D8821D0D852E1
:105990001D50D058DD0DDDFF77DD5E580DD505219A
:1059A0008D81256DD2185C58D5C585ECDDFF78CD8D
:1059B000DDD588D80D0D05218D6512DD0521DE5858
:1059C000805ED5805ECDD5FF76CDDDD588D82150DF
:1059D000D65128D0521DD885EDDDFF77C4DDDD58C6
:1059E0000D82150D65128D0521DD0585E5885EDDCD
:1059F000DF68CDDE4D85E450105E450305ED03DD27
:105A00008205E58605E58D5EDDFF78DDE58DDE58F6
:105A1000805E581505ED5350D45638054502805424
:105A2000D58DC4DDFF574DD545010545030D5030DB
:105A3000D830D0620D8DDD5F694DDD4501854503B0
:105A400050545638545030D4D2854588545050D490
:105A50005805E4DD5F78DDD0D80D0D8105E5820DB8
:105A6000D503060DD20505C5158D0580D50DDDFFC5
:105A700078DD5E580DE50510DD82060DD380D82057
:105A8000DD051DE5805EDD5F58DD5E5805E501053D
:105A9000E50205ED30D5028D0106DD85CDDF694DCE
:105AA000DD4D585450106545028DD30D5820D50555
:105AB000105E580DED8DEDDDFF794DDE4585E45826
:105AC0005E458DDD5A8D8218D059DD06505ED805B1
:105AD000EDDDFF76DD5E586DD505A8D82150DD9847
:105AE0005CD805C4DD5F76C4DDEDD065E58A0D5078
:105AF0005218D8950DD5805C4DD5FF684DD5E4582A
:105B000005E450505E450605EDADD0218D0950DD10
:105B1000805CDD5F67CDD5CD8DD80D828D0131DD07
:105B20000205ED5605ECDDFF57CDD4D8DD20D013AE
:105B30001D0520D860D80DDD5F88C4DD5EC4580D1A
:105B40004D5058D582050D81318D05028D5856D5A1
:105B5000ED805E4DD5FF86D50DDDDD80DD02050DC6
:105B6000061318D05020DD80DDDDD0D5FF77DD5E57
:105B7000580DE5820DED2310D450168545858DDD39
:105B80008D58DDFF77DD5E580DD505628D82310DB4
:105B9000D510D45885E4580DE4DD5F97CDDDDC5891
:105BA00088DD0DD0D862850D8231050D851D50D858
:105BB0005880DDDDD5FF99CDDEC58DD5C5888DD06A
:105BC000D58D062858D0231050DD51D505E45888CE
:105BD0005E4580585E4DDDDF67CDD54D80DD80D8D8
:105BE00030D50162D5830DD8DEDD5F664DDE458D93
:105BF000ED030D501620D838D858DDDDFF66CDD521
:105C00004D80D5038D0162D5838DD80DDDDF784DB4
:105C1000D5E4580DED058D503058D162050D038542
:105C20000DD885C58D5CDDFF77CDDEC585ED58DDF2
:105C300050238D83106D80DD58DEDD5F86DD5E587C
:105C40000DDD80580D5023685450318D458DDE4D4B
:105C5000DF77CDDEC5605EC58DED5230D58318D8B7
:105C600088DDD85CCDDF87CC4DDDDD8D8D80D80221
:105C700038D85310DD860DE458D5E4DDFF75DD0D11
:105C8000D60D50D0A0DD02018D509854DDD5FF68AF
:105C9000DDE585E560D5E50A0D502010DD9054580E
:105CA0000D45805E4DD5FF66DDDE5885E5885ED00A
:105CB000AD45026154D095CDD5FF65CDDDD80D0A37
:105CC00050D02610D890DDDDFF75C4DDDD568D8205
:105CD000310D880D58DDDD5FA6CCCDD5C4DD80DD6E
:105CE000582310D823180D50680DDD8DDEDDFF76AA
:105CF000DDDD58580D0A310D01810D013A6D8058D6
:105D0000DDDD5F85DDDDD80680D1A1A1D29292D8FC
:105D10000580DDDDDFE6CCCCDDE4DDD0585E4588F6
:105D2000D520DE4D06091020DECD02D588DC458564
:105D3000058805C4DD0DDD5FF7DDD58DDE588058A3
:105D4000585ED028DD20DE4D02099020DECD8DD8B2
:105D500060DC4585858805C4DD858DDCCCC4DDFF30
:105D6000894DDD5E458DDE4580205ED251515E5805
:105D70005650D50251510D8828DD505854D580D445
:105D8000DDD5FF77DDDD501810D1AA1D02920D027E
:105D90001720D1AA1D01810DDDD5FFAACCDDECC5F0
:105DA00085ECD521DED58805E501838DD020363000
:105DB00020DD0B30105C5880D5CD12D5EC4585EC3C
:105DC0004DDF67DDDD8506D02120D01210D0121006
:105DD000D02120D858DDDDFF68DDDD868D02020D83
:105DE0005131DD80D502120D01210D858DDDDF6879
:105DF0004DDD45068545032054501DD50A0D890DFE
:105E000080DD8DEDD5FF78CDDDC5068DD218D010A3
:105E10002DD052105E5050505E58805ED80DE4DD9B
:105E20005FA64DDDDED858D5ED125830D5806030F4
:105E300030D80D88DDD580DCC4DD5F86CCDDDDD8D3
:105E40000D501B60D8280D50D0DD5885EDDDFF6763
:105E5000DD5E580DD868D523515458A54509054530
:105E600083054DDDFF98CDD5E4D8DD54D888545056
:105E70001B28D505856D582B105E5888DEDD58DE51
:105E8000C4DD5F774DD5ED58DE5828D565250D501A
:105E900012101DD8854D8D5CDD5F764DD5E458051B
:105EA000ED80DD0B90D82026D8D8DDDD5F784DD58C
:105EB000ED585ED030DD828D565250D5012101DD86
:105EC000885C58D5CDD5FF864DDD5E458185E4588B
:105ED0002505ED5B60D4582505E458185E4DDD5F5F
:105EE0008ACC5E4DDD5E458585E4560285E45831F9
:105EF00005ED5303D54501385E458285E458585E6B
:105F00004DDD5ECC5FA9CCC5EDDDDDED580585E549
:105F100006931205E502020585EDD5050D5CC50564
:105F200085ECC5885ECCD585ECCDDDFFE7CCC4DD46
:105F3000DDDDDD580DD509980580D856D58850D0BF
:105F4000AA050588D88858050DDDDDD80DCCC4DD3F
:105F5000DDFF78C4DD5C4580DD580D892D58920D3C
:105F6000525650D0288D80DDDD5F97CC4DD5CDD8F1
:105F700005C58028DD852DD830185E58030565EDF0
:105F8000D5185ECCDD5FA8CC4DD5E4DD5805E458CE
:105F900050250DD0B838D8316580D8B0580D580D7F
:105FA000DD45805E4DD5FFC8CDDE4D8DDD5ED83040
:105FB00020585E583038B0D588056138DD8D0B85A6
:105FC000CDDD80DCCC45805ECCC4DD5F774DDED896
:105FD000D5E5818D58158D023A0DD18DC5865ECDE2
:105FE000D5FF994DDD5E45858DD5125090D0128A32
:105FF0000D80D0DDDD580D01888D0206521DD5853E
:1060000085ECDDD5FF88DDDDD80580D0505050D837
:106010003238DD161DD83238D0505050D8880DDDBA
:10602000DDFF874DDED8DDD83018D821250D83035C
:1060300060D5021210DD858DDDDDFF884DDD5E58F7
:106040000180D0525250D0210120D158051D02109C
:10605000120D0525250D8078054DDD5F88CDD5E431
:10606000D010DED12021D50203020D1036301D02E2
:1060700003020D512021D4D010DECDD5FF884DDD97
:106080005ED880D50212120D0121210D0216120DCB
:106090000121210D0212120D5880D4DDD5FFB6CC9E
:1060A000CCDDDDDD58D8881010D0A28058DD0DD0B1
:1060B000105C56880D5CDDDDFFC7C4DD8DDDD8DDED
:1060C0008D80280910D82028058DD50DD0105C5062
:1060D0002868D5C580DD5ECDD5FFA9DDDDE580581A
:1060E000DD50506880D05020A50D853D80D58318A7
:1060F000D54D90D5EC58DEC585ECDDFFEA4DDDDDF4
:10610000DE458058885E45058A5250DE4505888800
:1061100005E450D50DD505E450650990505ED85082
:1061200099050D58DDD2D8D828288A0DD580580574
:1061300085C4DDDDDDFF89DDD5E58805E51D50DDA4
:106140001502020D15828D1502020D1D560D58887F
:106150005E58DD5EDDFF89DDD5E58805E51D50DD96
:106160001502020D15828D1502020D1D06DD880532
:10617000E58DDEDDFF89DDD5E58805E51D50DD1502
:1061800002020D15828D1502020D1560DD5885E5A0
:106190008D5EDDFF68DDDDD80D51210D0212D501C8
:1061A000210D02120D5806DDDDDDD5FF68DDDD585D
:1061B0008D51210D02120D0121D502120D5806DD5F
:1061C0008DDDD5FF68DDDD588D51210D0212D50121
:1061D00021D502120D5806DD58DDDDFF68DDDDD862
:1061E0000D51210D0212D50121D502120D5806D5EF
:1061F0008DDDDDFFA84DDDD5ED858DDD125838D85C
:106200000603030D805838DDD530D5CCD80DCCD859
:106210000DCC4DD5FFF8DDDD5ED588D8DDE58830C5
:10622000D8585E50BB8DD21D58363888210D8BB0A2
:10623000DD80D5038858DDD588D5EDDDD5FFA94DA6
:10624000DE458DDD5450230580545892050DD05005
:10625000380D803056DD0502985E580503205EDD5E
:10626000D585ECCCDDFFCA4DDE458D5E450230DDC7
:10627000D54581020580DD050102050D8013531807
:106280000D050201056DD805020185EDDD503205D1
:10629000ECCCD585ECCCCDDFA8CDDD5ED5858DD819
:1062A000023280D050121050D052171250D05012DB
:1062B0001050D8032380DD858D5CDDD5FFA8CDDDB2
:1062C0005ED5858DD80B2020D05012180D0D170DDE
:1062D0000D80121050D020B280DD858D5CDDD5FFA1
:1062E00088DDDDE580585E5823205E5812105ED5AB
:1062F00018D5450161854502328545858054DDDD2F
:10630000FF884DDD5E458805ED0B20D5021218D0C3
:10631000516150D812120D50B20D458805E4DDD5FB
:10632000FF7ACCDDDD58D020A0D0938D510250549F
:106330005968D510250D0938D020A0DDD85CCDDFF7
:106340008ACC4DD4DD58545020A05450938DD15256
:1063500050D02968D8102DDD185ECD205EC4585E5F
:10636000C4DDFFAACC4DDEC4D58D5CD0A02054D0B6
:10637000918054501D020DD212132DE5021D185E9E
:106380005809185ED020A6DE4D58D5EC4DDF99CCCB
:10639000DDEDD585E50212035E581010DDD310A0A7
:1063A000545016180D521021DD0205205E58885EEB
:1063B000DDDDFFCADDDDDDD88D588D0A02020A0D54
:1063C000D0156510D5C5098105ECD15351DEC50145
:1063D0008905ED50150510DD0A02020A0D88D588E1
:1063E000DDDDDDDF8A4DD5E45805E45050DD4502A2
:1063F000138545012030DD35216D812030D05213C9
:106400008D8858D80DDDDDFF8A4DD5E4580DD45068
:10641000505854502138545012030DD35216D812EC
:10642000120D0521210D8858DDD585CC4DDF9A4D03
:10643000DE458DD5E45820205ED053905E58180D6F
:10644000D0A9A0DD8016054509350D45020285E479
:10645000DD585ECC4DDF9ACC4DDECDD85EC585854E
:10646000EC50A205ED59915E585212DE580210DD33
:106470000281060DD521285C458DDC4DDF9ACCDDEF
:10648000E4DD85E458585ED21521DD0212018D81CC
:1064900052120D5216012D45023185E4D80D5EC50C
:1064A000805ECDD5FF994DDD5E45858DE45125217A
:1064B0000D451202185450101020D521512DD02016
:1064C00010205E50605805ED8DD5E4DDFF8A4DDD6E
:1064D0005E458805ED05250D50102010D0210120C6
:1064E000DD030DD0216120D0102010D505250D45EC
:1064F0008805E4DDD5FF88DDD5E58585E512521DEB
:10650000D030380D81820D5030DD58305E586DED41
:10651000D5FFE8CCC45E4DDDDDD5E4581880185EAB
:10652000450121A212105ED1A2131A21D450121AD1
:10653000212105E45601880185E4DDDDDD5ECCC462
:106540005FE8CCC505E4DDDDDD5E4588121885ED2C
:10655000128212821D4521B30B3125ED1282128267
:106560001D45680121885E4DDDDDD5ECCC505FE82E
:10657000CCCD5E4DDDDDD5E45821801285ED830163
:1065800021038DD821232128DD830121038D45603E
:1065900021801285E4DDDDDD5ECCCD5FE8CC4505F4
:1065A00005E4DDDDDD5E45028880105E4501B80B47
:1065B000205ED038B3830D4502B80B105E4561886C
:1065C00080205E4DDDDDD5ECC450505FE8CC4D0D34
:1065D000E4DDDDDD5ED80180180DD0A3A23A0D45C3
:1065E00099139915ED0A3A23A0DD68180180D4DDCE
:1065F000DDDD5ECC4D0DFFE8C4D5050D5E4DDDDD66
:10660000D5E4588018805ED0120A21210DD32129AB
:1066100013123DD0121A20210D4568818805E4DD52
:10662000DDDD5EC4D5050D5FE8C50505050505E49E
:10663000DDDDDD5ED8181818D450A30A30205ED1F5
:106640003130303131D450203A03A05ED6018181FF
:106650008D4DDDDDD5EC50505050505FE8CD0D0D27
:106660000DE4DDDDDD5ED810101018DD021212120F
:10667000120D453A2030A235ED02121212120DD63B
:10668000010101018D4DDDDDD5ECD0D0D0DFF9CD9C
:1066900050DD0D5E4DDDDDDDED888888D452128140
:1066A0002121215ED121212121212DD2121212126C
:1066B000121D45121212182125ED6888880D4DDD36
:1066C000DDDDECD50DD0D5FFF9CD050D050DE4DDF3
:1066D000DDDDDED888888DDB1BA231BD45821092BE
:1066E0001285E458212901285EDB13A2B1BDD688AA
:1066F0008880D4DDDDDDDECD050D050DFFF9CDD8BB
:106700008DDE4DDDDDDDED8098980DD02323AA329E
:106710000D45031090121205E45021210901305E4D
:10672000D023AA32320DD6898980D4DDDDDDDECDDD
:10673000D88DDFF9CDD58DD5E4DDDDDDDED02010BF
:106740002102010DD8202121018DD1212182121297
:10675000DD21212812121DD8101212028DD6102010
:106760001201020D4DDDDDDDECDD58DD5FAAC4D583
:10677000ECD050DD4D8D58D502888D8062058DD0CE
:106780002D585C5859854D0D150D45888DE4588060
:10679000DE4DDD5F884D0DDD50D010D0D021054D90
:1067A0000280D50260DD028DE590D0D58050DEDD1F
:1067B000505FC9CDDDDD54D880586DD020A580D084
:1067C000D288A0D85820580DDD50DDD59092053DD7
:1067D000E50988D5E589DD5EDDDD5FCACCDDD5EC78
:1067E000C5880DEDD50D58D5888058D562B310D227
:1067F0000D8588D01D58D8502054D8DD1215CD886D
:10680000885C4DDD8DCCCCDDFF88DDDDD10188D10C
:1068100021018D50D560545828D450A0DE45820502
:10682000E458D5E4DDFFA8CDDED58DDE580680DE48
:1068300050510151DD0A20A20DD151515054D88838
:1068400005CDD8D5CC4DDF974DDD5ED88050D83101
:10685000215E583151DD0526A8D80D050DDD5805FE
:10686000CC4DD5FF8AC4DDEC45605ECD85EC501281
:106870005EC52105ED592DD8928D0202050DDD056D
:1068800005CC5805CCDD5F87CC4DDCC458DDD52167
:10689000D802021D026291D0A29D582095EDDDDF45
:1068A000E5DD50DDDDE580D5010285E58020390597
:1068B00020DD025093028654582010D58054DDDD2F
:1068C0000DD5FF9ADD5E580DD5E502020205ED50AB
:1068D00050505EC505805E4D0D50D45099165450F1
:1068E000202805450D50D5458805E4DDD5FF9ACC17
:1068F0004DDEDDD95E5880105E585895E58D0D5EF1
:1069000058828D58505206D8502020D8D020DDD53E
:10691000805ECCDD5FAA58D5E4D80DE4531285E53E
:106920000121201DE502121285E58216128545829D
:106930001212054D10212105C4582135EC4D80DE81
:10694000CC4D585FC64DD58DD54580DD80D5052110
:10695000312050D802161280D0502131250D580D0B
:10696000D805EDD58DD5FFCA4DDDDD5ED88588D53E
:106970000A31213A0D9188091D0A31213A0D5883B7
:1069800088D50A31213A0D9186891D0A31213A0DA7
:10699000588588D4DDDDD5FFC9CCCDDEDDD585E5D4
:1069A000880301DE50A5838DE5026053038DD0205E
:1069B00050303854D5051030305458018581545822
:1069C000058DD54DDDDFE94DDDDD5ED888805E5873
:1069D000DDD52DE505888020DD0591B313160D0565
:1069E00088802050D8DDD5258D5888828D4DDDD802
:1069F0000DECCCCDD5FFE8CCCCCDD5CDDDD580DD33
:106A00000202020218D812120212150D05139693F3
:106A1000150D051212021218D8120202020DD80D1D
:106A2000DDD5EDD5FFAA4DDDD5ED80380D585050A0
:106A300058D051212150D8212128D351262153D873
:106A4000212128D051212150D8505058D580380DBF
:106A50004DDDD5FFA9C4DDEDD85E5880DDE502052A
:106A6000810D5858018D505A518D588DDD060D5E9F
:106A70005805EDD5FF98CC4DDDDD580D82880D828F
:106A8000D50DD12101015450258854506DDD458527
:106A9000E4DDFF88CCDD54DD8054506025054505DC
:106AA00099D5202020D8D50D58885EDD585ECCDDE4
:106AB000FF89CDDDEC5810DC505385C5021205CDA1
:106AC000031054D02160D5050120D8A150D888DD0D
:106AD000DDDF794DDE4585ED01D5E581205E53038F
:106AE0008D5021A0D8180DD3DDC565ECD5FFB8DDDC
:106AF000DDD5E56858585E582528025ED859585E9D
:106B000045859585E4585958D452802528545858BD
:106B100058054DDDDD5F99CDDDD4D9906545850102
:106B20008D505850D58520505E5028050DD520D861
:106B30005C580A05C580585CDDDDFFAA4DDDE458D0
:106B40008DD54502035805458303020DD301038DFE
:106B5000030161030D830103DD02030385E5805317
:106B60000205EDD5885ECCDDDFAADDDDDD88388D60
:106B70000A0D020D8295A0D0D31318D3596953D8AA
:106B80001313D0D0A5928D020D0A0D88388DDDDD4E
:106B9000DFA94DDDD5E45803805E450D0D05E458B1
:106BA00030385ED5858DD8125218D0586850D8121A
:106BB0005218DD858D5CDDD5FFC9DDE58DDDD5E5C0
:106BC00088D885E50A258805ED91505A25E45915A0
:106BD00005915E45A28591D4588DA2054DDD506882
:106BE0005CCC4DDDFFC8CDDDD5E4D805805ED02579
:106BF00005052DD805101580D02031613020D8052D
:106C0000101580DD25050520DC580580DECDDDD59D
:106C1000FFF9CDD8DDEC58DD8DDED5880202805E2F
:106C20005885028391D502050DD0590D58058888E5
:106C300005450A0A60591D458058DDD5E4DD8050C0
:106C40005ECCDD5FBACCC4DDECDDD85E4D82820562
:106C5000ED8205285E582058025E58050D8DD52816
:106C60009585C58539165C5809DDC58DDECDDFDA21
:106C7000C4DD50DD5C45060D5805C450502880DD4C
:106C80005052020DD588502025E50D5020205E5928
:106C900099150DEDD0D0585EC4588585EC4DDD8535
:106CA000ECCCCDDFAAC4D0DE4D858DE4D880DE5893
:106CB000325238D82912854505161505E5829128E6
:106CC000D832523854D880DE4D858DEC4D0DFF6999
:106CD000DDE58D5E5885E50285ED50DD02020D96FD
:106CE0009D828DD8DCDDFF77DD5E586DD58218DDA5
:106CF0002150D82150D05218D88DDDD5FF89C4DD60
:106D00005EC45805EDD0505E50101505E581805EDB
:106D1000501D02DD85A054D80265CD8D5C4DDF98F5
:106D2000DD0DDE58D585E5850A05E50A0585E5888A
:106D300058DD5021585C5931615CD80D5C4DD5FF50
:106D4000A9DDD0DD588D58D0388030D505B35854E2
:106D5000583738DD0532350D58505058D88880D80E
:106D6000DDDDDDFFA9CDDDDE4D810105E4503250D2
:106D7000505E45185250DD305858D8050380D02554
:106D800060158D88020DD585805E4DDDDFC9C4DDBF
:106D9000EC4585EC45205EC45850DDEDD0DD85E541
:106DA0008090985E5823103126D5805202528DDD96
:106DB000805805CCDDDD5F994DDDDED888D501DD5D
:106DC0008D018850D030A050D03D058D078050D522
:106DD00002D585ED880DE4DDD5FF69DDDD868D0208
:106DE000120D5121DD020D502120D01210D01210B1
:106DF000D858DDDDFF88CCDD54DD805458A50D501A
:106E00003920D601518D02930D505A85E580DDED74
:106E1000D5FFA8DDD5E5880DDE50505018D50A2BDA
:106E2000A0D99699D0ABA20D5810505054DD8805CA
:106E3000CCDDD5FFB8CDDDDEC50580DEDD5050DD13
:106E40005020A02020D99999D02020A020DD50509A
:106E5000DD5CD060505ECDDDDFBACDDDDEC588857E
:106E6000ED53DD15E58820205E505999DD05205849
:106E700080D0510565050D0AD05250D8280280D81F
:106E8000DDDDDD5FAA4DDDD5E45805805ED05050D4
:106E900050D5031323130D88588DD02620DD885834
:106EA0008D031323130D50505050D45805805E4D60
:106EB000DDD5FFE84DD5ED80D0DDE585850585E59F
:106EC00003230D520DE50121091020DE503230D58B
:106ED00088D5858505886D580D0DDD54DD5F96DDFF
:106EE000DDD580588D05AA20D815158D8918DD505F
:106EF00060D5ECDD5F974DDDDED888D583938D05B9
:106F000028256D8BB8D5880D54D58DEC4DDF96CDE9
:106F1000DD5ED58585E581A10D5838360D501A18EE
:106F2000545858D54DDD5FC8CCCDDECDD58DD4D8E5
:106F300005828545015050538D50386830D58350B7
:106F4000505105E5828580DEDD8DD5EC4DDFC6CD67
:106F5000DDDEC58885ED50D050DD5831B0138D820F
:106F60008025060DDDD80D5CCCDD5FA8DDDDDD887C
:106F7000688D0D52D50D050121050D052010250D3B
:106F80008210128DD21012D5C58185ECDDD5FFAAF5
:106F90004DDD5E458805E4502020DDD50D018D8056
:106FA00051028D068153DDD05905ED020585E5803E
:106FB00020205E580D105EDDDD5FA8CCC4DDCDDD88
:106FC00085C58852154D0D058545020AA0D51313B8
:106FD000139D880680D80DDDDDDFAADD50DDDDDD07
:106FE000DDD80180DD0121210DD0232320D45926B5
:106FF000295ED0232320DD0121210DD80180DDDD94
:10700000DDDDD0DD5F99DDDDD50D858D05030DDD81
:10701000520120D58106030D038018D502102DDD05
:10702000503050D858D0DDDDD5FF99DDDDD580D882
:107030000D0218120D01B2310D5020630DD0382011
:10704000D50132B10D0218120D80D80DDDDD5F992A
:10705000DDDDDD5880D50213132D503520510D0193
:1070600086230D0328010D01502530D52313120D61
:107070005880DDDDDD5F99DDDDDD88DDD12121207A
:10708000D52121210D01206120D0218210D01212A2
:1070900012D50212121DDD88DDDDDDFF99DDDDD5A3
:1070A00082188D83838D030B032D8306301D1038CA
:1070B00038D230B030D83838D88128DDDDD5FF99C6
:1070C0004DDDDED8680D505212150D02121210D08F
:1070D000128120D0218210D01212120D05121250EE
:1070E000D5888D4DDDDF99DDDDD58880D502121282
:1070F00010D01212120D021D210D012D120D0212BF
:107100001210D01212120D58886DDDDD5F99DDDD91
:10711000D5801280D812128D01212120D121D212C6
:10712000D212D121D02121210D821218D802186D3E
:10713000DDDD5FAACDDD5E4D0D8DEDD582DD020971
:10714000850D803231DD50126210DD5132380D056F
:1071500089020DD28DD54D8D0DECDDD5FFAACDDD8B
:107160005E4D880DED52802DD021303120D8313147
:1071700038D8036380D8313138D021303120DD2830
:1071800002D54D880DECDDD5FFAACCDDE4DD8DE424
:1071900058503D5ED125830D580603030D805838A5
:1071A000DDD030305CCD030DCCD805ECC4D85ECC3E
:1071B000CDDF99CC4DD5CDD805C58028DD852DD81E
:1071C00030185E503030565E5830385ED50301DEE0
:1071D000CD805EC4DD5FE8CCDDEC4D8DDD5ECD8322
:1071E000020585E4D83038B0DD8303056138D83036
:1071F00030D0B8D880DD80DD58D85805ECDD80DD92
:107200005F88DDDDD80580D050580D01292D582923
:1072100020DD256505450218054580DD4DD5FFB704
:10722000CDDDDEC56858D5C5028280DD52D2D0D012
:10723000130130131D88888D585858D4DDDDDF8840
:10724000DDDDD85805E5123251D5812020D5091849
:10725000D02820D502D515E58068DDDDD5FF87CDA6
:10726000DEC58D5ED5018D580158D0A3A0DD018DFE
:10727000C501065ECDDDFF86DDDDD020180D80580E
:107280000DB30B3D805060D812120DDDDDFF88C4B8
:10729000DDEC458DDD5218D803010D6515250D0275
:1072A0000380D812DDD585ECDDFF98C4DDD5CD880F
:1072B0000DD01D50D0202850D631298D02028DDDF1
:1072C00005105EC580DECDD5FF67DDDE503015E5EB
:1072D0001825E515215E5802DD60205458854DDDE6
:1072E000FF87CCDDDDD060D82820D8BB1D81058D7F
:1072F0008D50DD8805E4DDD5FFAACCCDDEDDD5855A
:10730000E5883805E581212105ED02D5205E45316E
:10731000505135E4502D520D4501212185458038CD
:10732000854568DDD4DD5FB8DDDE588DDDD0D02049
:107330002020D810505050DD928685C5950DD5CDB2
:107340000525EC45805EC4DD5F9AC4DDE4D58DE49F
:1073500050A10D5450121A054D81010DD0650DD06C
:107360001018DE50A12105ED501A05ECD8D5EC4DD2
:10737000DFEACDDEC5850DD5EC5215ED58DDDDE536
:107380008888805E5051B39351DD0A2868A20DD1E0
:10739000DD5051505C58888805CDDDD8D5CCCC4D1A
:1073A000DFAACC4DDEDDD065E5858205E5821510CE
:1073B0005E588510DDD2131A05C50151805CD28D4F
:1073C000DC5020DEC5805ECDD5FFA9C4DDD5E4D577
:1073D000880D4583938545052825654583A38D58EC
:1073E000910DD825805E50B0DDE5885EDDDFFACCFA
:1073F000CCCDDDCCCCC588DDDDDD0D0D802102825C
:10740000850D0502931731050D80210282850DDD62
:10741000D0D0D505CCC5858835CCCD0DD505CCC40F
:10742000588805CCC4DDDD5FA8C4DDECD8DDDD8681
:10743000058D023212320D8101018D50123210D4AD
:10744000D858DECDD85EC4DDDFA8CCDD5EDD580DBA
:10745000E580505205E5058318D5023161320D589B
:1074600013850545025058054D80DD5CDD5F87DDE5
:10747000E58DDE5858DE51232105E5888D50123206
:1074800016D5858054DDDDFF99CCCDDCCC58DDDD13
:1074900020D8262020D0131318D82328DD929DE46D
:1074A00058585E458585E4DDD5FFA8CC4DDECC453A
:1074B00085ECDD205ED501010DD02307238D8101F0
:1074C0000150D50250A854D8058DCDDDDFB9CCCC04
:1074D000DDCCCD58DDDD88D802888D802D50DDD102
:1074E000291015EC5025885EC5020DD5EC50605E64
:1074F000CDD5FF78C4DDDD5060D02850D101250DF9
:10750000150150D81250D520285458DD4DDF88CCB5
:107510004DD4DD58D582030D812120D0103036D5D1
:107520000121215458203054D8585CDDD5FF8ACC35
:107530004DD4DD58D582030D812120D0103036D5B1
:107540000121215458303054501212054582030550
:107550004D8585CDDD5FD94DDDDD5E45888805ED46
:10756000151215152DD02125210180D012101015CE
:10757000256D02153515820D85820280D50A80DDC4
:10758000DE58DD5EDDFFAACDD5E4D8DD5E4D858019
:10759000D45832318D5031838DD20602DD83813053
:1075A000D58132385ED8058DE4DD58DECCDD5FAAAA
:1075B000D50DD5E50D58D5ED58380D4583A18D5025
:1075C00030928D032161230D829030D581A385ED0A
:1075D0008038D54D58D505CDD50D5FAACC4DDD4DA4
:1075E000D8DD4D8318D4583A185450381210D03280
:1075F000060230D01218305E581A385ED8138DED5E
:10760000D8DDEDDDFFAAD0DD50DDD8DD54582128CE
:107610005ED059050DD20202120D0905090D0212A4
:107620000202DD050950D45821285EDD560DDD0D1E
:10763000D50DFFF7DDDD8DDDD588DD580D80D8D582
:10764000028D068050D028DD0D09938DE502802D36
:1076500058DE58058DDDEDDDD8DFAADD58DD580D8B
:10766000D8D88818D52D5053054581A50D45051648
:107670001505ED05A185E50350D52D581888D8DDF1
:1076800080DD58DD5FA8C4DDE4D58D5E458038DD42
:107690005821280D031363130D802128DD58380568
:1076A000ECD58D5ECCDDFF974DD5E4580DD5450565
:1076B000A020D5016180D03159DD80A85EDD58055C
:1076C000ECCDD5FF88DDE58D5E58105E50121DDDD6
:1076D00003885450A62054501DD54585E4DDFF99FC
:1076E000C4DDDEC458605EC4505205EC4501315E15
:1076F0004DD520DD0101010D0202028D050DDD5881
:1077000005EDD5FFE9CDD5EC518DDDD5C5150DD5F0
:10771000805C532888805C51DD50505054D1DD5A34
:10772000020D501888D20D860580D58D80DDD0DD04
:10773000DD580DDFA9C4DDEDD8DE582060D5E58D1C
:10774000028DD1D015854505102020545150215867
:1077500054588DD5458D5E4DDFB7DD5E58050DDD86
:10776000582D5921D5060D98545825095154D0202B
:10777000AA05C58880DCDDDD5F9ACC4DD5CDD80566
:10778000C58028DD852DD830185E50303056D58321
:107790000380DD0303505CD030105C4D80DCCDD520
:1077A000FFAA4DDD5ED058D5E58288DED103058D78
:1077B00058303050D58036380D50503038D585038C
:1077C00001D4D88285CD5850DC4DDD5FAADD580D3F
:1077D000D58DDDD512D58054502802854512105024
:1077E0001D4505060505ED10501215E58280205E49
:1077F000580D521DDDD58DD580DD5F884DDD5ED8FD
:107800008DD503038D0312130D82628D0312130DA8
:1078100083030DD588D4DDD5FF88DDDDD805050DC2
:1078200050A80D89120D521612D502918D80A0D547
:10783000050580DDDDDF884DDD5ED880D5030203E0
:107840000D85058D510601D585058D0302030D5863
:1078500038D4DDD5FFAAC4DDDEC45885EDD0585E2E
:107860005812121DD8212128D051262150D821216B
:1078700028DD1212185C5850DDC5885ECDDDFFAAE8
:10788000CC4DDEC4D585EDD885E5812121DE58219A
:1078900021205ED0126210D45021212854D1212100
:1078A00085C588DDC58D5ECDDFAADD50DDD80D58DC
:1078B0000D0583850D8391320D501A210D4530261B
:1078C0002035ED01A210D50239138D0583850D8079
:1078D000D580DDD0DD5F97DDDED8DED02DDD5860D0
:1078E00058D50103521DD50302105C58885CDDDDBC
:1078F000FF67DDDD58DD580D501AD50380D9520DD4
:10790000806DDDD5FF77DDE58DDD810DD830DD5073
:10791000380545032605458DD4DDD5FF774DDD546B
:10792000D8D545010DD50380D06B20D88DD8DDDDAD
:107930005F794DD5E450605ED050DD0152DD0388A3
:10794000D0388D0152DD5050D545805E4DD5FF9920
:10795000DDDDED5885ED52D65E5013905E58A0DD0A
:10796000D505885C588505CD05805CD80D5CDDDDCE
:10797000FFC7DDDED8DED02DDDDD8605858D50101C
:107980003521521DD50302102105C5888805CDDD9E
:10799000DD5F99DD5ED85ED02DE58605E50103DD6E
:1079A000DD030285C5810305CD50585CC580DCCD63
:1079B000DDFFBAC4DDDD5C458880DD5020A20D808E
:1079C0002525050D13939210D52515958D580591F4
:1079D0000DD5206028DC502020DDCD8D5ECDDD5F13
:1079E000C8D58880DDDDDDDDD50101010D545012E3
:1079F0000302105E450A23A205E450120302105E42
:107A0000D50107010DDDDDDDDD58880D5FC84D585E
:107A100080D5E50DDDD50DD018010DD58212128D62
:107A20004513A0A315ED8212128DD50106010DD0CC
:107A3000DDDD5054D5880D5FC8CDDDD5ECD8D85EDE
:107A4000DD120102DD02028510DD815060518DD012
:107A50001582020DD201021DDC58D8DECDDDD5FF26
:107A6000AADD8DDD8DD80D8805020D5021238054AF
:107A70005013153D54502161205ED53513105E58CA
:107A8000032120D50205880D80DD8DDD8DDF88CCBA
:107A90004DDDDD8D583030D812120D803036D812C1
:107AA000120D58303054D8585CDDD5FF984DDDD5D7
:107AB0004D88D54D052120D50121056D8030120D51
:107AC000812152DD058805458058054DDDD5FF8AA9
:107AD000CDDEC585ED502DD581210D5020102DD046
:107AE00052120D821056D83018D012150DDD80DCE0
:107AF0004DD5FFCADDD0DDD588DD80D8580588D8C2
:107B0000213031250D5012010218DD3523253DD8D5
:107B100012010210D50521303128D8858058D80DA2
:107B2000D806DDD50DDDFFF8C4DD0DDECD8D58DDC9
:107B3000DD88580580D0232123212328D810101058
:107B40001018DD01232123210DE4D8506580DECDFE
:107B5000D8DD5ECC4DDF97CDDDD4D01806D5012120
:107B6000210D821230D5021230DEDD805EC4580550
:107B7000EC4DD5FFA7DDD5E5818DE5060A0D5ED577
:107B80002918DD51020A0DDD5290D0DD1020DDDD17
:107B9000DDFFD9CCC4DDD5CCCD8185CCD50A060599
:107BA000C4D8912D54D50A0201DD58912DDD50A085
:107BB000201DD0D092DDDDD0201D505050DDDDDD08
:107BC000D5FF37DD561D20D8D02D10D8DD5F47DD1D
:107BD000D81D020D56DD2D580D18DDDF64DDDD10DA
:107BE000501D02620D858DDDDF54DDD5180DA8D640
:107BF0001DDD5F74DDD5E57180D5050A0D888DDD4D
:107C0000D5FF544DDD581D628D830DDD5F74C4DDDD
:107C1000DD580D62850D10281DDDD5FF74DDDD58A2
:107C2000158D82620D8D01DDDD5F47DDD18D020D89
:107C300056D5120D80D8DDDF74DDD5E5858D502653
:107C400028D10581DDDD5F47DDD81D020D56D51237
:107C50000D80D8DDDF64DDDD6058D8A0D8101DDDD3
:107C6000DF74DDDD58058D82620D81501DDDD5FF8D
:107C700077DDDD560580D8518D85020D5020D54524
:107C8000805E45185E4DD5FF474DDD60D020D80D94
:107C900058545215450154DDFF47DDD68D80D02064
:107CA000D12D5105E585EDDF67DDDD881D882D854A
:107CB0008DD50DC56205C5185CDD5F46DDD68D022C
:107CC0000D501545205450154DDF47DDD68D80D021
:107CD00020D20D5101D80DDDFF74DDDD57188D0266
:107CE000028DD58DC4DDFF74DDDD501568D8028DA1
:107CF0008380DDDD5F46DDD78D83D020D58545854A
:107D00004DDF77DD5E5805E5805E58DDD521560DE7
:107D10008820D80501DDDD5F46DDE585E510D5026B
:107D20006D020D10DDDF76DDD5E560595E58805EB1
:107D3000502020D58058DDD85CCDDF77DDDD5605BD
:107D400018D888D8518D8D8D0A80D8058DDDD5FF46
:107D500077CCDDCC58DDD01D68520D8802D8801D4F
:107D6000585854DDD5FF77DD5E56015E5805ED218C
:107D7000DD58580D8280D80DDDD5FF46DDE595E54F
:107D800002D5026D020D50154DDF77DDDD5601582D
:107D9000D80201D8058DD50205C45805C45805C4BC
:107DA000DD5F77DDDD56880D82020D80DD58595E7E
:107DB00058805E58805EDDD5FF77CDD5EC5685ECDA
:107DC0005805ED582D595020D888D888DDDD5F77CB
:107DD0004DD5ED685E50285E5820DED580DC588594
:107DE000C5895CDDDF77DDD5E501815E505805E5AD
:107DF00088DE58026D585020DD5805C4DD5F74DD03
:107E0000E560DDD82020D898DDDD5F77DDE560DD39
:107E1000D80510D8058D858D58A05E58815EDDD5BA
:107E2000FF77DD5E5685E5805E5020DD530518D86E
:107E300088D8058DDDD5FF77DDDD56858D02058D72
:107E40008058D02518D888D8518DDDD5FF77DDDD55
:107E500056859D888D58020D80DD58820D888DDDF8
:107E6000D5FF77DDDD5601010D8850DD580D82808C
:107E7000D052050D888DDDD5FF764DDDE456905E40
:107E8000D058D58580D0A80D588054DDD5FF674DDA
:107E9000DED615E50205E5020DD0258D1801D58D3C
:107EA00054DDFF744DDDD58261D82021D18DDDD523
:107EB000FF474DDD61D18D020D02D585E585EDDFF2
:107EC000744DDDD5788D8A8D1858DDDD5F77CDDD79
:107ED000C56805C5885C590DDD020D8028D8058D63
:107EE000DDD5FF774DDDD5788D8A8D8058D50D8D08
:107EF0008058D8158DDDD5FF774DDDE456095E45F8
:107F00002805E458DDD288D888D80DDDD5FF77DD87
:107F1000DD5605010D888D85010D02050D502805E2
:107F2000E580D5EDD5FF47DDE570D580D021D520A2
:107F3000D80D80DDDF77DDDD56880D888D8051D549
:107F4000025015E502805ED8D5E4DDFF77DDD5E58A
:107F5000880D58826D02058D8580D8580DD5101575
:107F6000C4DD5F77CCDDC4D60DD518D888D02058B5
:107F7000D05218D888DDDD5F67DD5E5815E5120543
:107F8000E580DD20560D8021D58D54DDFF474DDD88
:107F900060D020D121D521D80D80DDDF47DDD10192
:107FA000D81D020D52054562545854DDFF47DDD1FE
:107FB00001D81D020D5A54560545854DDF47DDE5B4
:107FC000605E585E5AD580D121D18DDDFF77DDD539
:107FD000E56058D5888D8509D8820D82DD5805ED7C
:107FE000D5FF47DDD68D021D02D5020D18D50154EF
:107FF000DDFF77DDDD57809D0A250D50580D8DDDA5
:1080000085E585EDDF77DD5E578DD501018D820237
:108010000D502DD4585E4585E4DDFF77C4DD54D581
:10802000805456028D5802D501585E58805ED10D9D
:108030005E4DDF77DDDE56805E505205E5028DD85D
:10804000580D81010D8580DDDD5F67DD5E51015ECC
:108050005185E5020DD02560D8020D8DDDDF77DD7D
:10806000DD570580D02028D1058D5020D5E5815ED3
:1080700058DEDDFF77DD5E568D5E502805E502D0C7
:10808000D58518D888D8510DDDD5FF67DDDD881D71
:108090008A0D8501D526DD185E5805EDD5FF74DD06
:1080A000DD56809D0A28D8581DDDD5FF774DDDD5DA
:1080B000858D82620D10D20D888D8018D10580DDEE
:1080C000DD5F77DDDD5888D8851D5288D60D01D05B
:1080D0002058D8058DDDD5FF77DDDD560581D885A3
:1080E0001D888D02580D30280D80DDDD5F77DDDDC8
:1080F000501568D015A0D88DD8805E505805E58001
:10810000D5EDD5FF77DDD5E5688D5888D8058DDDAF
:108110000D502028D80101DDDD5F76C4DD5C4510FF
:108120001DD5020D6858D02028D1058DDDD5FF76EC
:10813000DDDD561810D05850D888D02028DD5120C9
:108140005C4DD5FF774DDDED88D562820D8D8D10AC
:10815000158D8058D58DD4DDFF77DDDD56880D0275
:10816000028D50580D121DD5805E5815EDD5FF7744
:10817000DDE5605E585E502DDD8518D120250D5857
:108180008154DDD5FF77DDDD56880D9850D58A0501
:108190004D885451025054588054DDD5FF77C4DDCA
:1081A000DD580D888D880DD9526545802054D58DB8
:1081B000C4DDFF77DDDE56805E505A5E5820DD015B
:1081C000509D888D888DDDD5FF67CDDED560D5804B
:1081D00020D0D8D01520D882D0181DDDDF674DDE25
:1081E000D60DD10101D858D58A54502854D585C40C
:1081F000DDFF77DDDD578101D2880D8D0DD20505BC
:10820000E458205E458D5E4DDF77DDDD58578D8566
:10821000120D830DD80205EDD85EC4585EC4DDFF93
:10822000774DDE45605E4585ED20DD58518D88AD8A
:108230005810154DDD5F77DDD5E58805E515805EC5
:1082400058805E5102DD505628D01280DDDD5F7708
:10825000C4DD54D58054572050D51580D82010D86F
:108260002DD5805EDD5F774DDDD56091D0288D8D79
:108270000D58058D0A80D8058DDDD5FF77DD5E515F
:108280008DD5102560D50280D8038D8058D5858581
:108290004DDD5F77C4DDE4D5605E45885ED12DD5C8
:1082A000888D01A8D01058DDDD5F77DD5E568D5ECC
:1082B000510185E5882D512D8D0288D585854DDDAF
:1082C0005F77DD5E580DD58268D5288545850154D8
:1082D000528854585954DDD5FF77DDE501DDD826A5
:1082E00020D0288D58DD45895E4D585EC4DDFF776E
:1082F000C4DDEC45605EC4585EDD10D581020D0220
:108300000210DDD85CCDDF76DDDD580560D8058D47
:108310005A8D4588054D5095C4DD5F77DD5E590D5A
:108320005E58185ED028DDDA6D888D888DDDD5FF2A
:1083300077DDE58DDD888D02580D80DD51A605EDD8
:10834000895E4DDDFF77C4DD54D58054562050D56D
:10835000A80D8D0D510180D5801054DDD5FF45DD70
:10836000E560D5020D38D81DDDFF74DDDD5105183F
:10837000D02628D8580DDDD5FF47DDD81D020D5673
:10838000D5120D80D80DDDFF76CCDDCC5605CC584E
:10839000DDD8D8020D580315EDDD5F47DDD78D150B
:1083A0000D020D80D020D5854DDF47DDD78D150D11
:1083B00080D020D020D5854DDF64DDDD0181D8A0BF
:1083C000DD60DCDDFF464DD456154520D501D020BB
:1083D000D80DDDFF46DDE585E58D5026D38D81DDA9
:1083E000DF65DD5E580DD8261D05020D18DDDDFFA9
:1083F00074DDDD5601010D8A8D80DDDD5F74DD5E8B
:10840000568DD58A8D8090DDDD5F67CDD5C5601531
:10841000C5020DD50D5850D5828D881DDDDF74DD68
:10842000DD501568D8028D8380DDDD5F47DDD68D98
:1084300080D020D502D101D80DDDFF77CDDDC5601C
:10844000105C58505C5820DD88D020DD5815EDD5E3
:10845000FF574DDE4585E4585ED85E562DD028D8AE
:108460009DDD5F77DDDD58D01D888D10D20D50D891
:10847000D62058D80DDDD5FF77C4DD5C45185C45A6
:1084800080DDD0D56858D8280D80210DDDD5FF7747
:10849000DDDD56880D052020D880D518D5E5188556
:1084A000EDD85EC4DDFF47DDE5605E5025E5105E7A
:1084B000512D580D80DDDF67DDE58DD502620D8D14
:1084C0001D188D880D80DDDDFF77DDDD560518D8A0
:1084D00088D8518D02058D0288D880DDDD5F77DD7B
:1084E000DD580501D80201DDD8D60502D58805E59D
:1084F0008585EDDD5F47DDE5705E5025E5205E5842
:10850000D5021D81DDDF474DD4561545A5458D5259
:108510000D18D18DDDFF77C4DD5C45805C4580DDC5
:108520005020D6858D80201D8158DDDD5F77DD5E92
:108530005685E5805ED02DD50288D05850D1818DEA
:10854000DDD5FF67C4DDDD8D0181D880D0D8D02690
:1085500020DD585C4DDF77CDD5EC56015EC520158A
:10856000ED58DD0288D05850D888DDDD5F74DDDD40
:1085700057858D8A8D518854DDD5FF67DDDD688D87
:108580000528D828D0158D880D518054DDDF77C49B
:10859000DDE4D560D45098D50D8D8058D0A80D88D5
:1085A0008DDDD5FF77DDDD51880D888D50581D623A
:1085B00058D502805ED8D5E4DDFF764DDD5456886F
:1085C000D5880D9058D02028DD58DC4DDF774DDD63
:1085D000ED6805E502805E58DDD020501D888D18BD
:1085E00080DDDD5F774DDED60D5E502805E502D1DA
:1085F0005E58051D5888D888DDDD5F774DDDD5686C
:108600008D0288D8580D8D0D50288D5810154DDDD0
:108610005F77DDDD56859D888D5880D0ADD5880586
:10862000ED885E4DDDFF77C4DD54D5805456280DAE
:1086300058501D85121D85020D8D8DDDD5FF66DD1F
:10864000DD7158D880D8A0DD8DC585ECDDFF77DDE4
:108650005E5805E5805E5120DD510568D8028D58D1
:10866000DD4DDF77DDD5E560510D5888D12580D50A
:108670008DD458205E45885E4DDDFF77C4DD54D52E
:108680008054562050D5828D0158D58585E50158F6
:108690005EDDD5FF77DD5E5685E5805ED20DD58542
:1086A00080D8028D509854DDD5FF77C4DD5C4568D5
:1086B0005C45020DD58D58825E58805E590D5EDD99
:1086C0005F77C4DD54D5701545880D5A80D80DD517
:1086D00005805E58805EDDD5FF77DD5E5601D5E50D
:1086E0008805E510D0DD05020D8028D8058DDDD583
:1086F000FF774DDDED6805E58805E580DD51858D69
:10870000152020D888DDDD5F77DDD5E58560D58053
:10871000A0D8058D8050D505185E581D5EDD5F77A9
:10872000DDD5E5688D5888D8D20D8510D581205EBD
:1087300058585EDDD5FF77DDDD56880D05090D0241
:10874000050DD850D4528854588054DDD5FF77DDBC
:10875000DD578010D8850D5880D8058D02028DD543
:10876000805C4DD5FF76DDDD5105601D025021D8BE
:10877000D8D8820D8D8DDDD5FF77DDD5E5880D58F4
:10878000826D52058D8580D85101D8DDDD5F77C4BB
:10879000DDE4D560D458101D52580D8D8D8280D8DF
:1087A00058DDDD5F77DDDD56858D8058D10D20D514
:1087B00005020D8801D880DDDD5F74DDDD57188D81
:1087C0008A20D1858DDDD5FF774DDDD5880D888D4B
:1087D00020DDD6288D1880D8510DDDD5FF77DDDD61
:1087E00056880D02851D02581D8D8D888D880DDDE2
:1087F000D5FF77DDDD5889D8A8D50581D62DDD8553
:10880000E585EDDF77DDD5E5858D51828D10D8D5F5
:10881000265854585854585854DDD5FF774DDDD557
:108820008560D8028D8580D101DD50205ED85E4DF7
:10883000DF77DDDD5988D8A8D1850DDD6205C45804
:1088400005C458DC4DDF77DDDD585030D8280D8861
:108850008DDD0DC456205C45095C4DD5FF77DDDD0F
:10886000580560D38021D80501D520DD5805E58065
:108870005EDD5F77C4DDEC45605EDD205E588DE532
:10888000881D515028D8038DDDD5FF76DDDD5815C4
:1088900061D051A0D8028D58DD4585E4DDFF77DD3C
:1088A000D5E5010105E58A15ED526DE4580D5458E2
:1088B0008054588054DDD5FF77DD5E5101D5E588C1
:1088C00005E58825ED0526D58820D8018DDDD5FF65
:1088D00077DD5E568D5E5020205E58805E50258D7F
:1088E00058810D5018154DDD5F77C4DD5C4560156E
:1088F000C4580DDD20D888D8A51DD5815C4DD5FF85
:1089000077CCDDDD501D60D21D02D01D50280D88B2
:1089100050D888DDDD5F764DDD54501026D58A0DA8
:108920008D0D58805E59DDEDDF774DDDE458015E39
:10893000450285ED8DD5102560D8820DDD015CCD19
:10894000DF77DD5E578DD515A8D1880D80DD5825E0
:10895000ED85E4DDFF77DDDD56858D888DD2805C89
:1089600058D5C52015EC5815ECDD5F77DDDD568850
:108970000D82020D8D0DDD12D4588154518854DDC5
:10898000D5FF67DDDD7181D80ADD58D8020D880D6D
:108990008DDDDF77CDDDC5885C588DD0AD56050205
:1089A0000D8801D81501DDDD5F77DDDD568501D845
:1089B0002020D85103D8058D888D858DDDD5FF67A2
:1089C000C4DDDD01D880D2058D852D510365E58D8F
:1089D0005EDDFF764DDD545698D5A020D01058D0DE
:1089E0005058D80DDDD5FF67DDDD7058D881D10531
:1089F00020D05020D8020DD585C4DDFF77DDDD51B4
:108A000020560D8028D8580D10DDD0288D10580D17
:108A1000DDD5FF76C4DD54D5685450A8D5880D182F
:108A200052D518105EDDD5FF77DDDD561280D802F5
:108A30008D50D20D01580D01580DD5805C4DD5FFDC
:108A400077DD5E5685E580DD58028D50280D102DAE
:108A5000D5905EDD5F77C4DD5C45685C4509DD501F
:108A60001D58020D502028D8580DDDD5FF66DDDDDC
:108A700062010D0A8DD805C50515C5815CDD5F76DF
:108A8000C4DD5C4578DD5010D8A20D881DDD85EC75
:108A90004DDF774DDE45605E45205E4501DDD2014C
:108AA0008D01280D80DDDD5F774DDED85E50215EC3
:108AB0005101DD58568D02028D588054DDD5FF7668
:108AC000DDD5E56885E5101525E5858D50288D50A7
:108AD00038054DDD5F774DDDD58501D6288D02D86F
:108AE000D50152D45880545018054DDD5F77DD5EB6
:108AF000580D5E582605E58051DD2581D888D0289F
:108B00001DDDD5FF77C4DD54D568545828D5828D36
:108B1000102DD5185E510DEDDF77DDDD560D8D0280
:108B2000018D10518D52050D58285E580D5EDD5F88
:108B300077DDD5E5980D58280D51058DD562D5887E
:108B400020D888DDDD5F76DDDD560591D8A8D028F8
:108B50000D58DDE585EDDF54DDD56030D028D581B9
:108B600054DD5F74DDDD58D8D02628D10518DDDD51
:108B70005F74DDD5E57180D5052020D888DDDD5F07
:108B800074DDDD56880D0A050D580954DDD5FF4604
:108B90004DD458D501D620D020D50154DDFF46DD77
:108BA000E5705E5025E510D5020D80DDDF46DDD68F
:108BB0008D020D8D5125E5105EDDFF464DD458D553
:108BC0008D620D83D18DDDFF47DDD68D80D020D520
:108BD0002154501545854DDF47DDD80D18D503D6F6
:108BE00020D80D80DDDF74DDDD568210D8280D80A1
:108BF000510DDDD5FF76C4DD5C4568DD580D805034
:108C00001D80A0DDD015CCDDFF4ADDE570D580D814
:108C10000D02D585E502D580D80D10DDDF77DD5E4C
:108C20005685E5805E502DDD020501D888D1858D01
:108C3000DDD5FF7ACCDDCC585CC58DDD8D8058D874
:108C4000058D58520D8560D58295ED8D5E4DDF4ABC
:108C5000DDD68D80D80D52154501D520D80D80D890
:108C60000DDDFF49DDE5705E512D580D80D80D02F8
:108C7000D580D80DDDFF48DDD80D80D121D56D50D0
:108C80002D580D80DDDF4ADDE5605E5025E58D580D
:108C90001D150D80D5854520545854DDFF4ADDD182
:108CA00001D050D80D020D56D5020D80D80D585464
:108CB000DDFF75DDDD5601010D8850D50202054D41
:108CC0005805C4DD5F4ADDE5605E5105E512D50259
:108CD0000D050D80D80D050D80DDDF4ADDD68D80B8
:108CE000D80D8D5125E510DD20D80D80DDDF474DF5
:108CF000D4561545A5458D520D18D18DDDFF77DD74
:108D0000DD561018D0588D80DD50205E50205E5802
:108D1000DEDDFF77DDDD501568D015020D8D0DD835
:108D200080545028054D5805C4DD5F4ADDD68D803E
:108D3000D02D5020D18D501D8D580D80DDDF77DD79
:108D4000DD56880D05850D888DDD8D02028D898D9E
:108D5000DDD5FF76DDDD560158D8158D8580D80A22
:108D60000D888DDDD5FF764DDDD5688D010250D89B
:108D700088D51502054588054DDD5F77DDDD571582
:108D800080D888D0280DDD285C45805C45805C4D0E
:108D9000D5FF744DDDD5788D8A8D1858DDDD5F4A9D
:108DA000DDD021D80D8DD05E4525ED6D5121D80D3A
:108DB00080DDDF774DDDD56180D0288D858D58D859
:108DC000D0288D8518DDDD5F77DDDD56880D8025A7
:108DD0000D5880D8052D51885E518D5EDD5F66DDB2
:108DE000DD6801D0A8D510D5458854D585C4DDFFF0
:108DF0004ADDD68D80D50D510D581D020D520D80C6
:108E0000D80DDDFF76DDD5E5890D582026D8058DF6
:108E1000DD85CC585CCDDF4ADDE560D580D020D53E
:108E20000D5101D80D520D80D80DDDFF47DDD68DD7
:108E300080D521D121D020D5854DDF77DDDD5605C8
:108E400009D888D02050D58D8D02058D8058DDDD64
:108E50005F77DD5E5685E581DD5888D85A0D81053E
:108E60000D8580DDDD5F48DDE5105E58D5026D02C1
:108E70000D02D5105E5105EDDF774DDE458D5E4567
:108E8000895EDA85E568DD5888D888DDDD5F79DDC3
:108E9000DD5888D0288D8050DD0518D8180D02DDEA
:108EA000D5605E4585E4DDFF77C4DD5C45785C45D3
:108EB0001854D5020D581DD0A05E5885EDDDFF7603
:108EC000DDE585E501DDD5828D62850D8209DDDD7B
:108ED0005F77DDDD5898D0A80D5015854D562D458E
:108EE000885E458D5E4DDF6ACDD5C56015C5201500
:108EF000C58DC5285C580DD80D88D5880DD805CDF1
:108F0000D5FF49DDD68D80D020D02D585E530D5130
:108F100001D80DDDFF77DD5E568DD580510D020540
:108F200010D5280D45885E458D5E4DDF49DDE57025
:108F30005E510D5020D020D501D02D585E585EDDF9
:108F4000FF7ADDD5E5880D50288DDD85CC50DCC558
:108F500025EDD565E510510D5888D8580DDDD5FFA4
:108F600077DDDD5888D888DDD20D60158D8281D8F7
:108F7000D8DDDD5F77DDD5E56885E580105ED2510F
:108F80000D58D8D8280D858DDDD5FF77CCDD4DD691
:108F900005458020D505020D8D8D888D890DDDD587
:108FA000FF7ADDDD56880D888D5850D4DD854588E3
:108FB0000D5858D18DD58285E501285EDDD5FF7726
:108FC0004DDDD56801D888D01580D880D505A05E44
:108FD000580D5EDD5F79DDDD560580D888D8580DE7
:108FE00052050D580505E58050DD258054581015B3
:108FF0004DDD5F49DDD68D80D020D050D120D521E8
:1090000054501545854DDF7ADDD5E56885E50528A1
:109010005E5828D58580D888D5880D50DDD805E5DF
:10902000905EDD5F794DDE4585E458DE450205E45E
:109030005185ED80DD625020D8518DD5185C4DD51D
:10904000FF7ADDD5E58560D582020D8058D888D0BD
:109050005850D01018D8058D8058DDD85CCDDF660B
:10906000CDD5C5815C581DD20D560A5E51805EDD9E
:10907000DF47DDD701D18D020D02D5020D80DDDF86
:1090800047DDD621D021D02D580D121D5854DDFFBB
:109090007ADDE5605E585E58DDD10580D888D12D37
:1090A000DD5805E58205E5885EDDDF47DDE570D545
:1090B00081D020D520D120D120DDDF77DDDE5780A3
:1090C0005E5885ED010DD85A0D888D8580DDDD5FF8
:1090D0007ADDE5105E5105E58DDD80560D8028D5E1
:1090E0002580D8DDD888D888DDDD5F78DDDD56883D
:1090F0000D888D5859D80DD5888D82020DD5805C8C
:109100004DD5FF77DDDD5988D8A8D1850DDD620505
:10911000458805458DD4DDFF67DDDE56805E515202
:1091200005E5885E510DD502020D188DDDDF7ADD73
:10913000D5E5688D5888D8058D505805450580D5EA
:1091400005101D02050D58285E580D5EDD5F7AC4BE
:10915000DDDD5601D8581D858D5888D888D020501F
:10916000DD0585E580205E580D5EDD5F7ADD5E58A9
:109170000DD58268D52580D888D8050D58518D50D9
:10918000518D888D8058DDDD5F79DDDD560518D87D
:1091900098D8D8D8028D8A8D8058DD58DC4585EC6A
:1091A0004DDF77C4DDE4D561D45880D520510D0260
:1091B000050D50588D888DDDD5FF7ADDDD571058AF
:1091C000D8A8D588054DD0DCC505EC4D05EC458DFE
:1091D000C45805C45805C4DD5F77DD5E568D5E500A
:1091E0002805E5020505E58D0D5888D5810154DD7A
:1091F000D5FF79DDD5E56885E58805ED02DD4528F3
:109200008545880545851D4D5015EC4585EC4DDFA0
:109210007ADD5E5685E5805ED8DD580501D888DDAB
:10922000D01D8058D02820D880DDDD5F7AC4DD5C79
:1092300045805C45805CD585C56ADC5805ED580DD8
:1092400058580D8850D889DDDD5F774DDDD5603801
:10925000D0A80D858DD88054588154D5815C4DD5CA
:10926000FF77DD5E580DD58A60D0288D58501D8857
:109270008D8059DDDD5F7A4DDD54571805458050EE
:1092800054D580D5880D02028D8D8D8058D05058D0
:10929000D8058DDDD5FF76CCDDCC561DDD8D8580E6
:1092A000D0A28D889DDDD5FF774DDED60DD5020588
:1092B0008D8280DD885C58505C50905CDDDF77DD0E
:1092C000DD5888D0A81D8059D8DDD02685ED885E70
:1092D0004DDDFF794DDD545688D505020D880D58BA
:1092E000825ED0585E5101D5E5805E5805EDD5FF10
:1092F000774DDD5456801545881D520501D0280D47
:1093000058285E580D5EDD5F77C4DD54D568545033
:10931000A8D5828D1858D888D9058DDDD5FF76DD82
:10932000D5E56801D50A28D8509D80DD5805EDD5D2
:10933000FF7A4DDE4585E458DD4502620DD88D8803
:1093400050D888DD58D458805450101054DDD5FFC3
:1093500077DD5E5685E5805ED20DD58518D88AD535
:10936000810154DDD5FF7ADDDD560158D888D81546
:109370008DD580545880D52058D02050D5888D88E0
:109380008DDDD5FF7ADDD5E5688D5888D10D10D8F3
:10939000051D5888D02028D520DD4585E4585E4D30
:1093A000DF78DDDD5888D888D505020D880D581284
:1093B00036DD50215C4501DC4DDF77C4DD5C45685E
:1093C0005C4580DD528D882D505805E590215EDD8D
:1093D000D5FF4ADDE585E585E502D5020D101D12B4
:1093E0000D56D5020D18DDDF77C4DD5C45685C45A0
:1093F00080DDD20D82020D1880D9580DDDD5FF77A2
:109400004DDDD56158D12018D0288D02D8D8D8D8B4
:10941000DDDD5F77DDD5E56058D58028D8D02D809B
:1094200058D18121D858DDDD5F4ADDD18D020D563E
:10943000D5101D18D020D02D5020D80DDDFF77DDA0
:10944000D5E5881D58A26D8509DD58D4588054583B
:109450008054DDD5FF67DDE560DD512101D8020DC7
:1094600002DD585E585EDDFF4ADDD68D050D020D2A
:1094700028D020D10D530D5101D80DDDFF7ADDDD4F
:1094800057880D888DD580D8D01D888D8D0DD880BA
:109490005450A5054D5805C4DD5F784DDDD560916C
:1094A000D888D8050DD0580D0288D8A8D80DDDD59C
:1094B000FF7A4DDDED6095E58805E580DD58580DB6
:1094C000888D5880D028DD05820D888DDDD5FF7A06
:1094D000DDD5E510510D5888D888D10D20D026282B
:1094E000D505805458DD4585E4585E4DDF774DDD68
:1094F000D56058D8910D8D8D0A80D02028DD501070
:109500005C4DD5FF49DDE5605E5025E510D5121DA7
:10951000020D020D10D585EDDF774DDED60D5E50C4
:10952000A015E51885EDD50D502820D988DDDD5F23
:109530007ACCDDDD560D8D8D8D8D5858545858DD03
:10954000028D80A0D9850DD5185C4DD5FF774DDDF6
:10955000ED810D562820D02590D80DD5805E58DE9F
:10956000DDFF78DD5E580DD58280D02628DD8DD5D3
:10957000880D8801D90DDDD5FF7A4DDED10D5E58FD
:109580000205E5858DD052854505620D50D8D81D60
:10959000D5815E58DEDDFF7ADDDD562810D8A8DDE6
:1095A000580545820D4588054D5805C45185C45060
:1095B000515C45815C4DD5FF7ADD5E56015E5021E0
:1095C0005ED0DDD8518D8850D888D8D8D02820D505
:1095D0001020D4DDDF7AC4DDDD580D8820D0A02036
:1095E000D56050D458505ED1050D58018D1880D5E6
:1095F00010DD4DDF7ADDD5E560585E510185E585EA
:109600008D5888D8802D80521D50D8D02820D8154C
:109610008DDDD5FF764DDE4560DD45880DD89D0A90
:10962000251D888DDDD5FF77CCDDC4D615C4581D2A
:10963000D5021D8502D58820D888DDDD5F794DDE15
:109640004585E45105E450DE450DDD52580D60318D
:1096500020D05028D8158DDDD5FF77DDDD56880D5B
:109660008851DD5201DD581D8A8D880DDDD5FF49F9
:109670004DD4560D501D020D020D02D5020D18D10C
:1096800001DDDF77C4DDEDD85E518015E5020D5EAA
:1096900058560D5020A0D5018154DDD5FF4ADDE597
:1096A00070D5121D020D5205458D520D80D80D50FA
:1096B000154DDF7ADD5E568D5E58805EDD8D580576
:1096C0008D888D59503DD5020D8028D888DDDD5F0D
:1096D0007ADDDD58058D888D02058D5051854580D8
:1096E0005054D58054560AD45885E459D5E4DDFF4A
:1096F0007ADDDD580561D80501D80520D582854D74
:10970000850D58210D8D8D8058D8058DDDD5FF7ABA
:10971000DDD5E5688D58181D8581D880D5888D5890
:109720005854D0285C5A505C5885CDDDFF7ADDD581
:10973000E570585E518205E510520D585020D888CA
:10974000D50580D8050D5888D888DDDD5F7ADDDD48
:10975000570280D05028D020DD58280D051050D851
:1097600088D888D010510DDD85CCDDFF77C4DDDDD4
:10977000580D888D8820D50D2D509265E518D5EDB2
:10978000D5FF67DDDD10261D8020D1050D52D20DDD
:109790000180DD585C4DDF77C4DD5C45685C458049
:1097A000DDD8D90520D0A020D980DDDD5F774DDD63
:1097B00054560585450380DD5021D8D01D8820D81A
:1097C000281DDDD5FF7ADDDD58D01D8280D02D8D9E
:1097D000020DD5101560D50158D02580D8850D858E
:1097E00080DDDD5F7ADDDD580560D8820D5858D008
:1097F0002DDD8805ED2050DD0581D888D889DDDD97
:109800005F7AC4DDEC45605EDD85E5880D5888D85B
:109810005A0D8502DDD815C45815C4D015CCDDFF0E
:109820007AC4DDEDD8D5888D888D8050DD0D25E595
:109830001856D518520D15820D888DDDD5FF7ACDBD
:10984000DEC5605EC585EC58D54D5285450280D594
:109850008020D1858D1858D1858DDDD5FF77DDDD50
:1098600056880D02028D50580D020DD52885E51041
:10987000915EDDD5FF7ADDDD560580D8580D850275
:10988000D58058D101520D1858D505020D888D8804
:109890008DDDD5FF7ADD5E5805E5805E502DED7DCE
:1098A000E50305E580DDD8805450215054D5805C17
:1098B0004DD5FF7ADDDD5705101D888D02028D50D4
:1098C000DD54525ED05E58DDE58805E58585EDDD29
:1098D0005F7A4DDDD58501D81A0D8580D85020D806
:1098E000D6DDD020D888D8850D598054DDD5FF7AB3
:1098F000DDE561DDD01D01D888D888D05050D588ED
:109900008D82020D85250DD5805C4DD5FF7ADDE574
:1099100085E58DDD8568D525020D02850D888D5084
:10992000D8D1098D888DDDD5FF7ADDD5E5880D5834
:109930000A0D10D8D50512154505050D50580D62B4
:10994000D8D8580DD5815C4DD5FF7A4DDDD5801026
:10995000D888D8580D8050D580515E58050D5025B7
:1099600018D026202D5850154DDD5F7ADD5E5685C6
:10997000E5825E5020D5ED885E4D285ED88D592554
:109980008D8801D188DDDD5F77CCDD4DD605458A38
:109990000D505020D0158D58805E5101D5EDD5FF6A
:1099A0007ADDD5E5858D50A80D8058D1858D50D8AC
:1099B000D620DD5805E50515E5815EDD5F77DDD54F
:1099C000E5098D505801D8058D02D8D026020D58D2
:1099D0005854DDD5FF6A4DDD456805450A05458DBE
:1099E000D5025E5805E580DD1058D188D1058DDDA2
:1099F000DF7ADDDD58580D888D8DDD80260D052838
:109A00000D0303DD98DEDD85EC4585EC4DDF77C485
:109A1000DDDD509D605201D8581D8202D58285ED52
:109A20008D5E4DDF7AC4DD5C4568DD528D80A0D847
:109A300080D505805E580D5E5885E501015ED8151C
:109A4000E4DD5F79DDDD50188D8A8D02580D36DD3D
:109A5000D8095E58585ED8D5E4585E4DDF7ADD5E91
:109A6000580DD51858D10D8D8580D8850D5828D81A
:109A700082D5015236D8580DDDD5FF7ACCDD4DD8D0
:109A8000545818D50D20D62028D8820D8D0D588811
:109A9000D05180D81501DDDD5F7AC4DD54D5815405
:109AA0005880D5288D18DD515815E58050D58D8DFD
:109AB000026A0D588D4DDDFF4ADDD80D80D520D1CD
:109AC00001D020D10D5205E5625E5105EDDF77DD55
:109AD000DD56880D888DD58DD8A0D8280D91DDDD77
:109AE0005F76C4DD5C4581DD5210D6288D0A01D534
:109AF00010585EDDD5FF774DDDED60105E5020A57E
:109B0000E58530DD880545815054D5185C4DD5FF7D
:109B100077DDDD568021D8820DDD8D80501D8202DB
:109B20001DDD015CCDDF7A4DDDD5858D80520D8048
:109B300058D01D8D105620D9528D58805450205029
:109B400054D5805C4DD5FF79DDDD56880D80A0D5DC
:109B5000858D8102D505185E518125EDD85EC458EA
:109B60005EC4DDFF7ACCDDC4D605C4518DD518D8CE
:109B7000058D3828D81020DD20D5C5885C5885CDC6
:109B8000DDFF774DDE458DD4502610D50280D020E4
:109B9000DD5185E51215EDD5FF77C4DD54D5805430
:109BA0005880D510DD56A81D02028DD5095C4DD513
:109BB000FF76DDDD560218D15028D10202D585800E
:109BC000D10580DDDD5F7ADD5E5185E51015E502AA
:109BD00005E58DDE58285ED88DDDA6D8801D80DD98
:109BE000DD5F774DDED8D5E5630105E58A0D5805C3
:109BF0008D05218D80501DDDD5FF6ADDE560DE51CC
:109C0000015E580DD8501D02021D588D02DD58020C
:109C10000D880DDDDF77DDD5E560585E58585E585C
:109C2000585E502D2D502820D590954DDD5F77C47E
:109C3000DD54D51015456280D52518D10D2D582835
:109C40000D8580DDDD5F67DDE560DD5880D8032DA3
:109C5000D031D02050D8010DDDDF674DDD45618565
:109C600045018D5032D5850D5828D02010DDDDFFFF
:109C70007ACCDDC4D015C45805C45805C4D0DDD590
:109C800005E56850D582020D05281D03010DDDD5BF
:109C9000FF7AC4DDEDD85E5605205E50280DD880D1
:109CA000D8058D020501D8580D85101D8580DDDD94
:109CB0005F774DDDD57058D01A03D888DDD8D888A5
:109CC000D880DDDD5F76DDE560DDD10518DA88D886
:109CD000212D585105EDDD5F77DDDD581560D8A8E1
:109CE000D10158D50250D450385E458D5E4DDF7796
:109CF0004DDDD50158D1858D02058D8D8D80A1D585
:109D00000126D4DDDF77DDDD58580D0288D82DDD42
:109D10002659545028054580954DDD5F78C4DD5C9B
:109D20004580DD580D78530D8380D80A1DDD85CC24
:109D3000585CCDDF7ADD5E580DD58058D02058D5DF
:109D400088D4D20DE457230D458805451058545149
:109D500005854DDD5F794DDDD5858D8028D8D20D07
:109D60008820D05801D0910DDD5265CC585CCDDFF4
:109D70007ADDDD56880D02028D50D8D121DD5809DB
:109D80000D5288545058D4588054D5805C4DD5FF1E
:109D90007ADDDD580560D8258D58A0D188D585029B
:109DA0000D8580D50DDD8805E59185EDDD5F7AC4F3
:109DB000DD54D5805456280D50D0D59050D58028EC
:109DC000D51D03D85020D8580D8D8DDDD5FF77C413
:109DD000DD54D580545620505450281D50150D5830
:109DE0002315E580D5EDD5FF77DDDE58105E5050A8
:109DF00025E5836DDD028D8138D8058DDDD5FF7AAF
:109E00004DDDD56180D02850D8280D858D5028DEB5
:109E1000D88D452050154588054D5095C4DD5F7A95
:109E2000C4DDE4D560D458A0D505020D0288D80D54
:109E3000DD8D5E501805E505805E59815EDDD5FF3C
:109E400047DDD80D80D021D56D5020D18DDDFF4765
:109E5000DDD18D020D56D5120D80D80DDDFF46DD0A
:109E6000D68D020D58545215450154DDFF64DDDDD9
:109E70007018D02020DD585C4DDF46DDE585E58D8E
:109E80005026D38D81DDDF76DDDE56805E50585E54
:109E90005820DDD51205C45185C4DD5F47DDD68D60
:109EA00080D020D52154501545854DDF47DDD80D94
:109EB00018D503D620D80D80DDDF55DD5E580D5353
:109EC000026D058D018DDD5F4ADDD80D80D02D58E6
:109ED0000D80D101D50D5620D80DDDFF77DDDD5881
:109EE000D61D18020D8D8D020DD5805E5805EDD55D
:109EF000FF67DDDD698D8020DD5205C5805C58057A
:109F0000C5805CDD5F76CCDDCC58DDD20D68501DA0
:109F10008280DD5815C4DD5F76DDDD58568D858085
:109F2000D8058D82130D8D8DDDD5FF67CDDED56013
:109F30005E502025E588DD88D9050D880DDDDF74AC
:109F4000C4DDDD5601D8A8D881DDDD5F474DDD6178
:109F5000D18D020D02D580D80DDDFF4ADDD80D80F0
:109F6000D101D50D4525ED65E502D580D021DDDF98
:109F700077DDDD560580D8A8D888D8D8D8518DD5BA
:109F8000185C4DD5FF674DDDD680D0280D8DD518D6
:109F90005E50215E58DEDDFF77DDDD560580D02581
:109FA00080D1388DD8D5C585EC585ECDDF47DDE54D
:109FB00060D5020D121D12D580D80DDDFF77C4DDEE
:109FC000DD568D85250D105020D888D18050D85869
:109FD0000DDDD5FF494DD4560D520D80D051D18D98
:109FE00002D5020D81DDDF77DDDD56858D8280D8DB
:109FF000058D8502D580105E581D5EDD5F77DDDD45
:10A0000056880D02028DD580D10158D888D5880593
:10A010004DDD5F77C4DD5C45815C4580DDD0D56872
:10A02000520D05028D8318DDDD5F77DDDD5605807D
:10A03000D8801D858DDD80545828545821054DDD6C
:10A040005F774DDED60D5E58905E58D2D58058D8D9
:10A05000028D8058DDDD5F78DD5E5710D5E588051F
:10A06000E58825EDD8DDD020D888D80DDDD5FF7A5C
:10A070004DDD5458101545828DDD0D560580D028D4
:10A080008D8580D80DD5805E5805EDD5FF76DD5ED7
:10A090005685E50ADDD5810D888D80501DDDD5FF03
:10A0A00076DDD5E56885E50280D502D10D02058D06
:10A0B000101DDDD5FF7AC4DD54D581545818545095
:10A0C000D0D45850D4D88D5880D62058D05280D86B
:10A0D000058DDDD5FF76DDDD570D8D0A80D105803C
:10A0E000D8580D8DDDD5FF76DDDD58568D8280D0B8
:10A0F0002050DD051854581854DDD5FF7ADD5E5622
:10A1000085E5805ED8DD502581D8280D8D0DDD10C8
:10A11000DC45805C45805C4DD5FF47DDD68D020D6A
:10A12000520D020D81D101DDDF7AC4DDEC4585EDF4
:10A13000D205E58805E580505EDD505E4DD0D456F1
:10A14000820545810154D5805C4DD5FF74DDD5E590
:10A150006801D5A2020D95010DDDD5FF7A4DDE45D2
:10A160008D5E45885ED88D58D8D80A0D5856D4D5FE
:10A170001015C45805C45805C4DD5F49DDE585E503
:10A180008D5026D120D020D58545015450154DDF66
:10A190004ADDD68D80D50D5101D81D020D520D021C
:10A1A0000D80DDDF7ADDDD56880D888DD8DD020279
:10A1B00005E58805E58DDD50580D888D10180DDDFD
:10A1C000D5FF7A4DDDD56181D888D858D58D8D8859
:10A1D0008D8580D8820D82DD5805EDD5FF4ADDD111
:10A1E0008D020D56D5020D80D10D5121D020D8DD24
:10A1F000DF77DD5E5805E5805ED20DD458571545F2
:10A200000202154585854DDD5F76DDD5E5958D5AD4
:10A21000280D6858DD50205C451015C4DD5F4ADD0F
:10A22000D80D80D520D80D121D56D5120D80D80D11
:10A23000DDFF4A4DD456154520D502D80D050D1029
:10A240001D02D5020D81DDDF77CCDD4DD6154588A9
:10A250000D50D01D02058D8280D858DDDD5F7ADD7E
:10A26000DD56880D05280D02058D888DD5805C454D
:10A270008054D58D45985E458D5E4DDF77DDD5E503
:10A280007018D50A020D5050105458DD45885E45AF
:10A29000885E4DDDFF0002080007E000081401059C
:10A2A000001407E014081415050000FF0001FE006B
:10A2B00007320107C802079603073204050000FFB2
:10A2C0000002080007FF000832010828030500000B
:10A2D000FF00020700085F02040A020408020406E5
:10A2E00002040402040200084202030502040202FE
:10A2F00003050203050204020203050000F804033B
:10A300000504040504030504040504030504040509
:10A3100004030501050000FF0002010007FF00081B
:10A320006401050000FF00000095A200000000018C
:10A330000000ACA200000000000000C0A20000006D
:10A3400000000000D1A20000000000000018A300DF
:10A350000000000011241FBECFEFD0E1DEBFCDBF53
:10A360002AE0A0E0B1E001C01D92A936B207E1F7F2
:10A3700014BE0FB6F894A895809160008861809310
:10A380006000109260000FBEF89480E990E0FC013C
:10A3900025913491F901FF273083029620E0823C19
:10A3A0009207A9F70E94C754811102C00E94A554C8
:10A3B00081E08093EE018093EF018093ED01109294
:10A3C000DA011092E0011092E6011092EC01109275
:10A3D000F2011092C4011092C60192E19093C5015E
:10A3E00090EC9093CC0193E29093CB011092D0012A
:10A3F0001092CF011092D4011092D3018093D90111
:10A400000E94016078940E9400600E943D660C9456
:10A4100091660C940000E0E0EA95F1F7E1ECEA9532
:10A42000F1F7C0E0D1E0A090CC0166277CE049D1F3
:10A4300038E33A95F1F700000E9445523FE23A9521
:10A44000F1F700C0AA9489F0C8956395603129F0AE
:10A45000C895C895C8950000EACF6627002430E16A
:10A46000C30FD01DC8950000E2CF35E03A95F1F753
:10A4700000C027D1E091C60142E0E160E427E0930B
:10A48000C601E2E0E09336000895DE0110EC809111
:10A49000C0019091C101679F800D911D4D91419F19
:10A4A000080E191EF00120E1059108B94D910591A2
:10A4B00008B9419F059108B9AC01400D059108B953
:10A4C000511D0000059108B9C895059108B9C895B6
:10A4D000059108B9C895059108B9C895059108B9BD
:10A4E000C895059108B9C895059108B90591FA0173
:10A4F0002A9508B9C9F600C00000002708B90895D8
:10A500000F921F92EF93FF93FFB7E0918400FF93A8
:10A51000E2FD04C0E1FD02C0000000C0E0FF00C099
:10A52000E091C501EA95E093C501F091C401F0FD09
:10A5300051C0EC3098F0F3E0F0938900FDE8F0931F
:10A540008800E0FB289826F4E1E00E947253B2C034
:10A55000E5E1EA95F1F70000289AACC0E63008F191
:10A5600000C000C02898E0FBE4E016F40E9472539B
:10A57000E4E0E0933600E6E0E0936F009BC0EF93E9
:10A58000E0918400E2FD04C0E1FD02C0000000C0D3
:10A59000E0FF00C0E2E00000289AE0936F00EF9136
:10A5A000189500C0E0FB289826F4E1E00E94725361
:10A5B00005C0E5E1EA95F1F70000289AE091C501B0
:10A5C000E03009F077C0EDEFE093C501E1E0E09302
:10A5D000C40170C0E7E0E0938900EBE1E0938800FC
:10A5E00000C02898E2E000C00E947253FDEF009086
:10A5F000CB01F019E091C501EF17D8F4FDEF009001
:10A60000CB01F0190090CC01F019EF1790F0EDE1BB
:10A61000FF2700800F92EA95E1F70DE00A95F1F728
:10A6200000C00E940B52E1E0FF270F900192EE3133
:10A63000E0F3E091C501E03009F03CC02F933F9377
:10A640004F935F936F937F938F939F93AF93BF933A
:10A6500078941124EE27E093C401E2E1E093C50170
:10A660008091D5019091D60101968093D501909368
:10A67000D601E091C701F091C801E115F10509F09B
:10A6800009950E9495540E9402600E946C53112407
:10A69000E091C901F091CA01E115F10509F00995B0
:10A6A000BF91AF919F918F917F916F915F914F91EA
:10A6B0003F912F91EF91EFBFFF91EF911F900F907E
:10A6C00018952898E2E000C00E947253E091C501FD
:10A6D000EA95E093C5010895E091D901E0FD0E945B
:10A6E0007B5608952F931F930F932E2F1091DD010A
:10A6F000E091DE01F091DF010091DB01100F00918C
:10A70000DC01E01F0491E093DE011093DD01109164
:10A71000DA01010300081091E301E091E401F091F6
:10A72000E5010091E101100F0091E201E01F0491A9
:10A73000E093E4011093E301F0011091E0010103C3
:10A7400000081F0E1091E90120FD289A0E1EE091CD
:10A75000EA01F091EB010091E701100F0091E8018F
:10A76000E01F0491E093EA011093E901F0011091D8
:10A77000E601010300081F0E0E1E0091EE0110916C
:10A78000EF01F091EC01F695889400FDF195EE0B48
:10A790001F0E0E1EE091F001E25020F0E491E491D2
:10A7A000E4910AC0E02F16950795E027E0FB16F923
:10A7B000E091ED01E0FF06F90093EE011093EF0147
:10A7C000E093F00110E0E091F501F091F30121FD3B
:10A7D000289AEF0FE093F501E091F601F091F7016F
:10A7E0000091F401E01FF11F0091FA011091FB01AB
:10A7F000E017F10718F4E49100C006C00091F801D9
:10A800001091F901E01BF10BE093F601F093F701D1
:10A810000491F0011091F201010300081F0E0E1EB9
:10A82000F0010F911F91F058EF4F1AF4F0E0000083
:10A8300003C0E03009F0FFEFF093B3002F910895CB
:10A840008093C0019093C10108958091C6018170E9
:10A8500008952091C6012E7F2093C6010895882374
:10A8600029F48091CD019091CE0108958091D1017C
:10A870009091D2010895E0E6F0E0808183FD089593
:10A8800088E198E0F894808390837894FFCFF999D9
:10A89000FECF92BD81BD60BDF894FA9AF99A789482
:10A8A0000895F999FECF92BD81BDF894F89A80B5CC
:10A8B000789408956093CC018093CB010895129A07
:10A8C000C895C895C895C895129840E180E090E079
:10A8D00020E030E03695279596958795C895C895E0
:10A8E000C895C8951398009B3068019B9068139A8F
:10A8F000C895C895C895C895415061F73093CE0169
:10A900002093CD019093D2018093D1018091CD010C
:10A910009091CE010F9731F08091D1019091D201A9
:10A920000F9711F40C943B5408951092FC01009978
:10A9300003C081E08093FC01019905C08091FC0176
:10A9400082608093FC010C945F54CF93DF93C0E04E
:10A95000D0E0FE01E059FF4F6491CE010E944754C0
:10A960002196C032D105A9F7C0E2D0E06FEFCE0149
:10A970000E9447546FEFCE0101960E944754A09663
:10A98000C11588E0D80791F7DF91CF910895CF9353
:10A9900080E090E00E945154C82F81E090E00E9436
:10A9A0005154282F30E0322F22272C0F311D81E007
:10A9B0002A35354509F080E0CF910895EF92FF9256
:10A9C0000F931F93CF93DF9300D01F92CDB7DEB7C5
:10A9D0008C011A8219821B82AE014D5F5F4FBE014E
:10A9E0006F5F7F4FFC01808191810E945B558823BE
:10A9F00011F0833019F589819A81892B49F48B8173
:10AA00008823D9F0F0E28F9FC00111249A838983B3
:10AA1000780120E2E20EF11CF80161918F01898139
:10AA20009A819C012F5F3F4F3A8329830E944754AC
:10AA30000E151F0589F780E001C082E00F900F908E
:10AA40000F90DF91CF911F910F91FF90EF9008959C
:10AA5000CF92DF92FF920F931F93CF93DF9300D09B
:10AA6000CDB7DEB78B0140E050E0BE016F5F7F4F96
:10AA70000E945B55F82E811113C0680180E2C80E58
:10AA8000D11C89819A819C012F5F3F4F3A83298392
:10AA90000E945154F80181938F01EC15FD0589F74F
:10AAA0008F2D0F900F90DF91CF911F910F91FF90FD
:10AAB000DF90CF9008958F929F92AF92BF92CF92E6
:10AAC000DF92EF92FF920F931F93CF93DF93FB01DF
:10AAD000118210828F3FFFEF9F0789F16A018B017E
:10AAE0007C01A12CB12CC0E0D3E0912CC5010E94C7
:10AAF0005154882EC50101960E945154282F30E0F0
:10AB0000322F2227280D311D2E153F0529F4F8017B
:10AB1000B182A082D0E00BC02F3F3F4F41F4911093
:10AB200006C0C114D10411F0F601C0839C2ECF5F82
:10AB3000F0E2AF0EB11CC034C9F68D2F01C081E028
:10AB4000DF91CF911F910F91FF90EF90DF90CF9009
:10AB5000BF90AF909F908F900895FC0167870895F4
:10AB6000EAEDF1E081E091E0958B848B638B0895B1
:10AB7000FC0182810C94ED59FC019181690F618384
:10AB800082810C94D659FC019181961B692F918387
:10AB900082810C94D659FC0190819F759083089511
:10ABA000FC019081906490830895FC01668708956C
:10ABB0001F93CF93DF93EC01162F8A810E94D65901
:10ABC00019838881877F8883DF91CF911F910895B2
:10ABD000FC0162870895FC0163870895CF93DF939A
:10ABE000EC01462F298130E0F901EE0FFF1FEC5EEA
:10ABF000FB4465917491F901E40FF11D47FDFA954D
:10AC0000EE0FFF1FEC5EFB4485919491861B970B22
:10AC1000688570E00E947D666115710511F461E040
:10AC200070E0EA8186E0E89FF0011124E652FE4FD1
:10AC300081819281860F971F928381837E836D83AA
:10AC40008881886088838981480F4F83DF91CF9105
:10AC50000895FC0160870895FC0164830895DC0178
:10AC600014968C911497882319F155962D913C9147
:10AC70005697662379F0062E000C770B6F5F7F4F97
:10AC8000AB01440F551F640F751F261B370B09C0FE
:10AC9000EF3F39F023503109F9013297E491ED305B
:10ACA000B9F756963C932E935597815014968C93F2
:10ACB000089590937502809374028FE680937702D3
:10ACC0001092D801EFE0F2E080E090E13FEF28E160
:10ACD000DF011E978C9312979C931D961C921197DF
:10ACE0003C93108211972C9313979C938F5F7796C8
:10ACF000853071F708956F927F928F929F92AF92F5
:10AD0000BF92CF92DF92EF92FF920F931F93CF9358
:10AD1000DF93CFEFD1E00AED11E0D8019E0140E0D2
:10AD200050E0CA0181509E4F6C01FC018785882349
:10AD300091F06685082E000C990B860F911D8F3FB0
:10AD4000910519F014F08FEF90E097FF02C080E0BA
:10AD500090E0F6018687F901F080F3FE2AC0658154
:10AD6000768111968D919C911297860F971F12965E
:10AD70009C938E931197F601E780EE2DF0E0EE0F95
:10AD8000FF1FEC5EFB44C590D4901616170624F402
:10AD90008C159D0530F40DC0672B59F0C816D906E7
:10ADA00040F01296DC92CE9211978F2D877FF90199
:10ADB0008083495E5F4F295E3F4F169643375105AA
:10ADC00009F0AFCF8091D801882309F4CCC057E1B6
:10ADD000F52E809172029091730220917802309149
:10ADE00079028217930709F0B9C020917B02309154
:10ADF0007C02B9016F5F7F4F70937C0260937B028E
:10AE0000F90144914F3F79F5A9014E5F5F4F50938F
:10AE10007C0240937B02FB0164916F3219F4109223
:10AE2000D8019CC0663009F08CC0FA014491C90178
:10AE3000049690937C0280937B02F9013396E4910F
:10AE4000E33529F490937E0280937D027AC0E53445
:10AE500009F077C080917D0290917E0290937C02F0
:10AE600080937B026EC047FD4093760290917602FC
:10AE7000892F8F7047FF08C02E5F3F4F30937C02B1
:10AE800020937B02FB014491907F903BE1F0903C4A
:10AE900009F451C0903909F054C0E0917B02F0915F
:10AEA0007C029F012F5F3F4F30937C0220937B02F7
:10AEB0002491220FF89EF0011124E150FE4F608989
:10AEC0000E9496593EC0E0917B02F0917C029F0166
:10AED0002F5F3F4F30937C0220937B02E4914730F9
:10AEE00049F4F89ED0011124A150BE4FEE0F1C96DC
:10AEF000EC9327C04B3049F4F89ED0011124A150A7
:10AF0000BE4FEE0F1396EC931CC04C3549F4F89EDF
:10AF1000D0011124A150BE4FEE0F1A96EC9311C030
:10AF2000443679F4F89ED0011124A150BE4FEE0FA3
:10AF30001B96EC9306C0F89EF0011124E150FE4FE1
:10AF4000408B8BE792E00E949A589093790280930D
:10AF5000780210927302109272023BCF0196909386
:10AF600073028093720298E0A92E92E0B92E22E13A
:10AF7000C22E22E0D22E33E1E32E32E0F32E6624FD
:10AF80006A94712C888185FF42C02D893E89232BCC
:10AF900009F43DC086FD3BC04701F2E08F1A9108DD
:10AFA000D6019C91F401808198132EC0ED89FE8911
:10AFB000BF016F5F7F4F7E8B6D8B84918F3F31F42C
:10AFC00088818F7788831E8A1D8A1EC09F012E5F0D
:10AFD0003F4F3E8B2D8BFB016491E82FF0E0EE0F8D
:10AFE000FF1FEE53FF4F25913491CE01F9010995D2
:10AFF000ED89FE89CF0101969E8B8D8BE491D40162
:10B00000EC93F6011082CCCF9F5FD6019C93988180
:10B0100095FF6CC0F70180818F3F11F08F5F8083B7
:10B0200097FD04C0F7013897908101C09FEFF701A9
:10B0300037978081882309F44EC03196508155237B
:10B0400009F449C0992309F446C04091770244238A
:10B0500009F441C0899FC00111249395892F992734
:10B06000589F9001599F300D1124C9019395892F44
:10B0700099273B975081589F9001599F300D11247B
:10B080003395232F3327429FC001439F900D1124F6
:10B090009395892F9927379620812223F1F0D501A6
:10B0A000EC91F0E0E050FA44E491E0582E9FF0017A
:10B0B0001124F395EF2FFF27A3014E1B5F0B489F31
:10B0C0009001499F300D589F300D1124C90193956F
:10B0D000892F992702C080E090E0F5013081F701C7
:10B0E00039972081230FD5012C9302C080E090E096
:10B0F000F801808367960A5F1F4FF7E1AF0EB11C1E
:10B1000087E1C80ED11C97E1E90EF11CA2E0C2371D
:10B11000DA0709F037CFDF91CF911F910F91FF90A0
:10B12000EF90DF90CF90BF90AF909F908F907F90E7
:10B130006F900895DC01ED91FC9111979F012F5FB5
:10B140003F4F11963C932E93E491E7FD03C08E2F61
:10B1500090E00895EF778E2F90E09695982F8827AE
:10B16000979587952F5F3F4FF9013197E4914E2FC7
:10B170004F77840F911DE7FDF0CF2D933C930895F9
:10B18000EF92FF920F931F93CF93DF931F92CDB750
:10B19000DEB77C01162FFC018081082F001F0027DD
:10B1A000001F17869FEF96874587148A877B8083C9
:10B1B000128611862183148293838281833069F4FD
:10B1C000011101C0122F81E091E09093EF01809373
:10B1D000EE0181E08093ED0139C0843069F5109271
:10B1E000F5018091740290917502F9E06F9F800DD6
:10B1F000911D1124FC013196A591B491B093F701F2
:10B20000A093F601AC01495F5F4FFA01659174911B
:10B210000596FC0185919491681B790B7093F90157
:10B220006093F801FA0185919491A80FB91FB0932A
:10B23000FB01A093FA0105C060E029830E94ED594B
:10B240002981622FF70182810E94D659F7010023DC
:10B2500011F0118B01C0108BE0917402F091750216
:10B2600039E0139FE00DF11D1124339685919491DF
:10B27000F701009719F4168A158A08C0138AFC0191
:10B280002491F701228B0196968B858B0F90DF918D
:10B29000CF911F910F91FF90EF900895CF93DF937F
:10B2A000E0917402F091750299E0899FE00DF11D23
:10B2B0001124E491E130E9F0E230E9F02091160246
:10B2C00027FF1DC020912702281302C0411117C07B
:10B2D00020912D0227FF11C020913E02281302C0A9
:10B2E00041110BC020912A0290914102921728F43B
:10B2F00006C0C3E005C0C4E003C0C2E001C0C1E0B5
:10B3000097E1C99FE0011124C150DE4F90E8988376
:10B310001E8A1D8A20E5462F682FCE010E94C05844
:10B32000888180628883DF91CF910895CF93DF93E6
:10B33000A82FB0E097E1899FF0011124E150FE4F62
:10B34000808185FF02C087FD2EC0211118C097E1C2
:10B350009A9FF0019B9FF00D1124E150FE4F9785BD
:10B36000911102C086FF158697E19A9FF0019B9F7D
:10B37000F00D1124E150FE4F8F7B808314C0822F8B
:10B38000242F97E19A9FE0019B9FD00D1124C1507B
:10B39000DE4F18821E8A1D8A482FCE010E94C05897
:10B3A000888180628883DF91CF91089599277727DC
:10B3B000833009F40895E4E1F4EB660F771FE60F9C
:10B3C000F71FA591B491EAEDF1E026E0289FE00D8A
:10B3D000F11DA183B2831124089599277727EAEDFF
:10B3E000F1E026E0289FE00DF11D6E3F31F4609101
:10B3F000ED016E7F6093ED010BC06F3F31F4609102
:10B40000ED016E6F6093ED0103C076EB760F7583EF
:10B410001124089522002400260028002B002D006E
:10B4200030003300360039003D0040004400480041
:10B430004C00510056005B00600066006C00730019
:10B4400079008100880090009900A200AC00B6004D
:10B45000C100CC00D800E500F3000101100121017A
:10B460003201440157016C0181019801B001CA0108
:10B47000E50102022102410264028802AE02D70203
:10B480000303300361039403CB03050442048304E4
:10B49000C70410055D05AF0505066106C20629074C
:10B4A00096070908830805098E09200ABA0A5D0B68
:10B4B0000A0CC10C840D510E2B0F121007110A1229
:10B4C0001D1340147415BA1614188319071BA31CF6
:10B4D000571E24200E22142439267F28E82A752D91
:10B4E000293006330F364539AD3C49401B442848C6
:10B4F000734CFE50CF55EA5A51600C661D6C8B722E
:10B500005A79928037885090E598FDA19FABD3B5CA
:10B51000A3C00000000000000000000000000000C8
:10B52000000000000000000000000000000000001B
:10B53000000000000000000000000000000000000B
:10B5400000000000000000000000000000000000FB
:10B5500000000000000000000000000000000000EB
:10B5600000000000000000000000000000000000DB
:10B5700000000000000000000000000000000000CB
:10B5800000000000000000000000000000000000BB
:10B5900000000000000000000000000000000000AB
:10B5A000000000000000000000000000000000009B
:10B5B000000000000000000000000000000000008B
:10B5C000000000000000000000000000000000007B
:10B5D000000000000000000000000000000000006B
:10B5E000000000000000000000000000000000005B
:10B5F000000000000000000000000000000000004B
:10B60000000306090C101316191C1F2225282B2EC7
:10B61000313336393C3F414447494C4E51535558DC
:10B620005A5C5E60626466686A6B6D6F7071737499
:10B63000757678797A7A7B7C7D7D7E7E7E7F7F7F52
:10B640007F7F7F7F7E7E7E7D7D7C7B7A7A79787638
:10B6500075747371706F6D6B6A68666462605E5C4E
:10B660005A585553514E4C494744413F3C39363363
:10B67000312E2B2825221F1C191613100C09060326
:10B6800000FDFAF7F4F0EDEAE7E4E1DEDBD8D5D22D
:10B69000CFCDCAC7C4C1BFBCB9B7B4B2AFADABA8F8
:10B6A000A6A4A2A09E9C9A9896959391908F8D8C1B
:10B6B0008B8A888786868584838382828281818142
:10B6C0008181818182828283838485868687888A3C
:10B6D0008B8C8D8F9091939596989A9C9EA0A2A406
:10B6E000A6A8ABADAFB2B4B7B9BCBFC1C4C7CACDD1
:10B6F000CFD2D5D8DBDEE1E4E7EAEDF0F4F7FAFDEE
:10B70000808182838485868788898A8B8C8D8E8FC1
:10B71000909192939495969798999A9B9C9D9E9FB1
:10B72000A0A1A2A3A4A5A6A7A8A9AAABACADAEAFA1
:10B73000B0B1B2B3B4B5B6B7B8B9BABBBCBDBEBF91
:10B74000C0C1C2C3C4C5C6C7C8C9CACBCCCDCECF81
:10B75000D0D1D2D3D4D5D6D7D8D9DADBDCDDDEDF71
:10B76000E0E1E2E3E4E5E6E7E8E9EAEBECEDEEEF61
:10B77000F0F1F2F3F4F5F6F7F8F9FAFBFCFDFEFF51
:10B78000000102030405060708090A0B0C0D0E0F41
:10B79000101112131415161718191A1B1C1D1E1F31
:10B7A000202122232425262728292A2B2C2D2E2F21
:10B7B000303132333435363738393A3B3C3D3E3F11
:10B7C000404142434445464748494A4B4C4D4E4F01
:10B7D000505152535455565758595A5B5C5D5E5FF1
:10B7E000606162636465666768696A6B6C6D6E6FE1
:10B7F000707172737475767778797A7B7C7D7E7FD1
:10B8000000020406080A0C0E10121416181A1C1E48
:10B8100020222426282A2C2E30323436383A3C3E38
:10B8200040424446484A4C4E50525456585A5C5E28
:10B8300060626466686A6C6E70727476787A7C7E18
:10B840007F7D7B79777573716F6D6B6967656361F8
:10B850005F5D5B59575553514F4D4B4947454341E8
:10B860003F3D3B39373533312F2D2B2927252321D8
:10B870001F1D1B19171513110F0D0B0907050301C8
:10B88000FFFDFBF9F7F5F3F1EFEDEBE9E7E5E3E1B8
:10B89000DFDDDBD9D7D5D3D1CFCDCBC9C7C5C3C1A8
:10B8A000BFBDBBB9B7B5B3B1AFADABA9A7A5A3A198
:10B8B0009F9D9B99979593918F8D8B898785838188
:10B8C00080828486888A8C8E90929496989A9C9E88
:10B8D000A0A2A4A6A8AAACAEB0B2B4B6B8BABCBE78
:10B8E000C0C2C4C6C8CACCCED0D2D4D6D8DADCDE68
:10B8F000E0E2E4E6E8EAECEEF0F2F4F6F8FAFCFE58
:10B900007F7F7F7F7F7F7F7F7F7F7F7F7F7F7F7F47
:10B910007F7F7F7F7F7F7F7F7F7F7F7F7F7F7F7F37
:10B920007F7F7F7F7F7F7F7F7F7F7F7F7F7F7F7F27
:10B930007F7F7F7F7F7F7F7F7F7F7F7F7F7F7F7F17
:10BC00000309131E28313A40464C5054585B5E617C
:10BC1000636567696B6C6E6F70717273747576773C
:10BC2000777879797A7A7B7B7C7C7C7D7D7D7E7E62
:10BC30007E7E7F7F7F7F7F7F7F7F7F7F7F7F7F7F16
:10BC40007F7F7F7F7F7F7F7F7F7F7F7F7F7E7E7E07
:10BC50007E7D7D7D7C7C7C7B7B7A7A797978777739
:10BC6000767574737271706F6E6C6B696765636102
:10BC70005E5B5854504C46403A31281E130903006D
:10BC8000C6CCD5DBDFE3E5E7E9EAEBECEDEEEFEF81
:10BC9000F0F0F0F1F1F1F1F2F2F2F2F2F2F2F2F38D
:10BCA000F3F3F3F3F3F3F3F3F3F3F3F3F3F3F3F364
:10BCB000F3F3F3F3F3F3F3F3F3F3F3F3F3F3F3F354
:10BCC000F3F3F3F3F3F3F3F3F3F3F3F3F3F3F3F344
:10BCD000F3F3F3F3F3F3F3F3F3F3F3F3F3F3F3F334
:10BCE000F2F2F2F2F2F2F2F2F1F1F1F1F0F0F0EF41
:10BCF000EFEEEDECEBEAE9E7E5E3DFDBD5CCC60000
:10BD000000283D42302D2C2B2C2D2E2F3032333558
:10BD100037393B3D3F414345484A4C4E50535557B8
:10BD2000595B5D5F61636567696B6C6E707173749D
:10BD3000757778797A7B7C7D7D7E7E7F7F7F7F7F44
:10BD40007F7F7F7F7F7F7E7E7D7D7C7B7A7978772A
:10BD500075747371706E6C6B69676563615F5D5B51
:10BD600059575553504E4C4A484543413F3D3B3946
:10BD700037353332302F2E2D2C2B2C2D30423D28B1
:10BD800000E9E5FED4D7D7D7D6D4D2D0CECCCAC816
:10BD9000C6C3C1BFBDBAB8B6B4B1AFADABA9A7A554
:10BDA000A3A19F9E9C9A999795949391908F8D8C27
:10BDB0008B8A898888878685858484848383838326
:10BDC0008383838383848484858586878888898A1E
:10BDD0008B8C8D8F909193949597999A9C9E9FA10F
:10BDE000A3A5A7A9ABADAFB1B4B6B8BABDBFC1C327
:10BDF000C6C8CACCCED0D2D4D6D7D7D7D4FEE5E9E0
:10BE0000F9F8F9F5EBE1DDDEE0E2E4E5E6E5E4E2B0
:10BE1000DED9D2CAC1B7ACA299918A8683818080CB
:10BE20008182838586888A8C8D8F90929395969750
:10BE300098999A9B9B9C9D9D9D9E9E9E9F9F9F9F38
:10BE40009F9F9F9E9E9E9D9D9D9C9B9B9A99989730
:10BE500096959392908F8D8C8A8886858382818037
:10BE6000808183868A9199A2ACB7C1CAD2D9DEE219
:10BE7000E4E5E6E5E4E2E0DEDDE1EBF5F9F8F90022
:10BE80000708070B151F2322201E1C1B1A1B1C1E34
:10BE900022272E363F49545E676F767A7E7F7F7FFA
:10BEA0007F7E7D7B7A7876747371706E6D6B6A6954
:10BEB000686766656564646363626262616161614B
:10BEC0006161616262626363636465656667686934
:10BED0006A6B6D6E7071737476787A7B7D7E7F7F0E
:10BEE0007F7F7E7A766F675E54493F362E27221E0B
:10BEF0001C1B1A1B1C1E2022231F150B07080700E2
:10BF00001F313D444E5354565A5F64696E747679BE
:10BF10007C7F7F7F7F7F7F7F7F7F7F7F7F7F7F7F34
:10BF20007F7F7F7F7F7F7F7F7F7F7F7F7F7F7F7F21
:10BF30007F7F7F7F7F7F7F7F7F7F7F7F7F7F7F7F11
:10BF40007F7F7F7F7F7F7F7F7F7F7F7F7F7F7F7F01
:10BF50007F7F7F7F7F7F7F7F7F7F7F7F7F7F7F7FF1
:10BF60007F7F7F7F7F7F7F7F7F7F7F7F7F7F7F7FE1
:10BF70007F7F7F7F7F7F7F7F7F7F7F7C7871684C33
:10BF80002C1C120C0A0B0A05FDF3E9DFD4CAC0B75A
:10BF9000AEA69E97918B86858280808080808080EF
:10BFA0008080808080808080808080808080808091
:10BFB0008080808080808080808080808080808081
:10BFC0008080808080808080808080808080808071
:10BFD0008080808080808080808080808080808061
:10BFE0008080808080808080808080808080808051
:10BFF000808080808087919DACC4CBD4DDF2FAFA3A
:10C000000895089508950F931F93CF93DF938C01A4
:10C01000C0E0D0E0C017D10744F40E942554882323
:10C02000E1F30E9429542196F5CFDF91CF911F9122
:10C030000F9108958093630A6093680A4093820287
:10C04000209391028093920260938102089520913F
:10C05000920290918102E22FF0E0E050FF4F30E138
:10C06000939FE00DF11D112480832F5F2093920296
:10C0700080918202821778F48091630A8093920201
:10C080009F5F9093810280919102891720F48091A3
:10C09000680A809381020895EF92FF920F931F9395
:10C0A000CF93DF938C01C62FDAE08AE0E82EF12CE3
:10C0B000CC23C9F091E061E070E09C1741F09B0156
:10C0C000D29FB001D39F700D11249F5FF6CFC8019E
:10C0D0000E946966CB01B7010E946966855F0E9474
:10C0E0002760C150E5CFDF91CF911F910F91FF9055
:10C0F000EF9008958091630A80939202809181026B
:10C100008F5F8093810290919102981720F4809123
:10C11000680A809381020895DF92EF92FF920F9355
:10C120001F93CF93DF93CDB7DEB7A0970FB6F894E8
:10C13000DEBF0FBECDBF9C0143E0969587954A9523
:10C14000E1F76EE170E00E9469667C01822F8770E2
:10C15000D82EC90160EF70E00E9469668B010E570E
:10C160001F4FBE016F5F7F4FC8010E94285581118C
:10C1700021C0E3E0F0E0EC0FFD1FEE0DFF1D21E01C
:10C1800030E001C0220FDA94EAF78081282B208367
:10C19000CE0101960E94DE54A0960FB6F894DEBF41
:10C1A0000FBECDBFDF91CF911F910F91FF90EF9008
:10C1B000DF9008951A830983FE013396CE0181969C
:10C1C0001192E817F907E1F7D4CF0F931F93CF939C
:10C1D000DF93CDB7DEB7A0970FB6F894DEBF0FBEE2
:10C1E000CDBF8C0160EF70E00E946966CB01BE019B
:10C1F0006F5F7F4F8E579F4F0E942855811118C047
:10C20000C80123E0969587952A95E1F76EE170E0E5
:10C210000E946966FE01E80FF91F238130E0077074
:10C22000C90102C0959587950A95E2F7817001C012
:10C2300080E0A0960FB6F894DEBF0FBECDBFDF91B1
:10C24000CF911F910F9108950F931F93CF93DF9379
:10C25000CDB7DEB7A0970FB6F894DEBF0FBECDBF47
:10C26000182F092FBE016F5F7F4F86E890E00E9474
:10C270002855811111C008A31F8FCE0101960E947D
:10C28000DE54A0960FB6F894DEBF0FBECDBFDF918F
:10C29000CF911F910F91089586E890E09A8389834A
:10C2A000FE013396CE0181961192E817F907E1F766
:10C2B000E2CFCF93DF93CDB7DEB7A0970FB6F89458
:10C2C000DEBF0FBECDBFBE016F5F7F4F86E890E03F
:10C2D0000E94285581110CC028A130E0322F22275E
:10C2E0008F8D282B273E83E0380710F4C90102C048
:10C2F00080E090E0A0960FB6F894DEBF0FBECDBFF1
:10C30000DF91CF9108952BE04FE06BE080E00E9439
:10C310001A6080918002811102C085E101C086E12E
:10C320000E94276088E00E94276080918702909198
:10C33000880263E001960E944C608AE00E942760B8
:10C3400064E08091660A9091670A0E944C6089E0DF
:10C350000E94276065E080918502909186020C948E
:10C360004C60CF92DF92FF920F931F93CF93DF9396
:10C370001F92CDB7DEB710928602109285021092FE
:10C38000670A1092660A1092650A1092640A109267
:10C390008E0210928D02E0918F02F0919002A0E047
:10C3A000B1E094E080EC8A0F9D938A13FDCF249135
:10C3B0006F017FEFC71AD70A422F022E000C550BD0
:10C3C000407F552764E0559547956A95E1F72F70B2
:10C3D00081E0820F6AE070E0681B710977FF02C09C
:10C3E0006F5F7F4F759567958FE090E031E0340F78
:10C3F000831B910997FD019695958795260F480F08
:10C400000E941A60F6018491082F082E000C110B6F
:10C41000007F112794E0159507959A95E1F78F70A5
:10C4200089830E3011056CF4F02FF770FF2E8F2FDB
:10C430000E9427600830110534F08F2D0E9427607C
:10C4400002C00E947A6079817E3064F47770F72EA2
:10C45000872F0E9427607981783034F08F2D0E94D9
:10C46000276002C00E947A608FEFC81AD80A0F3086
:10C47000110549F48091630A509182024091680A43
:10C480006091910215C079817F3009F0BBCFF2CF66
:10C49000F90170E1979FE00DF11D1124E050FF4F6D
:10C4A0007081743009F410829F5F691788F78F5F7D
:10C4B000581720F0942F282F30E0F7CF8091870273
:10C4C000909188020E94E56080938002D09284025D
:10C4D000C09283020F90DF91CF911F910F91FF9037
:10C4E000DF90CF900C9483611092880210928702A3
:10C4F00084EE99E39093900280938F0210928C02C5
:10C5000010928B0210928A021092890208958091F3
:10C510008702909188020196909388028093870207
:10C5200020918302309184023093900220938F02F5
:10C53000873E934010F00C9474620895CF93DF937C
:10C5400061E081E00E945A54C0918702D091880234
:10C55000209711F0219702C0C6EED3E00E947462CA
:10C5600080918702909188028C179D0728F40E9481
:10C57000B1610E948762F4CF0E94B16160EC83E2F6
:10C58000DF91CF910C945A54CF93DF9380918D0219
:10C5900090918E02009709F46CC02091640A30914A
:10C5A000650A2115310519F02150310902C027EE25
:10C5B00033E03093650A2093640A019790938E02CA
:10C5C00080938D02E091640AF091650AEE0FFF1FDF
:10C5D000ED56FD4FC081D0E0C050DF4FE1810E2EFF
:10C5E000000CFF0B9E012E0F3F1FE20FF31F80E098
:10C5F00091E0DC0101964C914650423030F041E030
:10C60000803C9407B0F3A0E0B0E08C9186508C930E
:10C6100088818A5F8883808182508083F90180814C
:10C620008E5F80838091850290918602019690931F
:10C6300086028093850280918B0290918C020196F4
:10C6400090938C0280938B028091660A9091670A86
:10C6500001979093670A8093660A8091890290916E
:10C660008A02019790938A0280938902DF91CF9189
:10C670000895DF91CF910C94B1615F926F927F9298
:10C680008F929F92AF92BF92CF92DF92EF92FF92E2
:10C690000F931F93CF93DF93E0E0F1E094E080EC01
:10C6A0008E0F91938E13FDCF94E6C92ED12C20E2EC
:10C6B000A22EB12C34E0532E2091870230918802B3
:10C6C000C901B6010E946966C62F81E0809392027B
:10C6D0001092810263E0C90101960E944C6024E639
:10C6E000C29FE001112485010C1B1D0B00501F4F40
:10C6F00066246394712CF62C84E0860D809392025C
:10C70000109281028AE0681203C080E090E001C0CC
:10C71000C30161E00E944C6081E080939202F39437
:10C72000F092810263E0CE010E944C604E01EAE08B
:10C730008E0E911C7801EC0EFD1EC73EF3E0DF0764
:10C74000DCF48091870290918802C817D90749F4D8
:10C75000CE010E94E560811102C087E10AC088E134
:10C7600008C0CE010E94E560811102C085E101C0D0
:10C7700086E1F701858302C0F70155822196C8152D
:10C78000D905C1F60A5F1F4FFFEF6F1A7F0A2BE032
:10C790006216710409F0AFCF80E00E942F54892BFC
:10C7A000D9F780E00E942F54EC010097D1F384FF69
:10C7B00018C0809187029091880240E06FEF0A973D
:10C7C00068F084E00E944E5980918702909188021F
:10C7D0000A97909388028093870203C082E00E94A8
:10C7E0004E59C5FF19C0809187029091880240E0A0
:10C7F0006FEF8D3D934068F484E00E944E59809124
:10C800008702909188020A9690938802809387020B
:10C8100003C082E00E944E59C6FF18C08091870273
:10C820009091880240E06FEF892B69F084E00E94CC
:10C830004E598091870290918802019790938802C7
:10C840008093870203C082E00E944E59C7FF19C03F
:10C85000809187029091880240E06FEF863E93407E
:10C8600068F484E00E944E5980918702909188027A
:10C870000196909388028093870203C082E00E9411
:10C880004E59D2FF1AC0809187029091880240E0F1
:10C890006FEF8436910570F084E00E944E598091CC
:10C8A0008702909188028456910990938802809320
:10C8B000870203C082E00E944E59D3FF1AC08091C4
:10C8C00087029091880240E06FEF8338934070F4C4
:10C8D00084E00E944E5980918702909188028C5981
:10C8E0009F4F909388028093870203C082E00E944A
:10C8F0004E59CB70D370CD2B09F4DECE40E06FEFF4
:10C9000080E00E944E5961E081E00E945A540091FB
:10C910008702109188020E947462C0E0D0E0C017C4
:10C92000D10731F00E94B1610E9487622196F7CF52
:10C930000E94B16180918702909188020E942461D7
:10C9400060EC83E2DF91CF911F910F91FF90EF9008
:10C95000DF90CF90BF90AF909F908F907F906F901F
:10C960005F900C945A5440E06FEF83E00E944E5960
:10C970008CE390E00C9403600E94746261E081E0BB
:10C980000E945A540E9459618C01C0E0D0E0C01747
:10C99000D10731F00E94B1610E9487622196F7CFE2
:10C9A0000E94B16160EC83E20E945A5458EEE52E79
:10C9B00053E0F52EAA24A39480E00E942F54892BE3
:10C9C000D9F780E00E942F54EC010097D1F387FF44
:10C9D00003C0BB24B39402C0BB24BA94C4FF02C0FA
:10C9E00040EFB42EC5FF02C030E1B32ED0FF0FC020
:10C9F000809185029091860240E06FEF892B11F4BF
:10CA000082E001C084E00E944E590E94B161C0FFE3
:10CA10000FC0809185029091860240E06FEF892BD4
:10CA200011F482E001C084E00E944E590E94C46269
:10CA3000D1FF0FC040E06FEF84E00E944E590E948A
:10CA400087620E94B16180918702909188020E9462
:10CA50002461C1FF0DC040E06FEF84E00E944E5999
:10CA60000E949E6280918702909188020E942461B8
:10CA7000C2FD0E943D63C07FDD27CD2B09F48DC030
:10CA800080E091E0EC01019628812650223030F0C0
:10CA900041E0803C9407B0F3C0E0D0E0CB2C0B2CFD
:10CAA000000CDD088E010C0D1D1DC00ED11EF801FD
:10CAB0008081823040F0843008F06AC0F6018081C5
:10CAC000823008F065C080918B0290918C020196B3
:10CAD00090938C0280938B028091850290918602C4
:10CAE0000196909386028093850288818650888380
:10CAF000F801808140E06FEF823008F441C081E0AE
:10CB00000E944E598091640A9091650AFC01EE0FD3
:10CB1000FF1FED56FD4FC050D140C083B182209120
:10CB20008D0230918E02283E43E0340730F42F5FAF
:10CB30003F4F30938E0220938D020196B7010E94E1
:10CB400069669093650A8093640A80918902909146
:10CB50008A02019690938A02809389028091660AE4
:10CB60009091670A01969093670A8093660AF8018C
:10CB7000808182508083F60180818E5F808303C034
:10CB800080E00E944E59F80180818A5F808305C051
:10CB900040E06FEF82E00E944E590E948361E0E026
:10CBA000F1E08191823009F407CF21E0E03CF20707
:10CBB000C0F3A092800280918702909188020E9427
:10CBC0008C600E9483610E94B3640E9487620E940D
:10CBD000B16180918702909188020E942461ECCE1D
:10CBE0008F929F92AF92BF92CF92DF92EF92FF927D
:10CBF0000F931F93CF93DF93FA0184903196949013
:10CC0000A82CB12C90E0F0E16F9F800D911D1124B4
:10CC100000E010E0C0E0D0E030E0391509F1680133
:10CC2000C80ED91EA0E0B0E07E0162E0E60EF11C65
:10CC3000A81580F4B7016A0F7B1FFA01E60FF71FF2
:10CC40006491FD01EC0DFD1DE050FF4F620F60830C
:10CC50001196EECF3F5FCA0DDB1D005F1F4FDDCF8A
:10CC6000DF91CF911F910F91FF90EF90DF90CF90C8
:10CC7000BF90AF909F908F90089580EE90E00E94BB
:10CC8000205486E293EA0E9459562AE140E658E38E
:10CC900060E080E00E94F06580E00E942F54892BC4
:10CCA000D9F780E00E942F54892BD9F32AE142E280
:10CCB00059E360E080E00E94F06580E00E942F541C
:10CCC000892BD9F780E00E942F54892BD9F30E9439
:10CCD000BC64AA1BBB1B51E107C0AA1FBB1FA61740
:10CCE000B70710F0A61BB70B881F991F5A95A9F715
:10CCF00080959095BC01CD01089597FB072E16F401
:10CD0000009407D077FD09D00E94696607FC05D022
:10CD10003EF4909581959F4F0895709561957F4F52
:06CD20000895F894FFCF16
:00000001FF
